:100000000C9434290C94BC4E0C94914E0C94664E76
:100010000C943B4E0C94104E0C94E54D0C94BA4D40
:100020000C948F4D0C9465290C9465290C946529CA
:100030000C9465290C943E4F0C9465290C94652909
:100040000C9465290C948DDB0C9465290C9465291E
:100050000C9465290C9465290C94F6970C94265100
:100060000C9465290C94A2A20C943CA30C946529D1
:100070000C9465290C9465290C9465290C946529C8
:100080000C9465290C9465290C9465290C946529B8
:100090000C9465290C9465290C9465290C946529A8
:1000A0000C9465290C9465290C9465290C94652998
:1000B0000C9465290C9465290C9465290C94652988
:1000C0000C9465290C9465290C9465290C94652978
:1000D0000C9465290C9465290C9465290C94652968
:1000E0000C9465292B492E491D4921492749654909
:1000F000324936493C49404944494A494E495249A6
:10010000654958495C496049035008500D501750E3
:1001100021509A502B5033503B5045504F5059501E
:10012000685072509A507C5086509050D5A2DBA2F5
:10013000ECA2F7A2FFA214A303A314A307A30BA38B
:1001400014A311A3E200E200DC00DC00DC00DE000E
:10015000DE00DE00E400D600D600D600084AD73B19
:100160003BCE016E84BCBFFDC12F3D6C74319ABD86
:1001700056833DDA3D00C77F11BED9E4BB4C3E91AA
:100180006BAAAABE000000803F05A84CCDB2D44E99
:10019000B93836A9020C50B9918688083CA6AAAA9B
:1001A0002ABE000000803F000D945A180D94DA27F3
:1001B0000D947E170D94DC190D94CC270D94D32744
:1001C0000D94C71D0D94C5270D94E0274E414E494F
:1001D0004E495459494E46CDCCCC3D0AD7233C1705
:1001E000B7D13877CC2B329595E6241FB14F0A0052
:1001F0000020410000C84200401C4620BCBE4CCA42
:100200001B0E5AAEC59D7420746F6F206C6F6E67A5
:1002100020657874727573696F6E2070726576658B
:100220006E7465640A0020636F6C64206578747274
:100230007573696F6E2070726576656E7465640A99
:100240000047322F47332062616420706172616D14
:1002500065746572730A00536C6565702E2E2E00EE
:1002600050726F62696E67206661696C6564004DEB
:1002700031313720426564206C6576656C696E6744
:10028000206661696C65642E0A4730205A31300A55
:1002900047302045300A4D3330302050323520531E
:1002A0003838300A4D333030205035302053300A42
:1002B0004D3330302050323520533838300A4D33EA
:1002C0003030205035302053300A4D3330302050FC
:1002D000323520533838300A4734205331004D31FD
:1002E00031372050726F6265207375636365737375
:1002F00066756C0A0050524F4245204641494C20D9
:10030000434C45414E204E4F5A5A4C450A004D3100
:100310003137204C6576656C696E672058204178CE
:1003200069730A4732380A47302058313630204640
:10033000393939390A4730205A352046363030307D
:100340000A4739310A4D3231312053300A4D3430A9
:10035000300A4D393036205A3630300A4730205A6C
:100360002D313520463530300A4730205A35204669
:100370003530300A4739300A4D3430300A4D393083
:1003800036205A3936300A4D3231312053310A4D38
:100390003430300A4732380A4D313137204C6576D7
:1003A000656C696E6720646F6E652E0A4D3131375A
:1003B000205265776970696E67206E6F7A7A6C6516
:1003C0000A473132205030205331322054300A4D08
:1003D0003131372050726F62696E67206265640048
:1003E000205A3A200020593A200042656420583AA9
:1003F0002000526573756D696E67207072696E7446
:10040000004D696E6920322072656164792E004367
:100410006C69636B20746F20726573756D652E2E29
:100420002E004E6F206D6F76652E004D31323500F7
:1004300046696C652064656C657465643A00446562
:100440006C6574696F6E206661696C65642C20460A
:10045000696C653A20006F70656E206661696C6535
:10046000642C2046696C653A20005072696E7420D5
:1004700074696D653A200042656420646F6E652E74
:100480000020573A004265642068656174696E67B0
:100490002E0042656420636F6F6C696E672E004C9E
:1004A000756C7A426F742048696269736375732052
:1004B0004F66662E0053657474696E6720547261CE
:1004C00076656C20416363656C65726174696F6EFB
:1004D0003A200053657474696E67205265747261C6
:1004E000637420416363656C65726174696F6E3A11
:1004F000200053657474696E67205072696E7420B1
:10050000416363656C65726174696F6E3A20005374
:10051000657474696E67205072696E7420616E64D0
:100520002054726176656C20416363656C6572610D
:1005300074696F6E3A2000205A002059005800203C
:10054000204D61783A2000205A00205900580020A0
:10055000204D696E3A20004F6E20004F66660053B2
:100560006F667420656E6473746F70733A20005008
:10057000726F6265205A204F66667365743A200078
:1005800020643A0020693A0020703A0043290A00AA
:1005900061626C656420286D696E2074656D7020E1
:1005A00000436F6C642065787472756465732061B4
:1005B000726520004B64200023646566696E6520C7
:1005C0002044454641554C545F004B69200023644C
:1005D0006566696E65202044454641554C545F0070
:1005E0004B70200023646566696E65202044454693
:1005F00041554C545F00504944204175746F7475E7
:100600006E652066696E6973686564212050757433
:1006100020746865206C617374204B702C204B69CA
:1006200020616E64204B6420636F6E7374616E741E
:10063000732066726F6D2062656C6F7720696E74CF
:100640006F20436F6E66696775726174696F6E2E95
:10065000680A00504944204175746F74756E6520B6
:100660006661696C6564212074696D656F75740AD3
:1006700000544845524D414C2052554E4157415926
:1006800000546865726D616C2052756E6177617996
:100690000048656174696E67206661696C65640015
:1006A00048656174696E67206661696C65640050B5
:1006B0004944204175746F74756E65206661696C7C
:1006C0006564212054656D70657261747572652072
:1006D000746F6F20686967680A00204B643A2000D5
:1006E000204B693A2000204B703A20000A20436CCE
:1006F000617373696320504944200A002054753A9D
:100700002000204B753A2000206D61783A200020AF
:100710006D696E3A200020643A200020626961739E
:100720003A2000426564204C6576656C696E6720EE
:10073000004661696C656420746F20656E61626C4F
:100740006520426564204C6576656C696E670A00B9
:10075000426564204C6576656C20436F72726563F8
:1007600074696F6E204D61747269783A00202020A0
:1007700020202846312E30203D2066756C6C206389
:100780006F7272656374696F6E2C2046302E302054
:100790003D206E6F20636F7272656374696F6E299E
:1007A0000A002020466164653A2020202020202075
:1007B0002020202020202020202046002020536DB3
:1007C0006F6F7468696E6720286D6D293A2020204C
:1007D000202020205300202044697374616E6365DB
:1007E00020286D6D293A20202020202020205A002A
:1007F0004261636B6C61736820636F7272656374CE
:10080000696F6E206973206163746976653A0A00C6
:100810004261636B6C61736820636F7272656374AD
:10082000696F6E20697320696E6163746976653AD9
:100830000A004261636B6C617368206D656173755A
:1008400072656D656E7420286D6D293A2020004117
:1008500063746976652045787472756465723A20B0
:1008600000556E6B6E6F776E20636F6D6D616E6499
:100870003A202200000020002300260029002C003E
:100880002F003200000100000301060109010225CA
:1008900069730025696D2025697300256968202525
:1008A000696D202569730025696420256968202504
:1008B000696D2025697300256979202569642025E3
:1008C00069682025696D20256973007A5F6D6178FC
:1008D0003A20007A5F6D696E3A2000795F6D617829
:1008E0003A2000785F6D696E3A20005265706F7231
:1008F00074696E6720656E6473746F7020737461C1
:100900007475730A001FFFFFFFFFFFFF6000000008
:100910000001FF400000000000FF80000000000018
:100920007F83CF00000C303F87FF80000C301F8694
:100930007980000C000F8C30C7838C30E78C30CF6F
:10094000C7CC31F38C30DCECEC33B98C30D86C6C28
:1009500033198C30D06C0C33198C30D86C0C3319A3
:100960008C30DC6C0E3B198C30CF7C079F198C309F
:10097000C77C038F194000000000000260000000E7
:100980000000061FFFFFFFFFFFF82020506C616E84
:100990006E657242756666657242797465733A2057
:1009A000002046726565204D656D6F72793A2000B2
:1009B000436F6D70696C65643A204A756C20333101
:1009C00020323031380A00207C20417574686F7203
:1009D0003A2028416C657068204F626A65637473C1
:1009E00020496E632E2C204C756C7A426F74204720
:1009F0006974205265706F7369746F7279290A0087
:100A00004A756C203331203230313830383A303644
:100A10003A333400204C61737420557064617465FE
:100A2000643A2000312E312E380A004D61726C6913
:100A30006E0020536F66747761726520526573652E
:100A4000740A00205761746368646F67205265738D
:100A500065740A002042726F776E206F75742052A1
:100A6000657365740A002045787465726E616C2048
:100A700052657365740A00506F77657255700A008D
:100A800073746172740A006572726F722077726992
:100A900074696E6720746F2066696C650A00456E24
:100AA0006473746F70732025632025632025632091
:100AB000256300205A3A0020593A0020583A006530
:100AC0006E6473746F7073206869743A2000446FA9
:100AD0006E6520736176696E672066696C652E0AA3
:100AE000004D3239002F2F20004F666673657473F6
:100AF000206170706C696564004572723A20546FB1
:100B00006F206661722100546F6F206661722066EB
:100B1000726F6D207265666572656E636520706FB9
:100B2000696E740A003A2000207A5F6D696E3A207F
:100B3000202D32207A5F6D61783A2020350A0050EE
:100B4000726F6265205A204F666673657400417546
:100B5000746F0020452F443D00416476616E6365EB
:100B6000204B3D004E6F2063617365206C696768A0
:100B7000740A003048483025753A25303275002512
:100B80003032753A25303275001A0025336400255D
:100B90003464002520200025200020706F736974C4
:100BA000696F6E206F7574206F662072616E676565
:100BB0002E0A003F50726F626520000A0A42656487
:100BC000204C6576656C20436F7272656374696F43
:100BD0006E204D61747269783A00202B000A436FD1
:100BE0007272656374656420426564204865696754
:100BF00068742076732E2042656420546F706F6C89
:100C00006F67793A0A00202B000A42656420486524
:100C10006967687420546F706F6772617068793AA1
:100C20000A2020202B2D2D2D204241434B202D2DFD
:100C30002B0A2020207C2020202020202020202063
:100C4000207C0A204C207C20202020282B292020BA
:100C500020207C20520A2045207C2020202020209B
:100C600020202020207C20490A2046207C20282D7E
:100C700029204E20282B29207C20470A2054207C24
:100C800020202020202020202020207C20480A20F6
:100C900020207C20202020282D29202020207C207E
:100CA000540A2020207C20202020202020202020CA
:100CB000207C0A2020204F2D2D2046524F4E5420BC
:100CC0002D2D2B0A2028302C30290A004D65616E0D
:100CD000206F662073616D706C656420706F696E43
:100CE00074733A200020643A200020623A200045C4
:100CF000716E20636F656666696369656E74733AC9
:100D000020613A20003474682070726F6265207030
:100D10006F696E742C2064697374616E63652066FC
:100D2000726F6D20706C616E653A2000202844520D
:100D30005952554E2900473239204175746F20426F
:100D40006564204C6576656C696E67002842296190
:100D5000636B00284629726F6E74002852296967F8
:100D6000687400284C29656674003F4E756D626595
:100D700072206F662070726F626520706F696E748A
:100D80007320697320696D706C61757369626C653D
:100D9000202832206D696E696D756D292E0A003F1D
:100DA0002856296572626F7365206C6576656C20C4
:100DB000697320696D706C61757369626C65202858
:100DC000302D34292E0A004D36303020423000506C
:100DD00072696E7420706175736564004D313235CF
:100DE00000004D3234005072696E742061626F727F
:100DF000746564004E6F2053442063617264005038
:100E000072696E742066726F6D2053440053746F64
:100E100070207072696E7400526573756D65207014
:100E200072696E740041626F7574204669726D77E5
:100E3000617265005061757365207072696E74002F
:100E40004368616E67652066696C616D656E7400EC
:100E5000436F6E66696775726174696F6E00546581
:100E60006D7065726174757265004D6F76656D6544
:100E70006E740054756E6500496E666F2073637200
:100E800065656E004D6F7665206178697300446911
:100E90007361626C65207374657070657273004D68
:100EA0003834004C6576656C2058204178697300B1
:100EB0004D313137204C6576656C696E672058205E
:100EC000417869730A4732380A4730205831363042
:100ED0002046393939390A4730205A3520463630CC
:100EE00030300A4739310A4D3231312053300A4D02
:100EF0003430300A4D393036205A3630300A4730D7
:100F0000205A2D313520463530300A4730205A35A9
:100F100020463530300A4739300A4D3430300A4DDA
:100F2000393036205A3936300A4D3231312053317A
:100F30000A4D3430300A4732380A4D313137204CAF
:100F40006576656C696E6720646F6E652E0041750D
:100F5000746F20686F6D6500473238004D61696EAF
:100F6000004D3530320A4D353030004C6F61642011
:100F700073657474696E677300526573746F72651C
:100F8000206661696C736166650053746F726520D9
:100F900073657474696E677300416476616E63652E
:100FA000642053657474696E6773004D61696E00E7
:100FB00020737465616C746843686F70206D61782C
:100FC0002073706565642073657420746F20002041
:100FD00064726976657220686F6D696E67207365EB
:100FE0006E73697469766974792073657420746F9F
:100FF0002000656E7175657565696E672022002039
:10100000643A0020693A0020703A002F2F6163741F
:10101000696F6E3A726573756D650A004D363030D2
:1010200020486F74656E6420746F6F20636F6C640A
:1010300020746F206368616E67652066696C616DFE
:10104000656E740A002F2F616374696F6E3A706168
:101050007573650A004572726F72207772697469E0
:101060006E6720746F20454550524F4D210A00296C
:101070000A002062797465733B2063726320005319
:10108000657474696E67732053746F726564202889
:10109000004F6666004F6E2000456E6473746F707B
:1010A0002061626F72740053746570732F6D6D00F0
:1010B0004A65726B00416363656C65726174696F48
:1010C0006E0056656C6F63697479005A204F6666CE
:1010D00073657400416476616E6365642053657462
:1010E00074696E67730043616E6E6F7420656E7411
:1010F0006572207375626469723A2000022E2E00B8
:101100004D61696E0020204E6F7A7A6C653A20003E
:1011100020004261636B004D696E696D756D2054EE
:10112000656D70206973203132302E00486561741E
:10113000696E67206661696C6564004578747275D4
:101140006465206D6F726500526573756D65207002
:1011500072696E7400524553554D45204F505449A5
:101160004F4E533A0020204E6F7A7A6C653A200039
:101170006368616E6765006F6620746865206669E4
:101180006C616D656E74005761697420666F7220C2
:101190007374617274005052494E5420504155533B
:1011A00045440020204E6F7A7A6C653A200020007A
:1011B00066696C616D656E7420756E6C6F6164003C
:1011C0005761697420666F72005052494E54205026
:1011D00041555345440020204E6F7A7A6C653A2081
:1011E000002000506C6561736520776169742E2E54
:1011F0002E0048656174696E67206E6F7A7A6C653F
:10120000005052494E54205041555345440020202F
:101210004E6F7A7A6C653A20002000686561742010
:101220006E6F7A7A6C652E005072657373206275EA
:1012300074746F6E20746F005052494E54205041A8
:10124000555345440020204E6F7A7A6C653A200051
:10125000746F20636F6E74696E75652E2E2E00613B
:101260006E6420707265737320627574746F6E00A3
:10127000496E736572742066696C616D656E740089
:101280005052494E54205041555345440020204E61
:101290006F7A7A6C653A2000200066696C616D6532
:1012A0006E74206C6F6164005761697420666F72A0
:1012B000005052494E54205041555345440020207F
:1012C0004E6F7A7A6C653A2000200066696C616D19
:1012D000656E742065787472756465005761697411
:1012E00020666F72005052494E542050415553456C
:1012F0004400000040C000004043000037430000AD
:1013000048420000484200002042000000005761AF
:10131000726E696E673A20486F6D696E672042751C
:101320006D702044697669736F72203C20310A0029
:101330000202040000000000000000000000400065
:101340000026430000454300003743FF010162656A
:10135000640A002C2073797374656D2073746F7048
:1013600070656421204865617465725F49443A2064
:101370000048656174696E67206661696C65642008
:101380004245440048656174696E67206661696C16
:1013900065640048656174696E67206661696C65A3
:1013A000640048656174696E67206661696C656494
:1013B000204530001000AD0330016A0150022B01BE
:1013C00070030A019004F500B005E500D006D800CE
:1013D000F007CE001009C500300ABE00500BB70060
:1013E000700CB100900DAB00B00EA600D00FA200A3
:1013F000F0109D00101299003013950050149200C7
:1014000070158E0090168B00B0178700D0188400DE
:10141000F0198100101B7E00301C7B00501D7900EC
:10142000701E7600901F7300B0207000D0216E00F7
:10143000F0226B00102469003025660050266300FE
:101440007027610090285E00B0295C00D02A590006
:10145000F02B5600102D5400302E5100502F4E000E
:1014600070304B0090314800B0324500D03342001C
:10147000F0343E0010363B00303737005038330030
:1014800070392E00903A2900B03B2300D03C1B005D
:10149000F03D1100103F0100F03F00004572723A2C
:1014A000204D494E54454D5020424544004D494E33
:1014B00054454D50207472696767657265640045D4
:1014C00072723A204D494E54454D502045310045E9
:1014D00072723A204D494E54454D502045300045DA
:1014E00072723A204D415854454D502042454400B7
:1014F0004D415854454D5020747269676765726557
:1015000064004572723A204D415854454D50204573
:1015100031004572723A204D415854454D50204596
:1015200030004B494C4C45442E2000746F207265AE
:1015300073756D65005761697420666F72207072F3
:10154000696E74005052494E5420504155534544E1
:10155000000000007E006000600060F87ECC60CC7F
:1015600060CC60F860CC00CC00CC00CC0000000067
:10157000000000000000000000000000000000006B
:1015800000000000000000FE7FFE7F0660000000FB
:101590000000000000F00FF81FF81FF81FF00FF018
:1015A0000FF81FF81FF81FE007C0038001000000BC
:1015B000000000FE7F0E702664724E7A5E324C820E
:1015C00041324C7A5E724E26640E70FE7F0000003F
:1015D000000000FE7F0E70C663C24382411A58BAF3
:1015E0005D1A588241C243C6630E70FE7F00000040
:1015F000000000880888081011202220221011887D
:101600000888081011000000000000000000000021
:1016100000000020221011880888081011202220C4
:1016200022101188080000000000000000000000E7
:1016300000436172642072656D6F7665640043617A
:10164000726420696E7365727465640020202020C6
:10165000004C696E65204E756D626572206973205D
:101660006E6F74204C617374204C696E65204E75EA
:101670006D6265722B312C204C617374204C696E45
:10168000653A200053544F505045442E200050726C
:10169000696E7465722073746F7070656420647510
:1016A0006520746F206572726F72732E20466978A0
:1016B00020746865206572726F7220616E64207597
:1016C0007365204D39393920746F207265737461E8
:1016D00072742E202854656D706572617475726520
:1016E0002069732072657365742E205365742069B8
:1016F00074206166746572207265737461727469B6
:101700006E67290A004E6F20436865636B73756DC1
:101710002077697468206C696E65206E756D6265EE
:10172000722C204C617374204C696E653A20006302
:101730006865636B73756D206D69736D6174636843
:101740002C204C617374204C696E653A20004D3139
:101750003130004D3331005344207265616420659F
:1017600072726F720A00446F6E65207072696E74D7
:10177000696E672066696C650A0020496E76616C47
:101780006964206578747275646572200000004099
:10179000C00000A0C0000000000000234300004083
:1017A0004300003743486F6D65202573257325730B
:1017B000206669727374002066697273740A005A35
:1017C0000059005800486F6D652000436F6F6C64CE
:1017D0006F776E0046616E207370656564004661C8
:1017E0006E20737065656400426564004265640044
:1017F0004E6F7A7A6C65004E6F7A7A6C65004D6137
:10180000696E005654726176206D696E005654728E
:101810006176206D696E005654726176206D696E36
:1018200000566D696E00566D696E00566D696E00EA
:10183000566D6178204500566D6178204500566DE3
:101840006178204500566D6178205A00566D6178A8
:10185000205A00566D6178205A00566D61782059E3
:1018600000566D6178205900566D617820590056F8
:101870006D6178205800566D6178205800566D6172
:10188000782058004D6F74696F6E00416D6178204B
:101890004500416D6178204500416D6178205A0016
:1018A000416D6178205A00416D6178205900416D89
:1018B0006178205900416D6178205800416D617850
:1018C000205800412D74726176656C00412D747250
:1018D0006176656C00412D726574726163740041BC
:1018E0002D7265747261637400416363656C0041BD
:1018F0006363656C004D6F74696F6E0056652D6A89
:1019000065726B0056652D6A65726B0056652D6AAF
:1019100065726B00567A2D6A65726B00567A2D6A75
:1019200065726B0056792D6A65726B0056792D6A67
:1019300065726B0056792D6A65726B0056782D6A58
:1019400065726B0056782D6A65726B0056782D6A49
:1019500065726B004D6F74696F6E004573746570CE
:10196000732F6D6D004573746570732F6D6D005A24
:1019700073746570732F6D6D005A73746570732F77
:101980006D6D005973746570732F6D6D00597374AC
:101990006570732F6D6D005873746570732F6D6D66
:1019A000005873746570732F6D6D004D6F74696F9F
:1019B0006E0020746F6F206C6F6E67206578747294
:1019C0007573696F6E2070726576656E7465640AF2
:1019D0000020636F6C6420657874727573696F6E34
:1019E0002070726576656E7465640A00434F4D4DD4
:1019F000554E49434154494F4E0044525952554E59
:101A0000004552524F525300494E464F00454348FD
:101A10004F006D0046696C616D656E74207573656D
:101A2000643A200053746174733A20002C204C6F88
:101A30006E67657374206A6F623A2000546F746138
:101A40006C2074696D653A200053746174733A2098
:101A5000002C204661696C65643A20002C204669A0
:101A60006E69736865643A20005072696E74733AE7
:101A7000200053746174733A200045787472756461
:101A80006572202573006F6B00436F6F6C696E6722
:101A900020646F6E652E0048656174696E6720640E
:101AA0006F6E652E0020573A004578747275646534
:101AB00072202573000D1A081A011AFA19EC196F11
:101AC00066660044454255473A004D31343520534F
:101AD0003C696E6465783E206F7574206F66207275
:101AE000616E67652028302D31290A00205A3A009E
:101AF00020593A0020436F756E7420583A002045F3
:101B00003A00205A3A0020593A00583A003A004325
:101B100061703A00454D455247454E43595F50412B
:101B20005253455200434153455F4C494748545F27
:101B30004252494748544E45535300544F47474C2F
:101B4000455F4C494748545300534F465457415200
:101B5000455F504F574552004255494C445F5045F0
:101B60005243454E54004C4556454C494E475F4400
:101B7000415441005A5F50524F4245004155544F25
:101B80004C4556454C005052494E545F4A4F420016
:101B900050524F4752455353004155544F524550B0
:101BA0004F52545F54454D5000564F4C554D45547F
:101BB00052494300454550524F4D0053455249410B
:101BC0004C5F584F4E5F584F4646004649524D575E
:101BD0004152455F4E414D453A4D61726C696E20F0
:101BE000204649524D574152455F56455253494F41
:101BF0004E3A312E312E382E363620455854525515
:101C00004445525F545950453A4165726F7374723E
:101C10007564657220534F555243455F434F4445A9
:101C20005F55524C3A68747470733A2F2F636F6427
:101C3000652E616C6570686F626A656374732E638C
:101C40006F6D2F646966667573696F6E2F4D4152B3
:101C50004C494E2050524F544F434F4C5F564552C3
:101C600053494F4E3A312E30204D414348494E455D
:101C70005F545950453A4C756C7A426F74204869EC
:101C80006269736375732045585452554445525FD9
:101C9000434F554E543A3120555549443A653535F0
:101CA00030323431312D643436642D343231642D88
:101CB000626133612D61323031323664373933300D
:101CC000660A0024F4D43050C38E20C2A24017828A
:101CD0008B7011127A910D816CD90AA861E108C745
:101CE000586607615143061E4B5D05C145A7041A9E
:101CF000411104093D9803713931034036DB026517
:101D0000339102D4305402802E1D02632CEE0175F3
:101D10002AC501B028A001102781018F2564012B5D
:101D2000244B01E0223401AC211F018D200D0180E4
:101D30001FFC00841EED00971DDF00B81CD200E6DA
:101D40001BC600201BBC00641AB200B219A8000A0E
:101D500019A0006A189900D117910040178B00B59F
:101D600016840031167E00B31579003A157300C74A
:101D7000146F0058146A00EE136600881363002580
:101D8000135E00C7125B006C12570015125400C19D
:101D900011510070114F0021114B00D61049008DD8
:101DA0001047004610440002104200C00F4000805F
:101DB0000F3E00420F3C00060F3B00CB0E38009355
:101DC0000E37005C0E3500270E3400F30D3200C1D3
:101DD0000D3100900D3000600D2E00320D2D0005EC
:101DE0000D2C00D90C2B00AE0C2900850C29005CB1
:101DF0000C2700350C27000E0C2600E80B2400C42D
:101E00000B2400A00B23007D0B23005A0B2100396B
:101E10000B2100180B2000F80A1F00D90A1E00BB76
:101E20000A1E009D0A1D00800A1D00630A1C00474F
:101E30000A1B002C0A1B00110A1A00F7091A00DD00
:101E4000091900C4091900AB091900920917007B90
:101E5000091800630917004C0916003609160020FE
:101E60000916000A091500F5081500E0081400CC51
:101E7000081400B8081400A4081400900813007D8A
:101E80000812006B081300580812004608120034AC
:101E9000081100230811001208110001081100F0B8
:101EA000071000E0071000D0071000C0071000B0B6
:101EB000070F00A107100091070E0083070F0074A1
:101EC000070F0065070E0057070E0049070E003B7D
:101ED000070D002E070E0020070D0013070D00064A
:101EE000070D00F9060C00ED060D00E0060C00D40D
:101EF000060C00C8060C00BC060C00B0060C00A4C2
:101F0000060B0099060C008D060B0082060B00776D
:101F1000060B006C060B0061060A0057060B004C0E
:101F2000060A0042060A0038060A002E060A0024A5
:101F3000060A001A060A001006090007060A00FD34
:101F4000050900F4050900EB050900E2050900D9BF
:101F5000050900D0050900C7050900BE050900B53F
:101F6000050800AD050800A50509009C05080094BA
:101F70000508008C050800840508007C050800742D
:101F80000508006C050700650508005D050700569B
:101F90000508004E05070047050700400508003802
:101FA000050700310507002A050700230507001C67
:101FB000050600160507000F0507000805060002C4
:101FC000050700FB040600F5040700EE040600E820
:101FD000040600E2040700DB040600D5040600CF77
:101FE000040600C9040600C3040600BD040600B7C9
:101FF000040600B1040500AC040600A6040600A017
:102000000405009B04060095040500900406008A60
:1020100004050085040500800406007A04050075A7
:10202000040500700405006B0405006604050061EA
:102030000405005C04050057040500520405004D2A
:1020400004050048040500430405003E0404003A6A
:1020500004050035040500300404002C04050027A5
:10206000040400230405001E0404001A04040016DE
:10207000040500110404000D040400090405000413
:1020800004040000040400FC030400F8030400F44A
:10209000030400F0030400EC030400E8030400E47C
:1020A000030400E0030400DC030400D8030400D4AC
:1020B000030400D0030400CC030400C8030300C5DC
:1020C00003030024F404D9201BC40C5C0E9804C440
:1020D000095F0265077101F405F900FB04B30048CC
:1020E000048700C10369005803550003034500BE7F
:1020F000023A008402310053022A0029022500041A
:10210000022000E4011C00C8011900AF011700986B
:1021100001140084011300710110006101100051CD
:10212000010E0043010D0036010B002B010B0020B6
:10213000010B00150109000C01090003010800FB57
:10214000000800F3000800EB000700E4000600DED2
:10215000000600D8000600D2000600CC000500C72B
:10216000000500C2000500BD000400B9000400B570
:10217000000400B1000400AD000400A9000400A5A3
:10218000000300A20003009F0004009B00030098CE
:102190000003009500020093000300900003008DEF
:1021A0000002008B00030088000200860002008409
:1021B000000300810002007F0002007D0002007B1E
:1021C000000200790002007700010076000200742E
:1021D00000020072000100710002006F0002006D39
:1021E0000001006C0002006A000100690002006743
:1021F0000001006600010065000100640002006249
:1022000000010061000100600001005F0002005D4C
:102210000001005C0001005B0001005A0001005950
:102220000001005800010057000100560001005550
:10223000000100540001005300000053000100524F
:1022400000010051000100500001004F0001004E4C
:102250000000004E0001004D0001004C0001004B49
:102260000000004B0001004A000100490001004845
:102270000000004800010047000100460000004641
:10228000000100450000004500010044000100433A
:102290000000004300010042000000420001004134
:1022A00000000041000100400001003F0000003F2D
:1022B0000001003E0000003E0001003D0000003D26
:1022C0000001003C0000003C0000003C0001003B1D
:1022D0000000003B0001003A0000003A0001003914
:1022E000000000390001003800000038000000380C
:1022F0000001003700000037000100360000003602
:1023000000000036000100350000003500000035F7
:1023100000010034000000340000003400010033EC
:1023200000000033000000330001003200000032E2
:1023300000000032000100310000003100000031D7
:102340000001003000000030000000300001002FCC
:102350000000002F0000002F0000002F0001002EC1
:102360000000002E0000002E0001002D0000002DB6
:102370000000002D0000002D0001002C0000002CAA
:102380000000002C0000002C0001002B0000002B9E
:102390000000002B0000002B0001002A0000002A92
:1023A0000000002A0000002A000100290000002986
:1023B0000000002900000029000000290001002879
:1023C000000000280000002800000028000000286D
:1023D0000001002700000027000000270000002760
:1023E0000000002700010026000000260000002653
:1023F0000000002600000026000100250000002546
:102400000000002500000025000000250000002538
:10241000000100240000002400000024000000242B
:10242000000000240001002300000023000000231E
:102430000000002300000023000000230000002310
:102440000001002200000022000000220000002203
:1024500000000022000000220001002100000021F5
:1024600000000021000000210000002100000021E8
:1024700000000021000100200000002000000020DA
:1024800000000020000000200000002000000020CC
:10249000000000200001001F0000001F0000001FBE
:1024A0000000001F0000001F0000001F0000001FB0
:1024B0000001001E0000001E0000001E0000001EA3
:1024C0000000004D38342058205920450020450098
:1024D000205A0020204D3930372058005374657041
:1024E000706572206D6F746F722063757272656EA5
:1024F00074733A0A0020520020204D393030204BAE
:10250000004C696E65617220416476616E63653A64
:102510000A0020590020580053656E736F726C6575
:10252000737320686F6D696E672074687265736875
:102530006F6C643A0A002045302000205A200020A9
:102540005920002058200053746570706572206413
:1025500072697665722063757272656E743A0A00EC
:1025600020204D383531205A005A2D50726F626547
:10257000204F666673657420286D6D293A0A002025
:10258000440020490020204D3330342050002044A6
:102590000020490020204D33303120500050494464
:1025A0002073657474696E67733A0A0020460020D0
:1025B000420020480020204D3134352053004D6129
:1025C00074657269616C20686561747570207061F2
:1025D00072616D65746572733A0A0020204D343261
:1025E000302053004175746F20426564204C65763D
:1025F000656C696E673A0A00205A00205900202055
:102600004D323036205800486F6D65206F66667316
:1026100065743A0A00204500205A002059002058CD
:102620000020420020540020204D3230352053003D
:10263000416476616E6365643A20533C6D696E5FF8
:1026400066656564726174653E20543C6D696E5FB9
:1026500074726176656C5F66656564726174653E0F
:1026600020423C6D696E5F7365676D656E745F7463
:10267000696D655F75733E20583C6D61785F787950
:102680005F6A65726B3E205A3C6D61785F7A5F6A63
:1026900065726B3E20453C6D61785F655F6A65726F
:1026A0006B3E0A0020540020520020204D3230346E
:1026B000205000416363656C65726174696F6E20C0
:1026C00028756E6974732F7332293A20503C7072EA
:1026D000696E745F616363656C3E20523C72657421
:1026E000726163745F616363656C3E20543C747215
:1026F0006176656C5F616363656C3E0A002045002E
:10270000205A0020590020204D3230312058004DF1
:102710006178696D756D20416363656C6572617484
:10272000696F6E2028756E6974732F7332293A0AA7
:1027300000204500205A0020590020204D3230331F
:102740002058004D6178696D756D2066656564720D
:10275000617465732028756E6974732F73293A0A42
:1027600000204500205A0020590020204D393220F9
:10277000580053746570732070657220756E6974AB
:102780003A0A0020204D3230302044300A00202008
:102790004D3230302044002044697361626C6564BE
:1027A0000A0046696C616D656E74207365747469A6
:1027B0006E67733A0020204D3134392043203B208E
:1027C000556E69747320696E2043656C7369757307
:1027D0000A002020473231202020203B20556E69FE
:1027E000747320696E206D6D0A005344206361721A
:1027F00064206F6B0A006F70656E526F6F74206695
:1028000061696C65640A00766F6C756D652E696E22
:102810006974206661696C65640A00534420696EBE
:102820006974206661696C0A006175746F25692E90
:1028300067000A003B20454550524F4D20496E64C9
:1028400065783A20005570646174696E67207A6F0C
:10285000666673657420696E20454550524F4D3A47
:1028600020000E000E000E000E000E000E000E00E6
:102870000E007FC03F801F000E00040004000E0009
:102880001F003F807FC00E000E000E000E000E00E5
:102890000E000E000E0007F8000C0C0010020020C5
:1028A00001006001804000804003E04001C0400022
:1028B0008040000040000060000020000010000088
:1028C0000C0C0007F80001FE000303000400800860
:1028D00000401800601000207C002038002010000C
:1028E0002000002000002000006000004000008068
:1028F00003030001FE00FFFFFF7F80FFC0FFC0FF5A
:10290000C07F807F80FFC0FFC0FFC03F001E000C63
:10291000005A204F6666736574005A204F666673CE
:10292000657400466C6F7700466C6F770046616E89
:102930002073706565640046616E20737065656420
:102940000042656400426564004E6F7A7A6C6500EF
:102950004E6F7A7A6C6500537065656400537065DC
:102960006564004D61696E004D6F76652058004DBD
:102970006F76652059004D6F7665205A0045787452
:102980007275646572004D6F766520302E316D6D05
:10299000004D6F766520316D6D004D6F766520318D
:1029A000306D6D004D6F76652061786973004578F4
:1029B000747275646572004D6F7665205A004D6FB4
:1029C00076652059004D6F76652058004578747201
:1029D00075646572004175746F20686F6D6500479E
:1029E0003238004D6F7665205A004D6F766520595C
:1029F000004D6F76652058004D6F76656D656E747D
:102A0000004D3234004D3233202573005772697403
:102A1000696E6720746F2066696C653A20006F707C
:102A2000656E206661696C65642C2046696C653A48
:102A300020006F70656E206661696C65642C2046AD
:102A4000696C653A200046696C652073656C656346
:102A50007465640A002053697A653A200046696CFF
:102A600065206F70656E65643A20006F70656E203A
:102A70006661696C65642C2046696C653A200020AB
:102A800066696C653A2000646F696E6700667265FE
:102A90007368004E6F772000454E442053554252D4
:102AA0004F5554494E450A002220706F7300222072
:102AB000706172656E743A2200535542524F5554FC
:102AC000494E452043414C4C207461726765743A0D
:102AD00022004B494C4C45442E2000747279696E9B
:102AE0006720746F2063616C6C207375622D67635F
:102AF0006F64652066696C657320776974682074FB
:102B00006F6F206D616E79206C6576656C732E2019
:102B10004D4158206C6576656C2069733A004572AA
:102B2000726F723A0043616E6E6F74206F70656EE3
:102B30002073756264697220006563686F3A00549F
:102B40004845524D414C2052554E41574159204223
:102B5000454400546865726D616C2052756E6177F2
:102B6000617900544845524D414C2052554E4157D1
:102B7000415920453100544845524D414C20525551
:102B80004E4157415920453000526573656E643A95
:102B900020002042002050006F6B004B494C4C45F8
:102BA000442E20004B494C4C2063617573656420B2
:102BB000627920746F6F206D75636820696E616340
:102BC000746976652074696D65202D206375727255
:102BD000656E7420636F6D6D616E643A2000506C99
:102BE00065617365207265736574005052494E5477
:102BF00045522048414C544544005072696E7465FA
:102C0000722068616C7465642E206B696C6C282975
:102C10002063616C6C6564210A002061786973200F
:102C20006472697665722063757272656E743A209B
:102C300000747275650066616C7365002061786967
:102C4000732074656D706572617475726520707241
:102C5000657761726E207472696767657265643A40
:102C60002000207072657761726E20666C6167204B
:102C7000636C65617265640A001000C90210012C62
:102C8000014001220170011801B0010E01F00104A0
:102C9000015002FA00B002F0003003E600D003DC7D
:102CA000009004D2007005C800A006BE000008B461
:102CB00000B009AA00D00BA000600E960060118C35
:102CC000000015820020197800C01D6E00A022644B
:102CD00000B0275A00902C500000314600E0343CF0
:102CE0000010383200903A2800603C1E00A03D14CD
:102CF00000803E0A00203F0000202F002042403A82
:102D00000020403A007C3C3E5E2B3D3F2F5B5D3B0C
:102D10002C2A225C00202863616C63756C617465E9
:102D20006429210A0020213D2000454550524F4D85
:102D300020435243206D69736D61746368202D20B8
:102D40002873746F726564292000290A0020627953
:102D50007465733B2063726320002073746F726527
:102D6000642073657474696E677320726574726928
:102D700065766564202800204D61726C696E3D5651
:102D80003437290A0028454550524F4D3D004545EE
:102D900050524F4D2076657273696F6E206D697366
:102DA0006D61746368200048617264636F64656478
:102DB0002044656661756C742053657474696E6730
:102DC00073204C6F616465640A0028230000282387
:102DD0000000C8000000E803000000009643000067
:102DE000964300009643000020420000C8420000C5
:102DF000C842000048430000D24300060900FE0616
:102E0000018902FE20FFFE07FE06FE00000006000C
:102E1000070106060602008080808000800303030D
:102E2000060103A0A0A00507070600FF5050F850B8
:102E3000F850500509090600FE2070A8A07028A8C7
:102E400070200608080600FF40A8481020485408D3
:102E50000507070600FF60909060989068010303E3
:102E60000602038080800207070602FF4080808000
:102E70008080400207070602FF80404040404080BB
:102E80000505050600008850F85088050505060070
:102E9000002020F820200204040602FEC0404080EA
:102EA000050101060002F8020202060200C0C00489
:102EB0000606060100101020408080040606060168
:102EC0000060909090906003060606010040C040AC
:102ED0004040E00406060601006090102040F00427
:102EE0000606060100F020601010E0050606060048
:102EF0000010305090F810040606060100F080E043
:102F00001010E00406060601006080E09090600466
:102F10000606060100F010102040400406060601D7
:102F2000006090609090600406060601006090903A
:102F3000701060020505060200C0C000C0C0020794
:102F4000070602FEC0C000C040408005050506001F
:102F5000001860806018050303060001F800F805FA
:102F60000505060000C0300830C004070706010050
:102F7000609010604000400506060600007090A8B2
:102F8000B08070050606060000205088F888880585
:102F90000606060000F088F08888F00406060601A0
:102FA00000609080809060040606060100E090902A
:102FB0009090E0040606060100F080E08080F004B6
:102FC0000606060100F080E0808080040606060107
:102FD00000609080B090600406060601009090F0BA
:102FE000909090030606060100E040404040E00556
:102FF0000606060000381010109060040606060150
:103000000090A0C0A0909004060606010080808079
:103010008080F005060606000088D8A8A8888804E5
:10302000060606010090D0B09090900506060600B6
:1030300000708888888870040606060100E0909079
:10304000E080800407070601FF609090D0B0601018
:10305000040606060100E09090E090900406060643
:103060000100609040209060050606060000F820F0
:103070002020202004060606010090909090906089
:10308000040606060100909090F0606005060606B2
:1030900000008888A8A8D888050606060000885081
:1030A0002020508805060606000088885020202031
:1030B000040606060100F010204080F00306060614
:1030C0000100E080808080E0040606060100808028
:1030D00040201010030606060100E020202020E01A
:1030E0000503030600032050880501010600FEF8D1
:1030F00002020206020480400404040601007090EB
:1031000090700406060601008080E09090E00404C0
:10311000040601007080807004060606010010108D
:103120007090907004040406010060B0C070040642
:1031300006060100205040E040400406060601FE5D
:103140006090907010600406060601008080E09098
:1031500090900306060601004000C04040E00308CE
:10316000080601FE200060202020A040040606067C
:1031700001008080A0C0A090030606060100C040A8
:10318000404040E0050404060000D0A8A8880404DC
:1031900004060100E0909090040404060100609091
:1031A00090600406060601FEE09090E08080040630
:1031B000060601FE709090701010040404060100D1
:1031C000A0D0808004040406010070C030E0040632
:1031D000060601004040E0405020040404060100BF
:1031E00090909070040404060100909060600504C3
:1031F0000406000088A8A85004040406010090609A
:1032000060900406060601FE9090907090600404A1
:1032100004060100F02040F00307070601002040EB
:1032200040804040200107070602FF8080808080A8
:103230008080030707060100804040204040800452
:10324000020206010350A0FFFFFFFFFFFFFFFFFF89
:10325000FFFFFFFFFFFFFFFFFFFFFFFFFFFFFFFF7E
:10326000FFFFFFFFFFFFFFFF000000060007010652
:10327000060602008000808080800406060601FFAA
:103280002070A0A070200507070600FF304840F01E
:103290004040F8050505060000A8508850A805061E
:1032A000060600008850F820F8200107070602FFF4
:1032B000808080008080800407070601FF708060A6
:1032C000906010E0030101060105A0060707060053
:1032D00000788494A494847803050506010160A015
:1032E0006000E00505050600002850A050280403F2
:1032F00003060100F01010040101060102F00607A8
:10330000070600007884B4A4A484780401010601AF
:1033100005F004030306010260906005070706003C
:10332000FF2020F8202000F803050506010140A039
:103330002040E0030505060101C0204020C0020234
:103340000206020440800405050601FF9090B0D0FB
:103350008005060606000078E8E8682828010101D3
:10336000060202800202020602FE408003050506F4
:10337000010140C04040E003050506010140A040B6
:1033800000E0050505060000A0502850A00508082B
:103390000600FF40C0405070307810050808060055
:1033A000FF40C04050680810380508080600FFC0FC
:1033B000204030F03078100407070601002000207C
:1033C000608090600507070600004020205070884C
:1033D0008805070706000010202050708888050720
:1033E0000706000020502050708888050707060057
:1033F00000285020507088880507070600005000FC
:103400002050708888050707060000205020507063
:10341000888805060606000078A0F0A0A0B8040879
:10342000080601FE60908080906020400407070637
:1034300001004020F080E080F00407070601002032
:1034400040F080E080F00407070601002050F08083
:10345000E080F00407070601005000F080E080F0F3
:103460000307070601008040E0404040E0030707F3
:103470000601002040E0404040E00307070601004D
:1034800040A0E0404040E0030707060100A000E044
:10349000404040E00506060600007048E8484870D5
:1034A00004070706010050A090D0B09090040707D1
:1034B000060100402060909090600407070601001C
:1034C0002040609090906004070706010020506043
:1034D0009090906004070706010050A060909090C3
:1034E0006004070706010050006090909060050599
:1034F0000506000088502050880408080601FF10C7
:1035000070B0B0D0D0E080040707060100402090E2
:1035100090909060040707060100204090909090E2
:103520006004070706010020509090909060040707
:103530000706010050009090909060050707060074
:10354000001020885020202004060606010080E09C
:103550009090E0800406060601006090A0A090A074
:1035600004070706010040200070909070040707D0
:1035700006010020400070909070040707060100CB
:103580002050007090907004070706010050A000C2
:1035900070909070040606060100500070909070C4
:1035A0000407070601002050207090907005040465
:1035B00006000070A8B0780406060601FE70808040
:1035C00070204004070706010040200060B0C07072
:1035D00004070706010020400060B0C07004070720
:1035E00006010020500060B0C0700406060601000D
:1035F000500060B0C070030707060100804000C0A3
:103600004040E0030707060100204000C04040E0C2
:1036100003070706010040A000C04040E003060683
:10362000060100A000C04040E0040707060100308A
:1036300060107090906004070706010050A000E041
:103640009090900407070601004020006090906071
:1036500004070706010020400060909060040707FF
:1036600006010020500060909060040707060100EA
:1036700050A00060909060040606060100500060B3
:103680009090600505050600002000F80020040465
:103690000406010070B0D0E00407070601004020D6
:1036A0000090909070040707060100204000909061
:1036B000907004070706010020500090909070045D
:1036C000060606010050009090907004090906015A
:1036D000FE2040009090907090600408080601FE63
:1036E0008080E09090E080800408080601FE500091
:1036F00090909070906000060900FE0701920321EF
:10370000207FFF07FF07FF000000060000010707FA
:10371000060200808080808000800302020601058E
:10372000A0A00507070600005050F850F8505005BB
:1037300007070600002078A07028F020050707067C
:103740000000C0C810204098180507070600006058
:1037500090A040A89068020303060104C0408003C3
:1037600007070601002040808080402003070706ED
:103770000100804020202040800505050600012032
:10378000A870A8200505050600012020F8202002C9
:1037900003030602FFC04080050101060003F80292
:1037A0000202060200C0C00505050600010810203F
:1037B00040800507070600007088888888887003A5
:1037C000070706010040C040404040E005070706EB
:1037D0000000708808708080F8050707060000F870
:1037E0001020100808F00507070600001030509060
:1037F000F81010050707060000F880F00808887028
:10380000050707060000708080F0888870050707AC
:10381000060000F8081020202020050707060000F9
:10382000708888708888700507070600007088888F
:1038300078080870020505060200C0C000C0C0027A
:1038400006060602FFC0C000C0408004070706004D
:103850000010204080402010050303060002F800FD
:10386000F80407070601008040201020408005076B
:1038700007060000708808102000200507070600D2
:103880000070880868A8A8700507070600007088FF
:1038900088F8888888050707060000F08888F0887F
:1038A00088F0050707060000708880808088700512
:1038B0000707060000F08888888888F00507070653
:1038C0000000F88080F08080F8050707060000F807
:1038D0008080F0808080050707060000708880B82F
:1038E000888870050707060000888888F888888817
:1038F000010707060200808080808080800507071E
:103900000600003810101010906005070706000030
:103910008890A0C0A09088050707060000808080DE
:10392000808080F805070706000088D8A888888866
:10393000880507070600008888C8A89888880507B2
:1039400007060000708888888888700507070600C9
:1039500000F08888F08080800507070600007088E6
:103960008888A89068050707060000F08888F0A0FE
:103970009088050707060000788080700808F00529
:103980000707060000F82020202020200507070652
:1039900000008888888888887005070706000088E6
:1039A000888888885020050707060000888888884E
:1039B00088A850050707060000888850205088888E
:1039C0000507070600008888885020202005070783
:1039D000060000F80810204080F8030707060100E1
:1039E000E08080808080E0050505060001804020A1
:1039F0001008030707060100E02020202020E00532
:103A00000303060004205088050101060000F802A7
:103A100002020602058040050505060000700878D0
:103A200088780507070600008080B0C88888F00500
:103A300005050600007080808870050707060000F5
:103A4000080868988888780505050600007088F8D9
:103A500080700507070600003048E0404040400500
:103A600006060600FF7088887808700507070600BC
:103A7000008080B0C888888801070706020080009F
:103A800080808080800308080601FF20002020201D
:103A900020A040040707060000808090A0C0A090EE
:103AA000030707060100C04040404040E00505050F
:103AB000060000D0A8A8A8A8050505060000B0C803
:103AC00088888805050506000070888888700506C6
:103AD000060600FFF08888F080800506060600FFD5
:103AE000788888780808050505060000B0C8808039
:103AF0008005050506000070807008F004070706C1
:103B000000004040E04040403005050506000088C8
:103B10008888986805050506000088888850200573
:103B200005050600008888A8A850050505060000C0
:103B300088502050880506060600FF888888780887
:103B400070050505060000F8102040F80307070679
:103B5000010020404080404020010707060200800D
:103B6000808080808080030707060100804040201D
:103B70004040800502020600026890000000060036
:103B80000000060900FE000000000001090008FE18
:103B9000000005080806000040F0C88888987810E2
:103BA000050808060000C0F88888888888F8050598
:103BB000050600012030F830200508080600002026
:103BC00070F820202020E00509090600FF2070A8D9
:103BD000A8B8888870200509090600FFE080C0B0F9
:103BE000A8283028280509090600FFF8A888888831
:103BF0008888A8F8050A0A0600FE20505050508810
:103C0000A8A8887003030306000340A0400105082C
:103C100000FF060121023520FFFF07FF06FF090014
:103C200050221656808080800080153353A0A0A0BB
:103C30000257575050F850F850500257572070A074
:103C40007028702013355580A040A02002475740AF
:103C5000A0A040A0A050251353808080122656407B
:103C6000808080804012265680404040408002453F
:103C7000559060F060900255552020F820201133B7
:103C800053604080044151F011335340E0400246FC
:103C90005610102040808012365640A0A0A0A040B0
:103CA00012365640C0404040E002465660901060D8
:103CB00080F0024656F02060109060024656206068
:103CC000A0F02020024656F080E010906002465698
:103CD0006080E0909060024656F010202040400244
:103CE00046566090609090600246566090907010CA
:103CF00060122555C0C000C0C0113656606000601B
:103D00004080123656204080804020034353F0000C
:103D1000F012365680402020408012365640A020B7
:103D2000400040015858304898A8A89040300246BA
:103D300056609090F09090024656E090E09090E0AF
:103D4000024656609080809060024656E0909090C7
:103D500090E0024656F080E08080F0024656F08007
:103D6000E0808080024656609080B09060024656A7
:103D70009090F0909090123656E040404040E00223
:103D8000465670202020A04002465690A0C0A0A019
:103D9000900246568080808080F002465690F0F077
:103DA00090909002465690D0F0B0B0900246566087
:103DB0009090909060024656E09090E0808001479D
:103DC00057609090D0B06010024656E09090E0901E
:103DD00090024656609040209060123656E0404077
:103DE0004040400246569090909090600246569017
:103DF0009090906060024656909090F0F09002464D
:103E000056909060609090025656888850202020EE
:103E1000024656F010204080F0123656E080808036
:103E200080E0024656808040201010123656E02076
:103E3000202020E016325240A0014151F0162252BB
:103E40008040024454709090700246568080E0900A
:103E500090E01234546080806002465610107090DA
:103E6000907002445460B0C060024656205040E05A
:103E7000404001455560907010600246568080E0D9
:103E80009090901236564000C04040E011375720C5
:103E900000202020A040024656808090E0909012A2
:103EA0003656C040404040E0025454D0A8A8A80272
:103EB0004454E090909002445460909060014555C5
:103EC000E090E080800145557090701010024454DD
:103ED000A0D0808012345460C020C00246564040BA
:103EE000E040502002445490909070123454A0A0AE
:103EF000A04002545488A8A8500244549060609096
:103F00000145559090709060024454F02040F002BA
:103F10004757304020C02040302216568080808095
:103F20008080024757C02040304020C00642525097
:103F3000A0FFFFFFFFFFFFFFFFFFFFFFFFFFFFFFF0
:103F4000FFFFFFFFFFFFFFFFFFFFFFFFFFFFFFFF81
:103F5000FFFF0900502216568000808080800146B5
:103F6000562070A0A070200246562050E04050A07D
:103F700002555588705070880256568850F820F8BF
:103F800020221757808080008080800247577080F1
:103F9000E0907010E0173151A002565670A8C8C8C2
:103FA000A87014355560A06000E003435350A05042
:103FB000123353E02020143151E002565670E8D8F5
:103FC000E8D870173151E015335340A040123555F1
:103FD00040E04000E014355540A02040E014355545
:103FE000C020C020C01622524080014555909090BC
:103FF000E08002565678E8E868282824115180119C
:104000002252408014355540C04040E014355540A0
:10401000A04000E0034353A050A002475780808097
:10402000A060F0200247578080A0D0102070024787
:104030005780408060A0F02012365640004080A09B
:104040004002475740206090F09090024757204030
:104050006090F0909002475760906090F0909002CE
:10406000475750A06090F0909002475790006090A2
:10407000F0909002475760906090F0909002465602
:1040800070A0A0F0A0B00147576090808090604081
:104090000247574020F080E080F00247572040F070
:1040A00080E080F00247576090F080E080F00247A7
:1040B000579000F080E080F01237578040E0404099
:1040C00040E01237572040E0404040E01237574070
:1040D000A0E0404040E0123757A000E0404040E000
:1040E0000256567048E848487002475750A090D092
:1040F000B0909002475740206090909060024757E0
:10410000204060909090600247576090609090903F
:104110006002475750A0609090906002475790000F
:104120006090909060123353A040A002465670B049
:10413000B0D0D0E002475740209090909060024766
:1041400057204090909090600247576090909090D8
:1041500090600247579000909090906002575710DF
:1041600020885020202002465680E09090E0800277
:1041700046566090A0A090A0024757402000709043
:10418000907002475720400070909070024757206F
:1041900050007090907002475750A000709090703F
:1041A00002465650007090907002475760906070C1
:1041B000909070025454F068B0781135556080804A
:1041C000604002475740200060B0C060024757205F
:1041D000400060B0C06002475760900060B0C060AF
:1041E000024656500060B0C060123757804000C091
:1041F0004040E0123757204000C04040E01237579F
:1042000040A000C04040E0123656A000C04040E050
:10421000024757A040A01070906002475750A0007E
:10422000E0909090024757402000609090600247D5
:104230005720400060909060024757609000609067
:10424000906002475750A0006090906002465690E0
:1042500000609090601235554000E00040024454E8
:1042600070B0D0E002475740200090909070024715
:1042700057204000909090700247576090009090B7
:1042800090700246569000909090700148582040DF
:104290000090907090600147578080E090E08080AF
:1042A0000147579000909070906001050700FE054F
:1042B00000FB01F220FFFE05FE05FE020040021594
:1042C000258080800080053242A0A002556550F80C
:1042D00050F8500146562070C030E02002556590DD
:1042E0001020404802556560806890680512228061
:1042F0008002253540808080400225358040404046
:1043000080043343A040A003334340E04001223205
:104310004080043141E002112180025565081020DF
:1043200040800245556090909060022535C0404025
:104330004040024555E0106080F0024555E01060B5
:1043400010E00245552060A0F020024555F080E0C5
:1043500010E00245556080E09060024555F0102065
:1043600040400245556090609060024555609070F5
:1043700010600313238000800214248000808002D8
:1043800035452040804020033343E000E0023545BE
:104390008040204080024555E01060004002556595
:1043A0007088B8A870024555609090F0900245550D
:1043B000E090E090E00235456080808060024555E5
:1043C000E0909090E0023545E080E080E0023545E5
:1043D000E080E080800245557080B09070024555C5
:1043E0009090F09090023545E0404040E002455505
:1043F000301010906002455590A0C0A09002354545
:1044000080808080E002556588D8A888880245555C
:1044100090D0B090900245556090909060024555C4
:10442000E09090E0800146566090909060100245C8
:1044300055E09090E09002455570806010E00235A4
:1044400045E04040404002455590909090600245C4
:10445000559090A0A04002556588A8A8A850024594
:104460005590906090900245559090701060023584
:1044700045E0204080E0022535C0808080C00255A4
:10448000658040201008022535C0404040C00532FC
:104490004240A0024151F005223280400244547053
:1044A00090907002455580E09090E0023444608026
:1044B0008060024555107090907002445460B0C006
:1044C000600235452040E0404000465670909070B4
:1044D000106002455580E090909002152580008084
:1044E0008080002737400040404040800245558092
:1044F00090A0E0900215258080808080025464F0B6
:10450000A8A8A8024454E09090900244546090906F
:1045100060004656E09090E0808000465670909093
:10452000701010023444A0C0808002445470C03027
:10453000E002354540E040402002445490909070A5
:104540000244549090A040025464A8A850500234F1
:1045500044A04040A00046569090907010600244E5
:1045600054F02040F002354560408040600215253F
:104570008080808080023545C0402040C005425286
:1045800050A0FFFFFFFFFFFFFFFFFFFFFFFFFFFF49
:10459000FFFFFFFFFFFFFFFFFFFFFFFFFFFFFFFF2B
:1045A000FFFFFF020040FFFFFFFFFFFFFFFFFFFFD6
:1045B000FFFFFFFFFFFFFFFFFFFFFFFFFFFFFFFF0B
:1045C000FFFFFFFFFFFFFFFFFFFFFFFFFFFFFFFFFB
:1045D000FFFFFFFFFFFFFFFFFFFFFFFFFFFFFFFFEB
:1045E000FFFFFFFFFFFFFFFFFFFFFFFFFFFFFFFFDB
:1045F000FFFFFFFFFFFFFFFFFFFFFFFFFFFFFFFFCB
:10460000FFFFFFFFFF01060D00FE09016602D62035
:10461000FFFE0BFE0AFE0D0060221969808080807B
:104620008080800080183363A0A0A003576750509B
:10463000F850F850500259692078A0A0702828F04E
:104640002002596948A85010204050A8900258688C
:1046500040A0A040A0989068281363808080113B00
:104660006B2040408080808080404020113B6B80E8
:104670004040202020202040408006556520A87022
:10468000A8200455652020F8202011336360408065
:10469000065161F811336340E0400259690808107F
:1046A000102040408080025969205088888888887E
:1046B00050200259692060A02020202020F80259B3
:1046C000697088880810204080F8025969F808103D
:1046D000207008088870025969101030505090F806
:1046E0001010025969F88080B0C808088870025913
:1046F0006970888080F088888870025969F808108D
:10470000102020404040025969708888887088884D
:10471000887002596970888888780808887011380C
:104720006840E040000040E04011386840E0400050
:104730000060408002596908102040804020100825
:10474000045464F80000F8025969804020100810F1
:1047500020408002596970888808102020002002BB
:10476000596970888898A8A8B08078025969205043
:10477000888888F8888888025969F04848487048CD
:104780004848F00259697088808080808088700273
:104790005969F048484848484848F0025969F88043
:1047A0008080F0808080F8025969F8808080F080F5
:1047B0008080800259697088808080988888700223
:1047C000596988888888F888888888123969E0401B
:1047D000404040404040E00259693810101010102D
:1047E000109060025969888890A0C0A090888802C3
:1047F00059698080808080808080F802596988882B
:10480000D8A8A88888888802596988C8C8A8A8989C
:104810009888880259697088888888888888700292
:104820005969F0888888F080808080015A6A708891
:104830008888888888A87008025969F0888888F074
:10484000A0908888025969708880807008088870F4
:10485000025969F820202020202020200259698850
:1048600088888888888888700259698888888850EC
:104870005050202002596988888888A8A8A8A85084
:104880000259698888505020505088880259698898
:104890008850502020202020025969F8081010204C
:1048A000404080F8113B6BE0808080808080808079
:1048B00080E0025969808040402010100808113BB8
:1048C0006BE0202020202020202020E008536320BF
:1048D0005088015161F82A226280400256667008B1
:1048E00078889868025969808080F088888888F084
:1048F00002566670888080887002596908080878B6
:1049000088888888780256667088F880887002598E
:104910006930484040F04040404000586870888806
:104920008878088870025969808080B0C888888833
:10493000881238684000C040404040E0004A6A1099
:1049400000301010101090906002596980808090A3
:10495000A0C0A09088123969C0404040404040400B
:10496000E0025666D0A8A8A8A888025666B0C888F3
:10497000888888025666708888888870005868F031
:10498000888888F0808080005868788888887808CF
:104990000808025666B0C88080808002566670881B
:1049A000601088700258684040F040404048300233
:1049B0005666888888889868025666888888505025
:1049C000200256668888A8A8A850025666885020FB
:1049D000205088005868888888986808887002562F
:1049E00066F810204080F8015B6B1820202020C062
:1049F000202020201822196980808080808080807B
:104A000080015B6BC0202020201820202020C008BF
:104A1000536348A890FFFFFFFFFFFFFFFFFFFFFF6B
:104A2000FFFFFFFFFFFFFFFFFFFFFFFFFFFFFFFF96
:104A3000FFFFFFFFFFFF0D006022196980008080EB
:104A400080808080800358682070A8A0A0A8702073
:104A500002596930484040E0404048B003566688FB
:104A6000705050708802596988885050F820F8209A
:104A700020221969808080800080808080124A6AAC
:104A8000609080609090601090601A3262A0A003E5
:104A900059697088A8D8C8D8A88870045767700862
:104AA00078887800F80356662850A0A05028045350
:104AB00063F80808163161E00359697088E8D8D8AE
:104AC000E8D888700A5161F81744646090906003D8
:104AD00057672020F8202000F807356540A02040C7
:104AE000E007356540A04020C02A2262408000587F
:104AF000688888888898E8808002596978E8E8E8BA
:104B0000E868282828262161C020226240800735D5
:104B10006540C04040E0045767708888887000F89E
:104B2000035666A050282850A0025A6A40C0404050
:104B3000E00818283808025A6A40C04040E01028AF
:104B4000081038025A6A40A04020A04818283808A7
:104B5000025969200020204080888870025A6A40EB
:104B6000200020508888F88888025A6A1020002087
:104B7000508888F88888025A6A304800205088880F
:104B8000F88888025A6A28500020508888F8888857
:104B9000025A6A50500020508888F88888025A6A61
:104BA00020502020508888F8888802596958A0A091
:104BB000A0B0E0A0A0B8005B6B708880808080808F
:104BC00088702040025A6A402000F88080F080807F
:104BD000F8025A6A102000F88080F08080F8025AAB
:104BE0006A304800F88080F08080F8025A6A50509D
:104BF00000F88080F08080F8123A6A804000E0403F
:104C000040404040E0123A6A204000E040404040CE
:104C100040E0124A6A609000E04040404040E012AC
:104C20003A6AA0A000E04040404040E0025969F0EC
:104C3000484848E8484848F0025A6A28500088889E
:104C4000C8A8988888025A6A402000708888888896
:104C50008870025A6A1020007088888888887002DC
:104C60005A6A30480070888888888870025A6A2892
:104C7000500070888888888870025A6A5050007086
:104C80008888888888700355658850205088015B23
:104C90006B08709898A8A8A8C8C87080025A6A4083
:104CA000200088888888888870025A6A10200088C6
:104CB000888888888870025A6A304800888888887E
:104CC000888870025A6A505000888888888888705E
:104CD000025A6A102000888850202020200259693A
:104CE00080F0888888F0808080025969609090A068
:104CF000A0908888B0025969402000700878889890
:104D0000680259691020007008788898680259690B
:104D100030480070087888986802596928500070F7
:104D20000878889868025969505000700878889807
:104D300068025A6A304830007008788898680256CD
:104D400066702870A0A850005868708880808870AD
:104D500020400259694020007088F880887002590C
:104D6000691020007088F880887002596930480006
:104D70007088F88088700259695050007088F880F7
:104D80008870123969804000C040404040E01239CC
:104D900069204000C040404040E0124969609000F6
:104DA000C040404040E0123969A0A000C0404040EF
:104DB00040E0025A6A50206010708888888870022B
:104DC0005969285000B0C8888888880259694020ED
:104DD000007088888888700259691020007088885F
:104DE0008888700259693048007088888888700205
:104DF0005969285000708888888870025969505015
:104E000000708888888870035767202000F8002089
:104E100020015868087098A8A8C870800259694095
:104E2000200088888888986802596910200088883E
:104E30008888986802596930480088888888986806
:104E4000025969505000888888889868005B6B1008
:104E500020008888889868088870005A6A8080B026
:104E6000C88888C8B08080005B6B505000888888F4
:104E70009868088870000000000000000000000032
:104E80000000000000000000000000000000000022
:104E900000000000000000000C0000000000000006
:104EA0000C000000000000001200000000000000E4
:104EB00023000000000000002100000000000000AE
:104EC0004C800000000000005E8000000000000038
:104ED0009240000000000000A1400000000000011E
:104EE00021200000000000027F900000000000026E
:104EF0000010000000000007FFF8000000000004A0
:104F00000008000000000008000400000000000885
:104F10000006000000000010000200000000003049
:104F20001E010000000000207F8100000000004101
:104F3000FFE0800000000043FCF0800000000087DC
:104F40003B7840000000018EDBFC60000000010F98
:104F5000EBCC20000000021FEDB610000000021F85
:104F6000DEB6100000000439CD7F080000000436D2
:104F7000E0FF08000000087EC0BB84000000187F2E
:104F8000005D86000000107FC0ED82000000203C24
:104F9000C07301000000203B337F01000000701B44
:104FA000E77E03800000C81DEEDE04C00000880F0D
:104FB000DEDC04400001240FDF3C0920000126074D
:104FC000DBF8192000027203E7F013900002510190
:104FD000FFE02290000489007F80244800090480BB
:104FE0001E004824000BFE400000DFF400100040CB
:104FF00000008002001FFFFFFFFFFFFE0000000017
:1050000000000000000000000000000000000000A0
:1050100000000000001022103C3C0E1F0010221067
:105020000422110400102210082211040010221082
:10503000083C11040010221010221104001022104C
:1050400020221104001E1C1E3C3C0E040000000027
:105050000000000000000000000000000000000050
:105060000000000000000000000000000000000040
:105070000000000000000000000000000000000030
:105080000000000000000000000000000000000020
:105090000000000000000000000000000000000010
:1050A0000000000000000000000000000000000000
:1050B00000000000002200250028002B002E0031F7
:1050C00000340002010000050108010B010000216D
:1050D00000240027002A002D0030003300010100C9
:1050E00000040107010A0105050505070508080870
:1050F00008020202020A0A08080404040401010169
:105100000101010101030303030303030304070770
:10511000070C0C0C0C0C0C0C0C020202020606060E
:1051200006060606060B0B0B0B0B0B0B0B010210F6
:1051300020200808102040102040800201020108B1
:105140000402010102040810204080804020100861
:1051500004020180040201804020100804020108BA
:10516000040201010204081020408001020408101A
:10517000204080456E642066696C65206C6973749C
:105180000A00426567696E2066696C65206C697308
:10519000740A005344207072696E74696E672062ED
:1051A00079746520004E6F74205344207072696ECC
:1051B00074696E670A00000125311D40FF24301C10
:1051C000FF45232F1B0A07FFFF040806FF06222BBB
:1051D0001AFFFF043803FF36FFFFFFFFFFFF507287
:1051E0006F7465637465642050696E0A0000000A7C
:1051F0000B02090C0D0E080703040100000000005B
:10520000000000000000000000000000000000009E
:10521000000000000000000000121110000000005B
:10522000000000000000000000000000000000007E
:1052300000000050726F62696E67206661696C657C
:10524000640A0050726F62696E67206661696C65FE
:105250006400205A3A200020593A20004265642018
:10526000583A2000DA00858011241FBECFEFD1E22A
:10527000DEBFCDBF00E00CBF14E0A0E0B2E0ECED7B
:10528000F8E602E00BBF02C007900D92AC34B10704
:10529000D9F728E1ACE4B4E001C01D92A436B2070E
:1052A000E1F719E2C3E3D9E200E006C02197010962
:1052B000802FFE010F94D933C233D10780E0080755
:1052C000A9F70E94C4510D945D340C9400002F92F4
:1052D0003F924F925F926F927F928F929F92AF9286
:1052E000BF92CF92DF92EF92FF920F931F93CF93D3
:1052F000DF93CDB7DEB7CC5AD1090FB6F894DEBF35
:105300000FBECDBFCC55DF4F8883C45AD0402DB7D8
:105310003EB7CB55DF4F39832883C55AD0408091A3
:1053200017078D3411F40C94B332843511F40C94B6
:105330007642873411F00C94B642E0901507F09055
:1053400016073AE1E316F10409F4ACC7CCF454E0D3
:10535000E516F1044CF482E0E816F1040CF061C0AB
:10536000F7FE33C00C94D04294E0E916F10409F43E
:1053700026C6ACE0EA16F10409F468C60C94D042E3
:10538000BEE1EB16F10411F40C94D33144F4FCE1CA
:10539000EF16F10409F4C0C70CF48BC7C2C73BE594
:1053A000E316F10411F40C9441324CE5E416F104D7
:1053B00011F40C9446325AE5E516F10411F00C9400
:1053C000D042109253040C94D0428091270288233B
:1053D00011F40C94D0428AE50E944BB7482F89E51E
:1053E000C855DF4F4883C85AD0400E944BB7682F3A
:1053F00088E5C955DF4F6883C75AD0400E944BB734
:10540000C855DF4F4881C85AD040C955DF4F688121
:10541000C75AD0400E94FDAF81110C94D0420C9429
:10542000DB4241E061E081E00E94FDAF81110C941C
:10543000D04280912702882311F40C94D04211E0CD
:10544000B2E0EB16F10409F010E00E9486B782E5A5
:105450000E947AB7882309F45CC10E9414B76B01DB
:105460007C014090F30E5090F40E6090F50E709019
:10547000F60E2091F70E3091F80E4091F90E5091F2
:10548000FA0E27962CAF3DAF4EAF5FAF27978091B6
:10549000E5069091E606A091E706B091E8062B9606
:1054A0008CAF9DAFAEAFBFAF2B972091E906309187
:1054B000EA064091EB065091EC062F962CAF3DAFDB
:1054C0004EAF5FAF2F9720E030E0A901C701B601D2
:1054D0000F94742C882309F458C5A30192012B96CC
:1054E0006CAD7DAD8EAD9FAD2B970F94742C81115B
:1054F00011C027962CAD3DAD4EAD5FAD27972F96D1
:105500006CAD7DAD8EAD9FAD2F970F94742C88231D
:1055100009F43BC520E030E0A901C701B6010F94B2
:10552000742C881F8827881F18130BC080E090E018
:10553000A0E8BFE36F968CAF9DAFAEAFBFAF6F97E4
:105540000AC020E030E040E85FEB6F962CAF3DAF43
:105550004EAF5FAF6F97A30192012B966CAD7DADFF
:105560008EAD9FAD2B970F94DD3067966CAF7DAFFE
:105570008EAF9FAF679727962CAD3DAD4EAD5FAD1B
:1055800027972F966CAD7DAD8EAD9FAD2F970F9465
:10559000DD306B966CAF7DAF8EAF9FAF6B9767962C
:1055A0002CAD3DAD4EAD5FAD6797CA01B9010F940B
:1055B000D92C4B015C016B962CAD3DAD4EAD5FAD72
:1055C0006B97CA01B9010F94D92C9B01AC01C5019D
:1055D000B4010F94DE300F94493363966CAF7DAF06
:1055E0008EAF9FAF639720E030E040E05FE30F9421
:1055F000D92C4B015C01A7019601C701B6010F949C
:10560000D92C6B017C01A5019401C501B4010F9453
:10561000D92C9B01AC01C701B6010F94DD300F946A
:1056200049339B01AC016F966CAD7DAD8EAD9FADE6
:105630006F970F94D92C4B015C012B962CAD3DAD8F
:105640004EAD5FAD2B97C301B2010F94DE3020E069
:1056500030E040E05FE30F94D92C6B017C016B9646
:105660006CAD7DAD8EAD9FAD6B97905863962CADB4
:105670003DAD4EAD5FAD63970F94BA319B01AC0168
:10568000C501B4010F94D92C9B01AC01C701B6012F
:105690000F94DE30A30192010F94DD306B017C0189
:1056A0002F962CAD3DAD4EAD5FAD2F9727966CADCF
:1056B0007DAD8EAD9FAD27970F94DE3020E030E0BA
:1056C00040E05FE30F94D92C2B013C0163962CAD95
:1056D0003DAD4EAD5FAD639767966CAD7DAD8EAD64
:1056E0009FAD67970F94BA319B01AC01C501B4011E
:1056F0000F94D92C9B01AC01C301B2010F94DE3091
:1057000027962CAD3DAD4EAD5FAD27970F94DD30A4
:1057100014C089E40E947AB7882329F00E9414B744
:105720006B017C0103C0C12CD12C76018AE40E945C
:105730007AB78823F9F00E9414B72F966CAF7DAF2B
:105740008EAF9FAF2F9720E030E0A901C701B601CF
:105750000F94742C81111EC020E030E0A9012F9617
:105760006CAD7DAD8EAD9FAD2F970F94742C8111D4
:1057700011C00BC420E030E0A901C701B6010F94AD
:10578000742C882309F401C42F961CAE1DAE1EAEE6
:105790001FAE2F97D701C601B05827968CAF9DAF8B
:1057A000AEAFBFAF27972F962CAD3DAD4EAD5FADE1
:1057B0002F9750582B962CAF3DAF4EAF5FAF2B9726
:1057C0009C01AD01BC01CD010F94D92C4B015C01B2
:1057D0002B962CAD3DAD4EAD5FAD2B97CA01B901F7
:1057E0000F94D92C9B01AC01C501B4010F94DE309C
:1057F0000F944933AF966CAF7DAF8EAF9FAFAF972D
:105800008091F30E9091F40EA091F50EB091F60EEA
:1058100063968CAF9DAFAEAFBFAF6397A701960104
:10582000BC01CD010F94DE306F966CAF7DAF8EAFB3
:105830009FAF6F972091F70E3091F80E4091F90EBF
:105840005091FA0E6B962CAF3DAF4EAF5FAF6B979A
:105850002F962CAD3DAD4EAD5FAD2F976B966CADD9
:105860007DAD8EAD9FAD6B970F94DE30A3966CAF80
:105870007DAF8EAF9FAFA3978091E5069091E6062E
:10588000A091E706B091E806A7968CAF9DAFAEAFAA
:10589000BFAFA7976F962CAD3DAD4EAD5FAD6F9787
:1058A000BC01CD010F94DD306B017C012091E90634
:1058B0003091EA064091EB065091EC06AB962CAF86
:1058C0003DAF4EAF5FAFAB97A3962CAD3DAD4EADA8
:1058D0005FADA397AB966CAD7DAD8EAD9FADAB9735
:1058E0000F94DD304B015C018091FB0E9091FC0E1A
:1058F000A091FD0EB091FE0EE7968CAF9DAFAEAFBE
:10590000BFAFE7979C01AD016091ED067091EE0687
:105910008091EF069091F0060F94DD3067966CAFA2
:105920007DAF8EAF9FAF67972091F1063091F20661
:105930004091F3065091F406E3962CAF3DAF4EAF85
:105940005FAFE3978091FF0E9091000FA091010F40
:10595000B091020FEB968CAF9DAFAEAFBFAFEB97A0
:10596000A701960127966CAD7DAD8EAD9FAD2797B3
:105970000F94D92C2B013C01A50194012B966CAD01
:105980007DAD8EAD9FAD2B970F94D92C9B01AC01B3
:10599000C301B2010F94DE302B013C01A50194013B
:1059A00027966CAD7DAD8EAD9FAD27970F94D92C0A
:1059B0004B015C01A70196012B966CAD7DAD8EADC0
:1059C0009FAD2B970F94D92C9B01AC01C501B4015D
:1059D0000F94DD30A30192010F9451316B017C01D2
:1059E00020E030E0A9010F94742C87FF0AC02BED52
:1059F0003FE049EC50E4C701B6010F94DE306B0183
:105A00007C01112351F02BED3FE049EC50E4C7013C
:105A1000B6010F94DD306B017C0120E030E0A9017C
:105A2000C701B6010F94742C811128C0A7962CAD24
:105A30003DAD4EAD5FADA79763966CAD7DAD8EADC0
:105A40009FAD63970F94742C811118C0AB962CAD49
:105A50003DAD4EAD5FADAB976B966CAD7DAD8EAD94
:105A60009FAD6B970F94742C811108C06BEDC62EFF
:105A70006FE0D62E69ECE62E60E4F62EAF962CADE4
:105A80003DAD4EAD5FADAF97C701B6010F94D92CB8
:105A90009B01AC010F94D92C4B015C0167962CAD96
:105AA0003DAD4EAD5FAD6797CA01B9010F94D92CDA
:105AB0009B01AC01C501B4010F94DE300F94493352
:105AC0004B015C012FE632E143E85AE30F94742C5A
:105AD00087FD57C2C501B4010F9453320F9427328A
:105AE0001B01672B19F422242394312CB10180E08F
:105AF00090E00F94782C4B015C019B01AC01C70135
:105B0000B6010F94BA3163966CAF7DAF8EAF9FAF85
:105B10006397A501940167966CAD7DAD8EAD9FAD89
:105B200067970F94BA31AF966CAF7DAF8EAF9FAFD2
:105B3000AF97EB962CAD3DAD4EAD5FADEB97E396D9
:105B40006CAD7DAD8EAD9FADE3970F94DD30A501BB
:105B500094010F94BA31E3966CAF7DAF8EAF9FAFD7
:105B6000E39763962CAD3DAD4EAD5FAD6397CA0133
:105B7000B9010F94D92C20E030E040E05FE30F94AE
:105B8000D92C9B01AC0160E070E080E89FE30F94AA
:105B9000DD30A7966CAF7DAF8EAF9FAFA797E7962E
:105BA0002CAD3DAD4EAD5FADE79729873A874B876A
:105BB0005C87EB968CAD9DADAEADBFADEB978D87A1
:105BC0009E87AF87B88B6091010270910202072E09
:105BD000000C880B990B0F947A2C2091A302309122
:105BE000A4024091A5025091A6020F94D92C2AE05C
:105BF00037ED43E25CE30F94D92C6BAF7CAF8DAFF4
:105C00009EAF0E94DB509B01AC0128533F4F4F4F8A
:105C10005F4FAB962CAF3DAF4EAF5FAFAB972496C7
:105C20004FAC249725965FAC259726966FAC2697A8
:105C300027967FAC279741E050E069965FAF4EAF63
:105C4000699759E164965FAF64976996AEADBFAD51
:105C50006997A215B30509F459C10E94A7990E943A
:105C6000DB50DC01CB01AB962CAD3DAD4EAD5FAD55
:105C7000AB97821B930BA40BB50BB7FD11C00E9411
:105C8000DB509B01AC0128533F4F4F4F5F4FAB960A
:105C90002CAF3DAF4EAF5FAFAB9780E00F94610488
:105CA00064963FAD6497315064963FAF6497332359
:105CB00009F44BC0A7962CAD3DAD4EAD5FADA79797
:105CC0002B966CAD7DAD8EAD9FAD2B970F94D92CDF
:105CD0006B017C0163962CAD3DAD4EAD5FAD63971E
:105CE000B201C3010F94D92CA70196010F94DE30A5
:105CF0007B018C01A7962CAD3DAD4EAD5FADA79756
:105D0000B201C3010F94D92C4B015C0163962CADF9
:105D10003DAD4EAD5FAD63972B966CAD7DAD8EAD59
:105D20009FAD2B970F94D92C9B01AC01C501B401F9
:105D30000F94DD302B013C01C701D8012B968CAFAD
:105D40009DAFAEAFBFAF2B9761C069964EAD5FAD53
:105D50006997BA0180E090E00F94782C63962CAD9F
:105D60003DAD4EAD5FAD63970F94D92C4B015C01F7
:105D70000F94B7316B017C01C501B4010F943F331F
:105D80004B015C01A701960127966CAD7DAD8EADF0
:105D90009FAD27970F94D92C2B013C01A5019401AD
:105DA0002F966CAD7DAD8EAD9FAD2F970F94D92CF6
:105DB0009B01AC01C301B2010F94DE302B013C0109
:105DC000A501940127966CAD7DAD8EAD9FAD279753
:105DD0000F94D92C4B015C01A70196012F966CAD55
:105DE0007DAD8EAD9FAD2F970F94D92C9B01AC014B
:105DF000C501B4010F94DD302B966CAF7DAF8EAF33
:105E00009FAF2B9759E164965FAF64979201A3010E
:105E10006F966CAD7DAD8EAD9FAD6F970F94DE30FC
:105E200069837A838B839C832B962CAD3DAD4EADDD
:105E30005FAD2B97A3966CAD7DAD8EAD9FADA39757
:105E40000F94DE306D837E838F839887AF962CAD61
:105E50003DAD4EAD5FADAF9769857A858B859C85ED
:105E60000F94DE3069877A878B879C87E3962CAD09
:105E70003DAD4EAD5FADE3976D857E858F8598898D
:105E80000F94DE306D877E878F87988B809100021C
:105E9000882321F0CE0101960E94327DE0904E04CD
:105EA00089819A81AB81BC8188A399A3AAA3BBA352
:105EB0008D819E81AF81B8858CA39DA3AEA3BFA326
:105EC00089859A85AB85BC8588A799A7AAA7BBA712
:105ED000CE0180960E9465638E01055C1F4F9E0176
:105EE000235F3F4FAE01485D5F4FBE016C5D7F4F4A
:105EF000CE0180960E9498CF69968EAD9FAD69972E
:105F0000019669969FAF8EAF69979FCEE0904E0441
:105F10008091E5069091E606A091E706B091E8062B
:105F200088A399A3AAA3BBA38091E9069091EA064E
:105F3000A091EB06B091EC068CA39DA3AEA3BFA3EA
:105F40008091ED069091EE06A091EF06B091F006DB
:105F500088A799A7AAA7BBA7CE0180960E946563D0
:105F60008E01055C1F4F21EF36E0AE01485D5F4FAB
:105F7000BE016C5D7F4FCE0180960E9498CF0E943B
:105F80009FB80E946D630C94D042EEE1FBE28491D5
:105F90008F010F5F1F4F882321F00E9440A1F8015D
:105FA000F6CFE1E4F2E084918F010F5F1F4F882369
:105FB00011F40C94D0420E9440A1F801F4CF80E586
:105FC0000E947AB7882329F00E94D4B66B017C0125
:105FD00003C0C12CD12C760183E50E947AB78823B7
:105FE00061F00E9414B720E030E04AE754E40F94D7
:105FF000D92C0F9427326B017C010E9435DB8091F4
:106000005C02811105C060E087E592E00E9472AAFF
:106010000E946D6380916A1190916B11A0916C1137
:10602000B0916D11C80ED91EEA1EFB1E0E94DB50F6
:10603000DC01CB018C199D09AE09BF09B7FD02C077
:106040000C94D04280E00F946104F0CF41E061E015
:1060500081E00E94FDAF81110C94D04280E50E9446
:106060007AB7882321F00E94E4B6F62E01C0F12C05
:1060700083E50E947AB7882321F00E94E4B68B0161
:1060800002C00CE010E084E50E947AB781110E9402
:10609000E4B682E50E947AB7882329F00E9414B7FB
:1060A0004B015C0106C0812C912C40EDA42E40E4F4
:1060B000B42EB1E0FB1611F40C94D042E2E0FE12D3
:1060C0008DC080E090E0A4E3B2E489839A83AB833F
:1060D000BC8380E090E0A0E3B3E48D839E83AF8334
:1060E000B88780E090E0A0E8BFE389879A87AB8714
:1060F000BC87002311F40C94D04218A219A21AA252
:106100001BA29E01205E3F4FAE01475F5F4FBE0165
:106110006B5F7F4FCE0101960E94E3B010E0E12C4F
:10612000F12C18A219A21AA21BA2B7010F2C000C65
:10613000880B990B0F947A2C2CE739ED40E25FE342
:106140000F94D92C2B013C010F94B731A501940178
:106150000F94D92C20E030E040E353E40F94DE307C
:106160006BAF7CAF8DAF9EAFC301B2010F943F33D5
:10617000A50194010F94D92C20E030E044E352E4CF
:106180000F94DE3023966CAF7DAF8EAF9FAF239719
:10619000AE01405E5F4FBE01655C7F4FCE01CF9682
:1061A0000E940EB2FFEFEF1AFF0A2AE0E216F10496
:1061B00009F0B7CF1F5F101708F4B1CF18A219A2CA
:1061C0001AA21BA2AE01405E5F4FBE016B5F7F4F04
:1061D000CE0101960E940EB20C94D04280E090E075
:1061E000A6EEB2E489839A83AB83BC8340E050E09F
:1061F00060E373E44D835E836F83788780E090E093
:10620000A0E8BFE389879A87AB87BC87C12CD12CD4
:1062100024E3E22E22E4F22EC8A2D9A2EAA2FBA233
:106220004CA35DA36EA37FA388A799A7AAA7BBA72A
:106230001BAE1CAE1DAE1EAE9E01255C3F4FAE01D7
:10624000485D5F4FBE016C5D7F4FCE0180960E941E
:10625000E3B0112715950795F12C8F2D90E080174D
:10626000910714F00C94D0421BAE1CAE1DAE1EAEB6
:10627000AE01455C5F4FBE016B5F7F4FCE01019663
:106280000E940EB21BAE1CAE1DAE1EAEAE01455C32
:106290005F4FBE016C5D7F4FCE0180960E940EB2B3
:1062A000F394DBCF81E0809327021092AE120C941E
:1062B000D04241E061E081E00E94FDAF81110C9489
:1062C000D04280E090E0A0E2B1E489839A83AB837E
:1062D000BC8380E090E0A6E3B3E48D839E83AF832C
:1062E000B88780E090E0A0EAB1E489879A87AB871D
:1062F000BC8780E50E947AB7882319F00E94E4B633
:1063000001C060E068A3BE016F5F7F4FCE01809641
:106310000F94A1220C94D04280E00E949C750C94B2
:10632000D04280E00E9490B613E001E010924E1837
:1063300010924F1810925018109251180093720436
:1063400024982C9A149A0E94376510927204249A09
:106350002C9814988091840E882351F08091840E9B
:10636000882369F08EED92E00F946F030C94D04275
:106370008EE093E00F946F031150C1F6EFCFE5EF7D
:10638000F2E084918F010F5F1F4F882321F00E945C
:1063900040A1F801F6CF8FE692E00F946F0380E6FC
:1063A00092E00F94DF03C090F30ED090F40EE090D3
:1063B000F50EF090F60E88E50E947AB7811108C0BC
:1063C00020E030E0A901C701B6010F94DE3002C021
:1063D0000E9414B768A379A38AA39BA3C090F70E69
:1063E000D090F80EE090F90EF090FA0E89E50E9438
:1063F0007AB7811108C020E030E0A901C701B601D9
:106400000F94DE3002C00E9414B76B017C016983D7
:106410007A838B839C8388A099A0AAA0BBA022E644
:1064200030E140E450ECC501B4010F94043387FF20
:1064300002C00C94D04222E430E043E253E4C501B0
:10644000B4010F94742C181614F40C94D04221E368
:1064500038E040E850ECC701B6010F94043387FFE1
:1064600002C00C94D04222E430E048E253E4C70179
:10647000B6010F94742C181614F40C94D0420C949A
:10648000904381E0809353040C94D0420E9435DB0A
:1064900040E453E025965FAF4EAF2597F3EFEF2E24
:1064A000FEE0FF2EA2E5CA2EA8E1DA2E312C00E094
:1064B00010E02596AEADBFAD25978D912596BFAF67
:1064C000AEAF25970E947AB78823B9F10E9414B71E
:1064D0002B013C01133049F0F601208131814281CA
:1064E00053810F94DD302B013C01D7012D913D915B
:1064F0004D915C91C301B2010F94DD304B015C0101
:106500002DEB37E346E855EB0F94043387FD0AC0C3
:106510002DEB37E346E855E3C501B4010F94742C25
:1065200018165CF4133011F001E002C033243394E8
:10653000F70140825182628273821F5FF4E0EF0EA6
:10654000F11C24E0C20ED11C143009F0B2CF00239C
:1065500019F00E94A8B503C031100E9493F20E9466
:1065600041D50C94D04280911507909116078D3734
:10657000910509F4F0C40CF0EFC08D34910509F4D5
:10658000B7C40CF05CC08931910509F4D6C21CF582
:106590008431910509F48EC27CF48131910509F4AE
:1065A0007EC22CF4029708F4F5C10C94D0424297B5
:1065B00009F467C50C94D0428631910509F482C272
:1065C0000CF47CC28731910509F482C2489709F422
:1065D00095C20C94D0428F31910509F455C47CF4D6
:1065E0008B31910509F4C7C20CF4B7C28C31910507
:1065F00009F4C5C24E9709F4CCC20C94D042893438
:10660000910509F46DC464F48032910509F4F0C376
:106610008A9711F00C94D0420F9437230C94D042F7
:106620008B34910509F460C48C34910511F00C94FD
:10663000D0428BEF94E10E9412510C94D0428B36E1
:10664000910509F484C40CF044C08435910509F423
:1066500018C5E4F48135910509F4F8C44CF48E347E
:10666000910511F00C94D0420E94A1D90C94D04213
:106670008235910509F401C58335910511F00C941B
:10668000D04281E0809352040C94D0428836910528
:1066900009F432C48CF48535910509F429C58C358B
:1066A000910511F00C94D04260E4E62E63E0F62EE2
:1066B00003E01FE0D12C37C58936910509F428C4C1
:1066C0008A36910511F00C94D0420E94FAD80C94AD
:1066D000D0428337910509F4A5C5ECF48E369105B7
:1066E00009F40EC44CF48D36910511F00C94D0428F
:1066F0000E9435D70C94D0428F36910509F404C41A
:106700008237910511F00C94D0420E9435DB0E9433
:1067100041D50C94D0428737910509F490C56CF4AB
:106720008537910509F482C58637910511F00C94DF
:10673000D0420E94975E0C94D0428837910509F4AC
:106740008DC58937910511F00C94D04210924718ED
:10675000109246180C94D042803931E0930711F41E
:106760000C943B410CF084C0833D910509F47BC639
:106770000CF042C0883C910509F47BC5C4F4813912
:10678000910509F472C54CF48C38910511F00C9404
:10679000D0420E9495D60C94D0428B39910509F4D1
:1067A000BBC38E3B910509F4BBC30C94D0428C3C17
:1067B000910509F466C56CF4893C910509F45DC541
:1067C0008B3C910511F00C94D0420E94075E0C9412
:1067D000D0428D3C910509F4C0C58E3C910511F065
:1067E0000C94D04240E4C42E43E0D42E53E7E52E6F
:1067F00054E0F52E10E025C68C3251E0950709F4DF
:10680000B5C7ACF48D3D910509F41AC734F48C3D3D
:10681000910509F408C70C94D042823E910509F411
:1068200056C78232914009F494C70C94D0428F32FB
:10683000E1E09E0711F40C94B13C64F48D3221E048
:10684000920709F496C78E32914011F40C945D3C86
:106850000C94D042803341E0940709F4B1C78336E9
:10686000914011F00C94D0420E946D570C94D0428C
:106870008835A2E09A0711F40C9464420CF040C0F1
:106880008C3AE1E09E0711F40C944442B4F482394E
:1068900021E0920711F40C94424114F40C943E410F
:1068A000843A41E0940711F40C944641893A9140AE
:1068B00011F40C94C6410C94D042863FA1E09A0793
:1068C00011F40C944A427CF4843FE1E09E0711F4F9
:1068D0000C944742853F914011F00C94D0420F94A4
:1068E0002C110C94D042873F21E0920711F40C94B4
:1068F0004D428C31924011F40C9459420C94D04288
:106900008F3843E0940711F40C946D42FCF4843802
:10691000A3E09A0711F40C9467424CF4833593403A
:1069200011F00C94D0420E94285C0C94D0428A381A
:10693000F3E09F0711F40C946A428B38934011F0F6
:106940000C94D0420E9488570C94D042823933E094
:10695000930711F40C9473427CF4803953E095074B
:1069600011F40C9470428139934011F00C94D04290
:106970000E94F5570C94D042803AB3E09B0709F48B
:1069800076C2873E934011F00C94D0420E94585733
:106990000C94D042009113071091140780E50E94D7
:1069A0007AB7882361F00E94D4B66B017C01BB24C6
:1069B000B394672B682B692B31F4B12C04C0B12C34
:1069C000C12CD12C760183E50E947AB78823F1F09F
:1069D0000E9414B720E030E04AE754E40F94D92C29
:1069E0000F9427326B017C01B11012C0672B682B0A
:1069F000692B71F40115110559F0D8018C91882388
:106A000039F061E0C8010E9490AA07C0BB2091F351
:106A100060E08FE094E00E9472AA81E08093810799
:106A20000E9435DB0E946D63C114D104E104F104BE
:106A3000F1F080916A1190916B11A0916C11B0915D
:106A40006D11C80ED91EEA1EFB1E0E94DB50DC0130
:106A5000CB018C199D09AE09BF09B7FF1CC08091FD
:106A600081078823C1F080E00F946104EECF80910C
:106A70008107882321F080E00F946104F8CF809192
:106A8000FB1460E0823019F481E094E002C082EFF0
:106A900093E00E9472AA109281070C94D04260E0A9
:106AA00082E294E00E9472AA17981698159814989A
:106AB0000C94D0420F94DC230C94D0420E9446EDFB
:106AC0000C94D04210925515109256150C94D04249
:106AD000E0911307F09114078081882329F0803218
:106AE00009F410823196F8CF40E061E080911307FD
:106AF000909114070E94E0FF0C94D04219821A82F0
:106B00001B821C8218A219A21AA21BA28091CC0679
:106B1000882341F040E0BE016F5F7F4FCE01809639
:106B20000E947B7F80915615882319F081E0809325
:106B300055150F94D91C0C94D042109255158BEF1B
:106B400094E10E9412518BE294E09093441180935F
:106B500043110E94C7B20C94D042809156158823ED
:106B600011F40C94D04283E50E947AB781110C9401
:106B7000E7430C94D0420F949F230C94D04240E002
:106B800060E080911307909114070E94E0FF0C943D
:106B9000D04280915615882311F40C94D04287E49A
:106BA00097E10E94D1A387E497E10F944A0A1092DB
:106BB00054151092531500911307109114078091EA
:106BC0005615882311F40C94D0420E94D5FF1D82E3
:106BD00018861C821B8281E394E09A83898389EA68
:106BE00095E19093C9158093C815F80180818F3283
:106BF00009F07EC06FE270E0C8010F942334019663
:106C00007C019E012F5F3F4F3901E114F10409F42B
:106C100077C06FE270E0C7010F9423344C010097F6
:106C200009F46DC0E816F90608F069C04DB65EB605
:106C30006C01CE18DF081C140CF062C00C2C000C88
:106C4000DD08C60101964DB75EB7481B590B0FB65C
:106C5000F8945EBF0FBE4DBF8DB79EB701965C0125
:106C6000A601B7010F944334F501EC0DFD1D108210
:106C70007501D7018D917D01882319F00E9440A1F3
:106C8000F8CF8AE00E9440A16091C8157091C915A3
:106C90006115710511F06C5F7F4F21E0A501CE01F8
:106CA00005960F945B0D811115C0B50186E594E042
:106CB0000E940F648EE20E9440A18AE00E9440A1DF
:106CC0000FB6F8945EBE0FBE4DBEC3010E94A280F7
:106CD0000C94D0427092C9156092C8157401BFEF30
:106CE000EB1AFB0A0FB6F8945EBE0FBE4DBE8DCFF9
:106CF0008AEC95E19093C9158093C81501C087016E
:106D00006091C8157091C9156115710511F06C5F1E
:106D10007F4F18A21BA222E0A801CE0180960F94FB
:106D20005B0D811102C0F12C1EC0CE0180960E9425
:106D300014FD8823C1F36CA57DA58EA59FA541E018
:106D40000F94F220882379F3E8A920E2E29FF00172
:106D50001124E35DF04F309731F385EE80831BA261
:106D60000F94B220F82ECE0180960E9486B8FF20A4
:106D700009F1E0E3F4E084917F013FEFE31AF30AC5
:106D8000882321F00E9440A1F701F5CFD8018D9111
:106D90008D01882319F00E9440A1F8CF8AE00E945B
:106DA00040A11092F8171092F9171092FA1710924A
:106DB000FB1718C0EEE3F4E084917F01BFEFEB1AFC
:106DC000FB0A882321F00E9440A1F701F5CFF801CA
:106DD00081918F01882319F00E9440A1F8CF8EE2A3
:106DE0000E9440A1CE0101960E94A2800C94D04244
:106DF0008091551581110E9435DB809156158823AD
:106E000011F40C94D04280E50E947AB7882319F0DF
:106E10000E9405B703C080E50E944BB7182F482F8A
:106E200061E080911307909114070E94E0FF83E5D1
:106E30000E947AB7882381F00E94E4B6AB01BC01BE
:106E40004093F8175093F9176093FA177093FB1754
:106E500087E497E10F94ED0780915615882319F088
:106E600081E08093551511110C94D04262CE80912F
:106E700013079091140721E02093541540E060E03F
:106E80000E94E0FF0C94D0428BEF94E10E94E75007
:106E900068A379A38AA39BA3BE016F5F7F4FCE0136
:106EA00080960E942F4A60E0CE0101960E9490AA2F
:106EB000E9E3FBE284918F010F5F1F4F882321F0EC
:106EC0000E9440A1F801F6CFBE016F5F7F4F8AE6B6
:106ED00094E00E940F648AE00E9440A10C94D0428A
:106EE0000E94C8DA0C94D0420F94D91C0C94D04262
:106EF0000F942C1D0C94D0420E9468D90C94D0425F
:106F00000E9425D70C94D0420E94AED60C94D04259
:106F10000E944BD90C9433480E941DD90C94D04246
:106F20008091E00883FF02C00C94D04283E50E9468
:106F30007AB72C968FAF2C9781110C94F84382E589
:106F40000E947AB781110C94F8430C94D0420E94AD
:106F5000EBD80C94D0428CE40E944BB7882319F0F4
:106F60000E9414B704C060E070E080E090EC6BAF6A
:106F70007CAF8DAF9EAF80E090E0A0E2B1E489836A
:106F80009A83AB83BC8380E090E0A6E3B3E48D8377
:106F90009E83AF83B88780E090E0A0EAB1E4898760
:106FA0009A87AB87BC8788E50E947AB7882379F0F7
:106FB00088E50E947AB7882319F00E9414B703C0AD
:106FC00060E070E0CB0169837A838B839C8389E5E1
:106FD0000E947AB7882379F089E50E947AB78823DE
:106FE00019F00E9414B703C060E070E0CB016D831C
:106FF0007E838F8398878AE50E947AB7882379F009
:107000008AE50E947AB7882319F00E9414B703C05A
:1070100060E070E0CB0169877A878B879C8718A234
:1070200019A21AA21BA28091CC0681110C94D04205
:1070300000E020E0AE01405E5F4FBE016F5F7F4F1A
:10704000CE01CB960E94847E0C94D0420E948C96F6
:107050000E9435DB0F94D6031092D2081092D1080B
:1070600068EE73E080E090E00E94F28A60E08FE9D1
:1070700094E00E9472AA0C94D042109252040C9494
:10708000D04283E50E947AB78823A1F00E9414B70A
:1070900020E030E04AE754E40F94D92C0F942732D3
:1070A00060934702709348028093490290934A028A
:1070B0000C94D04288E50E944BB781110C94744522
:1070C00089E50E944BB781110C9474458AE50E94B2
:1070D0004BB781110C94744585E40E944BB7811124
:1070E0000C9474450E9435DB0F94D6030C94D04267
:1070F00083E50E944BB7882311F40C94D0420E9480
:1071000014B720E030E04AE754E40F94D92C0F94F0
:10711000273260936E1170936F118093701190936A
:1071200071110C94D042D7018D917D010E944BB713
:10713000882309F46DC0B3E0DB1263C00E9414B76A
:107140004B015C0120E030E040EA51E40F94742CE4
:1071500087FF4EC0A501940160910F0F7091100F31
:107160008091110F9091120F0F94BA312B013C01B5
:107170009B01AC016091910E7091920E8091930EE3
:107180009091940E0F94D92C6093910E7093920E5F
:107190008093930E9093940EA30192016091C90E77
:1071A0007091CA0E8091CB0E9091CC0E0F94D92C79
:1071B0006093C90E7093CA0E8093CB0E9093CC0E41
:1071C0006091F2087091F3088091F4089091F508AD
:1071D0000F94782CA30192010F94D92C0F9427328D
:1071E0006093F2087093F3088093F4089093F50885
:1071F00080920F0F9092100FA092110FB092120F69
:1072000007C00E9414B7F80160837183828393835F
:10721000D3940C5F1F4FF4E0DF1285CF0E944EE540
:107220000C94D0420E94FAD40C94D04260E0809139
:107230001307909114070E9490AA0C94D04281E009
:107240008093720424982C9A149A0E948B4910926D
:107250007204249A2C9814980C94D04281E0809364
:107260004718809346180C94D0420E941ED60C9466
:10727000D0420E944E5E0C94D0420E94295E0C9433
:10728000D04283E50E944BB78823D9F00E9414B7FF
:10729000AB01BC014093A90E5093AA0E6093AB0EB4
:1072A0007093AC0E4093A10E5093A20E6093A30E68
:1072B0007093A40E8FE095E00E94B2638AE00E9472
:1072C00040A180E50E944BB7882399F00E9414B733
:1072D000AB01BC014093A90E5093AA0E6093AB0E74
:1072E0007093AC0E82EF94E00E94B2638AE00E9439
:1072F00040A182E50E944BB7882399F00E9414B701
:10730000AB01BC014093A50E5093A60E6093A70E4F
:107310007093A80E83ED94E00E94B2638AE00E940D
:1073200040A184E50E944BB7882311F40C94D0420D
:107330000E9414B7AB01BC014093A10E5093A20E62
:107340006093A30E7093A40E85EB94E00E94B26349
:107350008AE00E9440A10C94D04283E50E944BB782
:10736000882351F00E9414B760939D0E70939E0E77
:1073700080939F0E9093A00E84E50E944BB78823C4
:1073800051F00E9414B76093990E70939A0E8093F7
:107390009B0E90939C0E82E40E944BB7882351F081
:1073A0000E94D4B66093950E7093960E8093970EBC
:1073B0009093980E88E50E944BB7882351F00E9465
:1073C00014B76093850E7093860E8093870E90930A
:1073D000880E89E50E944BB7882351F00E9414B7AC
:1073E0006093890E70938A0E80938B0E90938C0E0F
:1073F0008AE50E944BB7882351F00E9414B760932E
:107400008D0E70938E0E80938F0E9093900E85E468
:107410000E944BB7882311F40C94D0420E9414B7F9
:107420006093910E7093920E8093930E9093940EAE
:107430000C94D0421F5FF4E0EF0EF11C133009F4FE
:107440008EC8D6018D916D010E944BB7882391F3B0
:107450000E9414B7F7016083718382839383812F25
:107460000E946BB2E7CFE9E3FBE284918F010F5FEB
:107470001F4F882321F00E9440A1F801F6CF83E539
:107480000E944BB7882321F00E9405B78093000229
:10749000EFE5F5E084918F010F5F1F4F882321F006
:1074A0000E9440A1F801F6CF80910002811103C033
:1074B000EBE5F5E002C0E7E5F5E084918F010F5FB1
:1074C0001F4F882321F00E9440A1F801F6CFEFE47E
:1074D000F5E084918F010F5F1F4F882321F00E94F8
:1074E00040A1F801F6CF20915218309153184091E5
:1074F0005418509155186091AE067091AF06809166
:10750000B0069091B1060F94DE30AB01BC018DE462
:1075100095E00E94B263209156183091571840911F
:107520005818509159186091B2067091B306809125
:10753000B4069091B5060F94DE30AB01BC018AE42D
:1075400095E00E94B26320915A1830915B184091E7
:107550005C1850915D186091B6067091B7068091E5
:10756000B8069091B9060F94DE30AB01BC0187E4F8
:1075700095E00E94B263EFE3F5E084918F010F5F25
:107580001F4F882321F00E9440A1F801F6CF2091DF
:1075900052183091531840915418509155186091D9
:1075A0001B0270911C0280911D0290911E020F948B
:1075B000DE30AB01BC018DE395E00E94B263209107
:1075C0005618309157184091581850915918609199
:1075D0001F027091200280912102909122020F944B
:1075E000DE30AB01BC018AE395E00E94B2632091DA
:1075F0005A1830915B1840915C1850915D18609159
:1076000023027091240280912502909126020F940A
:10761000DE30AB01BC0187E395E00E94B2638AE0F3
:107620000E9440A1BDC783E50E947AB7882309F470
:10763000B7C70E94E4B67093020260930102B0C71C
:107640008DED90E00E9446B88111AAC783E50E94A3
:107650007AB7882309F4A4C70091A31110E00E940F
:10766000E4B6000F111FF801E15DFD4F71836083E7
:107670008091A31190E08C01000F111F000F111FCA
:107680009801295C3D4F7901880F991FFC01E15D4C
:10769000FD4F60817181072E000C880B990B0F94B0
:1076A0007A2C2AE037ED43E25CE30F94D92CF80101
:1076B000E554F74F20813181428153810F94D92CB9
:1076C000D7016D937D938D939C93139769C780E544
:1076D0000E944BB7882309F463C70E94E4B6F62ED4
:1076E000062F172F83E50E947AB7882321F00E9486
:1076F000E4B66B0103C0CC24CA94DC2CC60101960D
:10770000039708F04DC717FD4BC70E9435DBBFEF4D
:10771000CB16DB0631F0CA94CD2871F401E010E0FD
:107720000DC08F2D0E94E74E31E020E0892B09F03B
:1077300030E0032F122F02C000E010E08F2D0E94D6
:10774000E74E8017910709F42BC780E00F9461047E
:10775000F5CF8AE50E947AB781110C94974583E5AD
:107760000E947AB781110C9497451AC70E94D25D86
:1077700017C785E40E947AB7811103C00E94C47DB7
:107780000FC70E94F4B68823C9F3EEE1FBE28491AF
:107790008F010F5F1F4F811103C003EF12E004C080
:1077A0000E9440A1F801F3CFD8018D918D0188236B
:1077B00019F00E9440A1F8CF8AE00E9440A1F0C6D3
:1077C00080E50E944BB7882351F00E9414B7609364
:1077D000680E7093690E80936A0E90936B0E89E425
:1077E0000E944BB7882381F00E9414B72CEA35EC35
:1077F00047E25EE30F94D92C6093640E7093650E9C
:107800008093660E9093670E84E40E944BB78823A2
:1078100081F00E9414B72CEA35EC47E25EE30F9446
:10782000BA316093600E7093610E8093620E9093F4
:10783000630EE9E3FBE284918F010F5F1F4F882302
:1078400021F00E9440A1F801F6CF4091680E5091BE
:10785000690E60916A0E70916B0E88E895E00E9447
:10786000B2632CEA35EC47E25EE36091640E7091FE
:10787000650E8091660E9091670E0F94BA31AB0140
:10788000BC0184E895E00E9495632CEA35EC47E260
:107890005EE36091600E7091610E8091620E909136
:1078A000630E0F94D92CAB01BC0180E895E00E94D7
:1078B00095638AE00E9440A173C683E50E944BB79E
:1078C000182F882371F00E9414B70F9422327093FE
:1078D00036026093350221E0672B09F020E0209307
:1078E000D70880E50E944BB7882359F020913502D4
:1078F00030913602232B11F00E9405B78093D708F0
:107900004FC611114DC6E9E3FBE284918F010F5F71
:107910001F4F882321F00E9440A1F801F6CF8091EB
:10792000D708811103C063EE72E002C066E473E021
:1079300081EA95E00E940F646091350270913602F1
:1079400080E995E00E94F663ECE8F5E084918F0110
:107950000F5F1F4F882309F423C60E9440A1F8013E
:10796000F5CF85E40E947AB7882321F00E94E4B61F
:107970007B0102C0E12CF12C83E40E947AB78823BA
:1079800041F00E94E4B6CF57DF4F6883C158D04022
:1079900006C045E0CF57DF4F4883C158D04085E54A
:1079A0000E947AB7882319F00E9405B703C085E5C5
:1079B0000E944BB7CF56DF4F8883C159D040F7FCA8
:1079C00007C0812C912CB6E1AB2EB3E4BB2E06C0D0
:1079D000812C912CACE8AA2EA2E4BA2E83E50E9459
:1079E0007AB7882321F00E9414B74B015C01E1149F
:1079F000F10411F41092A3112496EFAE24970E9483
:107A0000DB502B013C0124965FAD249757FD0EC03F
:107A100080E090E0A0E5B1E4C357DF4F888399830D
:107A2000AA83BB83CD58D04004E10DC020E030E0F4
:107A300040E051E4C357DF4F288339834A835B8397
:107A4000CD58D0400CE361E06E0D623028F4F4E0D4
:107A5000EF2EF3E0FF2E0BC007E113E0D8018D916C
:107A60008D01882309F4A8CE0E9440A1F7CFF70129
:107A700081917F01882319F00E9440A1F8CF8AE00C
:107A80000E9440A10E948C962496FFAD2497F7FF98
:107A900004C08FE78093A2110AC024962FAD2497CB
:107AA000E22F220FFF0BEF55FE4E8FE78083C501BB
:107AB000B4010F942232072E000C880B990B0F94FF
:107AC0007A2C60966FAF609764967FAF64976896E4
:107AD0008FAF68976C969FAF6C97202F30E0A8EE21
:107AE000B3E00F94CE30CE56DF4F688379838A831C
:107AF0009B83C259D040DC01CB01840D951DA61D8E
:107B0000B71DC256DF4F88839983AA83BB83CE59A2
:107B1000D04081E080932D02CB57DF4F48825982BD
:107B20006A827B82C558D040CA56DF4F488259824C
:107B30006A827B82C659D040CC57DF4F1882C45826
:107B4000D040C656DF4F188219821A821B82CA594A
:107B5000D040E4961FAEE49790E4E8969FAFE89794
:107B6000ACE1AC96AFAFAC97B6E4E096BFAFE097B0
:107B7000EC961FAEEC97ED961FAEED97EE961FAE0E
:107B8000EE97EF961FAEEF97AB961CAE1DAE1EAEF6
:107B90001FAEAB97A7961CAE1DAE1EAE1FAEA7972D
:107BA000C12CD12C76012FE730E040E050E02F9639
:107BB0002CAF3DAF4EAF5FAF2F977FE7872E912C55
:107BC000A12CB12CC757DF4F188219821A821B8251
:107BD000C958D04031E0CD57DF4F3883C358D0402B
:107BE000A1961FAE1EAEA19710E0212C312C00E013
:107BF00024964FAD2497842F440F990BDC01AF5589
:107C0000BE4ECE55DF4FB983A883C25AD040880FED
:107C1000991F880F991FFC01ED52F74FC158DF4F94
:107C2000F983E883CF57D040CF57DF4F2881C15821
:107C3000D040022E000C330BCF57DF4F39832883FF
:107C4000C158D04080912D02882309F440C10E9480
:107C5000DB502B966CAF7DAF8EAF9FAF2B97809193
:107C60007007882309F40FC10E94499724963FADFD
:107C7000249737FF09C01091A4112090A5113090CE
:107C8000A6110091A7110FC0C158DF4FA881B9817B
:107C9000CF57D0401C9111962C90119712963C9082
:107CA000129713960C91212F322D432D502FEC96C5
:107CB0006FADEC97ED967FADED97EE968FADEE97AD
:107CC000EF969FADEF970F94742C87FF0CC0EC9646
:107CD0001FAFEC97ED962FAEED97EE963FAEEE9779
:107CE000EF960FAFEF97212F322D432D502FE496B3
:107CF0006FADE497E8967FADE897AC968FADAC9703
:107D0000E0969FADE0970F940433181664F4E49660
:107D10001FAFE497E8962FAEE897AC963FAEAC97CE
:107D2000E0960FAFE097CD57DF4FB881C358D040F2
:107D300060962FAD609764963FAD649768964FAD9F
:107D400068976C965FAD6C97612F722D832D902F85
:107D5000BB2309F47AC00F94043318160CF093C0B7
:107D60002B962CAD3DAD4EAD5FAD2B97241935094B
:107D700046095709C755DF4F288339834A835B83F8
:107D8000C95AD040DA01C90188589341A109B10903
:107D9000B7FD79C0D501C4012F962CAD3DAD4EADD8
:107DA0005FAD2F97821B930BA40BB50B24963FADB1
:107DB0002497B595A7959795879537FF03C080932E
:107DC000A21107C0CE55DF4FE881F981C25AD040D9
:107DD0008083C755DF4F288139814A815B81C95A29
:107DE000D040C757DF4F288339834A835B83C95804
:107DF000D04060963FAD6097EC963FAFEC976496AD
:107E00004FAD6497ED964FAFED9768965FAD68976D
:107E1000EE965FAFEE976C968FAD6C97EF968FAF47
:107E2000EF972B962CAD3DAD4EAD5FAD2B97CB575D
:107E3000DF4F288339834A835B83C558D040CD57B1
:107E4000DF4F1882C358D0401EC00F94742C87FF98
:107E50001AC02B968CAD9DADAEADBFAD2B97CB5759
:107E6000DF4F288139814A815B81C558D040821B10
:107E7000930BA40BB50BAC01BD01485853416109EC
:107E8000710977FFCEC620E030E040EA51E4609609
:107E90006FAD609764967FAD649768968FAD689775
:107EA0006C969FAD6C970F94DE309B01AC01612FF7
:107EB000722D832D902F0F94043318167CF4EFEA63
:107EC000F6E084918F010F5F1F4F811103C00E9464
:107ED0008C9666C30E9440A1F801F3CF2B968CAD1F
:107EE0009DADAEADBFAD2B97CA56DF4F288139810E
:107EF0004A815B81C659D040821B930BA40BB50B02
:107F0000B7FDC5C00F94F10E8AE00E9440A12B96E8
:107F10008CAD9DADAEADBFAD2B978053984FAF4F9D
:107F2000BF4FCA56DF4F88839983AA83BB83C65944
:107F3000D040CC57DF4F9881C458D040911182C0B7
:107F4000C656DF4F288139814A815B81CA59D040AA
:107F5000612F722D832D902F0F94043318160CF07F
:107F600058C0C357DF4F288139814A815B81CD5882
:107F7000D04060966FAD609764967FAD64976896C9
:107F80008FAD68976C969FAD6C970F94DD309B0119
:107F9000AC01A1E0CC57DF4FA883C458D040612F7B
:107FA000722D832D902F0F94043318162CF0CC577C
:107FB000DF4F1882C458D04020E030E040E050E469
:107FC000612F722D832D902F0F94DE30C656DF4F18
:107FD000688379838A839B83CA59D0402B962CADC2
:107FE0003DAD4EAD5FAD2B97CE56DF4F8881998169
:107FF000AA81BB81C259D040280F391F4A1F5B1F7D
:10800000C256DF4F288339834A835B83CE59D040E1
:108010003EC02B968CAD9DADAEADBFAD2B97C2567D
:10802000DF4F288139814A815B81CE59D040821B44
:10803000930BA40BB50BB7FD2AC041E956E060EAEB
:1080400076E020C020E030E040EA51E460966FAD79
:10805000609764967FAD649768968FAD68976C96CD
:108060009FAD6C970F94DD309B01AC01612F722D99
:10807000832D902F0F94742C87FF09C041E756E0A1
:1080800061E876E024968FAD24970E946C972B963A
:108090008CAD9DADAEADBFAD2B97880F991FAA1FBC
:1080A000BB1FCB57DF4F288139814A815B81C5587F
:1080B000D040821B930BA40BB50B84199509A6091C
:1080C000B70981389F44A241B10568F0E3E5F6E0C5
:1080D00084918F010F5F1F4F882309F4F8CE0E940F
:1080E00040A1F801F5CFA1964EAD5FADA197CF5756
:1080F000DF4F88819981C158D040841795070CF0D3
:10810000B7C0E6EFF5E084918F010F5F1F4F882322
:1081100021F00E9440A1F801F6CF24969FAD24974C
:1081200097FD03C00DEC13E002C007EE12E0B801AA
:1081300084EE95E00E940F64B701A60180EE95E001
:108140000E94B2638AE00E9440A1B8018EEC95E0E3
:108150000E940F64A7964CAD5DAD6EAD7FADA79745
:108160008AEC95E00E94B2638AE00E9440A1B801C7
:1081700088EB95E00E940F64AB964CAD5DAD6EADA3
:108180007FADAB9784EB95E00E94B2638AE00E94DA
:1081900040A1CF56DF4FA881C159D040AA2309F48E
:1081A000FFC12496BFAD2497B7FF31C0C092680EBF
:1081B000D092690EE0926A0EF0926B0E2CEA35ECCA
:1081C00047E25EE3A7966CAD7DAD8EAD9FADA79700
:1081D0000F94D92C6093640E7093650E8093660E95
:1081E0009093670E2CEA35EC47E25EE3AB966CADFC
:1081F0007DAD8EAD9FADAB970F94BA316093600E9D
:108200007093610E8093620E9093630EC9C1C09209
:10821000740ED092750EE092760EF092770E2CEAE4
:1082200035EC47E25EE3A7966CAD7DAD8EAD9FADBC
:10823000A7970F94D92C6093700E7093710E809352
:10824000720E9093730E2CEA35EC47E25EE3AB9628
:108250006CAD7DAD8EAD9FADAB970F94BA31609391
:108260006C0E70936D0E80936E0E90936F0E98C18E
:108270000E94A0AAE7CC0E9435DB92C181E00E9457
:10828000C8B18EC180E00E94C8B18AC18091F30E4E
:108290009091F40EA091F50EB091F60E89839A8319
:1082A000AB83BC838091F70E9091F80EA091F90EEC
:1082B000B091FA0E8D839E83AF83B8878091FB0EB9
:1082C0009091FC0EA091FD0EB091FE0E89879A87C9
:1082D000AB87BC8786E50E944BB7882321F080E5F9
:1082E00097E00F94732783E50E944BB7882331F002
:1082F0000E9405B7182F0E9490B601C010E0F090C0
:10830000840E111103C0E9E3FBE21AC0F110FBCFA8
:10831000EEE1FBE284918F010F5F1F4F882321F074
:108320000E9440A1F801F6CFE1E3F7E084918F01CC
:108330000F5F1F4F882339F30E9440A1F801F6CF49
:1083400084918F010F5F1F4F882321F00E9440A16D
:10835000F801F6CFF11003C06FEE72E002C06BEED1
:1083600072E083E297E00E940F648AE00E9440A1DD
:108370004CE050E063EF7EE0CE0101960F94EF33C6
:10838000892B09F40DC10E9441D50AC18AE50E94DA
:108390004BB7882329F180914C0490914D04892B8F
:1083A00019F00E9414B708C060914E1870914F18D0
:1083B00080915018909151186093C4087093C5082B
:1083C0008093C6089093C70880E090E0A0E8BFE3E0
:1083D0008093C8089093C908A093CA08B093CB08AB
:1083E00086E40E944BB7882381F10E9414B720E0F5
:1083F00030E040E85FE30F94043318166CF40E94F9
:1084000014B720E030E040E85FE30F94043318161F
:1084100084F00E9414B711C00E9414B720E030E02D
:10842000A9010F94742C87FFEACF60E070E0CB01C4
:1084300004C060E070E080E89FE36093C808709338
:10844000C9088093CA089093CB0883E50E944BB774
:10845000882351F00E9414B7609331027093320266
:1084600080933302909334028AE50E944BB78111C6
:1084700097C086E40E944BB7811192C083E50E94A9
:108480004BB781118DC06AC50E948F5C89C00E9464
:108490002C8286C00F94740F83C083E50E944BB773
:1084A000882321F00E9405B791E089270E94BAE550
:1084B00077C083E50E944BB7882309F471C00E94FE
:1084C00005B7809384046CC00E94FC5A69C00E9466
:1084D000C35966C00E94425963C00E942A5960C0B5
:1084E0000E94CF585DC00E94C5575AC0F090150732
:1084F000FF2021F1E9E3FBE284918F010F5F1F4F21
:10850000882321F00E9440A1F801F6CF84E50E9463
:1085100040A16F2D70E080E090E04AE00E9499A1B8
:1085200080E20E9440A103EF12E0F80181918F01E7
:10853000882309F441C90E9440A1F7CF10924E044C
:10854000E9E3FBE284918F010F5F1F4F882321F045
:108550000E9440A1F801F6CF60E070E08FE498E05F
:108560000E94F6638AE00E9440A11AC0E9E3FBE2A0
:1085700084918F010F5F1F4F882321F00E9440A13B
:10858000F801F6CF609118077091190781E698E01D
:108590000E940F6482E20E9440A18AE00E9440A1F2
:1085A000CC55DF4FF881C45AD040FF2309F45BC596
:1085B0000F94EA0658C50E9486B78091000288236E
:1085C00021F085EE96E00E94327D0E946D638091DD
:1085D000E00883FD86C0C090F106D090F206E090DE
:1085E000F306F090F4062091FF0E3091000F4091B9
:1085F000010F5091020FC701B6010F94742C88230C
:1086000009F46FC00E94647E882301F1C092FF0EBE
:10861000D092000FE092010FF092020FE9E3FBE22B
:1086200084918F010F5F1F4F882321F00E9440A18A
:10863000F801F6CFE6E2F2E084918F010F5F1F4F61
:10864000882321F00E9440A1F801F6CFC090F106E6
:10865000D090F206E090F306F090F4062091FF0E21
:108660003091000F4091010F5091020FC701B601E8
:108670000F94DD309F77E0914E04A4E0EA9FF00173
:108680001124E95CFD4F20813181428153810F9497
:10869000D92C20E030E048E453E40F94043318165A
:1086A00004F5C092FF0ED092000FE092010FF092FD
:1086B000020FE9E3FBE284918F010F5F1F4F8823D4
:1086C00021F00E9440A1F801F6CFE7E0F2E08491AA
:1086D0008F010F5F1F4F882321F00E9440A1F801F6
:1086E000F6CF6091010270910202072E000C880BF8
:1086F000990B0F947A2C2091A3023091A4024091FF
:10870000A5025091A6020F94D92C2AE037ED43E23E
:108710005CE30F94D92C0E9419B20E949FB840CFFD
:1087200080E00E9490B60E94C3B085E40E947AB7B0
:10873000882319F00E9405B703C085E40E944BB757
:1087400021E0482FBE016F5F7F4FCE0180960F94CE
:108750003C256B017C019B01AC010F948A33811194
:1087600031C02CEA35EC47E257E368A179A18AA130
:108770009BA10F94DE30AB01BC018AEE93E00E9416
:1087800095632CEA35EC47E257E369817A818B8166
:108790009C810F94DE30AB01BC0185EE93E00E941A
:1087A00095632CEA35EC47E257E3C701B6010F9415
:1087B000DE30AB01BC0180EE93E00E9495638AE05D
:1087C0000E9440A10E94A9B00E9441D5E9CE0E941A
:1087D000E4B6AB01BC014093F8175093F9176093CE
:1087E000FA177093FB1787E497E10F94ED07D8CE43
:1087F0000E9414B70F9422326739710514F066E9AC
:1088000070E07093A9116093A8110E94F695609191
:10881000A8117091A911072E000C880B990B0F94C9
:108820007A2C2091A4113091A5114091A61150915C
:10883000A7110F94742C87FF04C060E082E994E0D4
:1088400003C060E085E894E00E9472AA81E0809312
:108850002D0280914E048093A3112B961CAE1DAE69
:108860001EAE1FAE2B9763961CAE1DAE1EAE1FAE86
:10887000639724961FAE249764961FAE6497FCE31B
:108880006896FFAF68972CE16C962FAF6C9736E433
:10889000A0963FAFA097C12CD12C70E8E72EEFEB4C
:1088A000FE2E812C912C54016091A8117091A91178
:1088B000072E000C880B990B0F947A2C162F072F7C
:1088C000782E692E262F372F482F592FB601C70132
:1088D0000F94742C882331F12091A4113091A511AB
:1088E0004091A6115091A711612F702F872D962DC1
:1088F0000F94742C881F8827881F24968FAF249785
:108900002C964FAD2C97442389F0882379F08091E1
:108910002D02882309F444CE60E087E794E00E94AA
:1089200072AA3ECE1C2D0D2D7E2C6F2C0E94DB508A
:108930006B017C01DC01CB0163962CAD3DAD4EADEE
:108940005FAD6397821B930BA40BB50BB7FD3DC0C6
:10895000D701C60188519C4FAF4FBF4F63968CAF74
:108960009DAFAEAFBFAF63970F94F10EE1E8F4E0B7
:1089700084912F019FEF491A590A882321F00E9400
:1089800040A1F201F5CF81149104A104B104B9F022
:10899000D501C40188519C4FAF4FBF4FBC01CD01E1
:1089A0006C197D098E099F0928EE33E040E050E004
:1089B0000F948030CA01B9010E94FFA103C08FE368
:1089C0000E9440A18AE00E9440A180E00F946104CF
:1089D0000E946D632090A4113090A5114090A611C3
:1089E0005090A7119101A201612F702F872D962D14
:1089F0000F94DD309F7720E030E040EA50E48114AE
:108A00009104A104B10429F40F94742C87FF07C0CA
:108A100004C00F940433181614F446015701249629
:108A2000AFAD2497AA2309F443C02B962CAD3DADDE
:108A30004EAD5FAD2B97211531054105510541F034
:108A4000D701C601821B930BA40BB50BB7FD30C039
:108A50009101A20164966FAD649768967FAD6897A7
:108A60006C968FAD6C97A0969FADA0970F94DD305C
:108A700020E030E040EC5FE30F94742C87FD47CF9B
:108A8000D701C601805A9541AF4FBF4F2B968CAF8F
:108A90009DAFAEAFBFAF2B9764962FAE649768962D
:108AA0003FAE68976C964FAE6C97A0965FAEA0975E
:108AB00080912D02882309F42ACF81149104A10406
:108AC000B10429F4C12ED02EE72CF62CEDCE98EE71
:108AD000C91A93E0D90AE108F108C818D908EA08C8
:108AE000FB08F7FE14CFEECF0E9435DB88E50E942D
:108AF0004BB7882319F0179A10926F0489E50E94EA
:108B00004BB7882319F0169A109270048AE50E94D8
:108B10004BB7882319F0159A1092710485E40E94CE
:108B20004BB7882309F43CCD0F94D40339CD0E9470
:108B300014B720E030E040E050EC0F94742C87FD37
:108B400015C00E9414B720E030E040E050E40F94DC
:108B5000043318162CF00E9414B76B017C010BC073
:108B6000C12CD12CE12C00E4F02E05C0C12CD12C5D
:108B7000E12C10ECF12E20910B0F30910C0F409155
:108B80000D0F50910E0FC701B6010F94D92C0F9401
:108B9000223220917104222351F020916A073091F2
:108BA0006B07620F731F70936B0760936A0780E512
:108BB0000E944BB7882329F00E9405B7882309F447
:108BC000EFCCA70196016091DF0E7091E00E8091CD
:108BD000E10E9091E20E0F94DE306093DF0E709301
:108BE000E00E8093E10E9093E20EE9E3FBE28491C4
:108BF0008F010F5F1F4F882321F00E9440A1F801D1
:108C0000F6CF4091DF0E5091E00E6091E10E709131
:108C1000E20E8FE695E00E94B2638AE00E9440A1D6
:108C2000BFCCA1964EAD5FADA197452B09F449C1CC
:108C3000C757DF4F488059806A807B80C958D04031
:108C4000480E591E6A1E7B1EC757DF4F2881398187
:108C50004A815B81C958D040281B390B4A0B5B0BFA
:108C6000CA01B9012F962CAD3DAD4EAD5FAD2F972A
:108C70000F947130A30192010F94A230820E931EC3
:108C8000A41EB51E34E183169104A104B1040CF1B5
:108C90004CEE84169104A104B1043CF450E885160E
:108CA0009104A104B10434F424C05BEE852E912C10
:108CB000A12CB12C8EEF90E0A0E0B0E088199909CA
:108CC000AA09BB092F968CAF9DAFAEAFBFAF2F9750
:108CD00016C044E1842E912CA12CB12C24E130E06B
:108CE00040E050E02F962CAF3DAF4EAF5FAF2F97D7
:108CF00006C02F968CAE9DAEAEAEBFAE2F97B5011F
:108D0000A4018BE197E00E94CF632F964CAD5DAD3F
:108D10006EAD7FAD2F9786E197E00E94CF63E4961A
:108D20004FADE497E8965FADE897AC966FADAC9722
:108D3000E0967FADE0978FE097E00E94B263EC96FB
:108D40004FADEC97ED965FADED97EE966FADEE976C
:108D5000EF967FADEF9788E097E00E94B263A1960F
:108D60004EAD5FADA197433051050CF4AAC02F96CC
:108D70006CAD7DAD8EAD9FAD2F970F947A2C20E01A
:108D800030E040E850E40F94D92C6B017C01E4966C
:108D90002FADE497E8963FADE897AC964FADAC9712
:108DA000E0965FADE097EC966FADEC97ED967FADFA
:108DB000ED97EE968FADEE97EF969FADEF970F94F0
:108DC000DD302BED3FE049E450E40F94D92C20E056
:108DD00030E040E05FE30F94D92C9B01AC01C70168
:108DE000B6010F94BA316B017C01C301B2010F943B
:108DF0007A2C2FE632E143E85AE30F94D92C2B0169
:108E00003C01B701A60182E097E00E94B263B30182
:108E1000A2018CEF96E00E94B2632AE939E949E1A8
:108E20005FE3C701B6010F94D92C6B017C019B0154
:108E3000AC010F94DE30A30192010F94BA31A796D2
:108E40006CAF7DAF8EAF9FAFA797A3019201C70113
:108E5000B6010F94D92C20E030E040E05EE30F949F
:108E6000D92CAB966CAF7DAF8EAF9FAFAB97ECEECE
:108E7000F6E084913F015FEF651A750A882321F0BF
:108E80000E9440A1F301F5CFB701A60186EE96E05E
:108E90000E94B263A7964CAD5DAD6EAD7FADA79756
:108EA00080EE96E00E94B263AB964CAD5DAD6EADC8
:108EB0007FADAB978AED96E00E94B2638AE00E9494
:108EC00040A12F968CAD9DADAEADBFAD2F97880D57
:108ED000991DAA1DBB1D2496EFAD2497B595A795A6
:108EE00097958795E7FF03C08093A21107C0CE55E1
:108EF000DF4FE881F981C25AD0408083A1962EAD20
:108F00003FADA1972F5F3F4FA1963FAF2EAFA197E7
:108F100060963FAD6097E4963FAFE49764964FAD9F
:108F20006497E8964FAFE89768965FAD6897AC9600
:108F30005FAFAC976C968FAD6C97E0968FAFE09774
:108F40002B964CAC5DAC6EAC7FAC2B9791E0CD57C3
:108F5000DF4F9883C358D0400C94433F40914E1844
:108F600050914F18609150187091511882E398E019
:108F70000E94B2638AE00E9440A18AE00E9440A160
:108F800020E030E0A9016091C4087091C50880918B
:108F9000C6089091C7080F94043318160CF056C0F9
:108FA00020E030E0A9016091C8087091C908809163
:108FB000CA089091CB080F94043318160CF046C0E1
:108FC000E0EFF7E084918F010F5F1F4F882321F0BE
:108FD0000E9440A1F801F6CF4091C4085091C50805
:108FE0006091C6087091C70886ED97E00E94B26351
:108FF0008AE00E9440A1409131025091320260917A
:109000003302709134028CEB97E00E94B2638AE0E5
:109010000E9440A14091C8085091C9086091CA08B7
:109020007091CB0882EA97E00E94B2638AE00E94C6
:1090300040A1EDE6F7E084918F010F5F1F4F882379
:1090400009F4AECA0E9440A1F801F5CFE0E1F8E0D2
:1090500084918F010F5F1F4F882309F4BDCF0E94B9
:1090600040A1F801F5CFCB55DF4F28813981C55A92
:10907000D0400FB6F8943EBF0FBE2DBFC455DF4F92
:109080000FB6F894DEBF0FBECDBFDF91CF911F9119
:109090000F91FF90EF90DF90CF90BF90AF909F9097
:1090A0008F907F906F905F904F903F902F9008959A
:1090B000CF92DF92EF92FF920F931F93CF93DF93A4
:1090C0006C017A018B01C0E0D0E0CE15DF0589F09C
:1090D000D8016D918D01D601ED91FC910190F08147
:1090E000E02DC6011995892B11F47E0102C021964D
:1090F000ECCFC701DF91CF911F910F91FF90EF90BF
:10910000DF90CF900895089580E090E0089580E08A
:1091100008950B96FC01849108950A96FC018491B0
:109120000895FC0184910895FCDF882321F08230AA
:1091300011F083E0089586E00895FC01E60FF11D2B
:10914000849190E0982F88273196E4918E0F911D9D
:10915000089568E0F2CF66E0F0CF0895FC01A681A3
:10916000B7818281481B8581483018F0A80FB11D56
:109170004770382F369536953695562F577080E8BC
:1091800090E002C0959587955A95E2F7439F402D50
:109190001124669566956695E62FF0E0E40FF11DC3
:1091A000EA0FFB1F3081222311F0832B02C0809530
:1091B000832380830895FB014181DC0112962C9169
:1091C0001297421760F013962C911397241738F0DA
:1091D000608115962C91621710F42481BFCF0895F9
:1091E000FC0180819281980F92832181921760F413
:1091F00094819F5F94839381890F821710F08FEF82
:10920000820F838381E0089580E00895FC0112823B
:109210008081815083831482089581E008950895A8
:1092200090E0FC013197E231F10508F04EC088274B
:10923000EE58FF4F8F4F0D94D933809180008F7778
:1092400003C0809180008F7D80938000089580917D
:109250008000877FF9CF84B58F7702C084B58F7D7A
:1092600084BD08958091B0008F7703C08091B000D5
:109270008F7D8093B0000895809190008F7707C014
:10928000809190008F7D03C080919000877F8093B4
:10929000900008958091A0008F7707C08091A00072
:1092A0008F7D03C08091A000877F8093A0000895E8
:1092B000809120018F7707C0809120018F7D03C0AE
:1092C00080912001877F8093200108953FB7F89413
:1092D0008091590490915A04A0915B04B0915C0470
:1092E00026B5A89B05C02F3F19F00196A11DB11D01
:1092F0003FBFBA2FA92F982F8827820F911DA11D3C
:10930000B11DBC01CD0142E0660F771F881F991F78
:109310004A95D1F70895CF93DF93EBEEF8E084916F
:10932000EF012196882321F00E9440A1FE01F7CF92
:10933000E3EEF8E08491EF012196882321F00E946A
:1093400040A1FE01F7CF8091060182FF03C0C4E473
:10935000D3E002C0C9E4D3E08991882319F00E94C8
:1093600040A1FACF8AE00E9440A1EBEDF8E08491A1
:10937000EF012196882321F00E9440A1FE01F7CF42
:109380008091060187FF03C0C4E4D3E002C0C9E4B2
:10939000D3E08991882319F00E9440A1FACF8AE096
:1093A0000E9440A1E3EDF8E08491EF01219688232B
:1093B00021F00E9440A1FE01F7CF1C9B03C0C4E432
:1093C000D3E002C0C9E4D3E08991882319F00E9458
:1093D00040A1FACF8AE00E9440A1EBECF8E0849132
:1093E000EF012196882321F00E9440A1FE01F7CFD2
:1093F0008091000184FD03C0C4E4D3E002C0C9E44D
:10940000D3E08991882319F00E9440A1FACF8AE025
:10941000DF91CF910C9440A1FC0127A1222349F0B8
:10942000658D768D6F5F7F4F40E150E00D960D9416
:1094300042300895CF93DF93EC0181E08FA3FE01CA
:109440003D9680E1DF011D928A95E9F7CE01E4DFC8
:1094500066E18D8D9E8DDF91CF910D9463304F929B
:109460005F926F927F92AF92BF92CF92DF92EF9214
:10947000FF92CF93DF93EB01FC01608171818281C8
:1094800093812CE3C22ED12CE12CF12CA701960163
:109490000F948030B62EA72ECA01B901A7019601FC
:1094A0000F9480306B017C01CA01B90128E130E0E2
:1094B00040E050E00F9480302B013C01C9016DE683
:1094C00071E00F94B23361157105D9F0AF92BF927C
:1094D000DF92CF925F924F929F938F937F936F9380
:1094E00087EB98E09F938F93DF93CF930F940D2C8E
:1094F0008DB79EB70E960FB6F8949EBF0FBE8DBF68
:1095000061C00097C9F0AF92BF92DF92CF925F9295
:109510004F929F938F9387EA98E09F938F93DF9367
:10952000CF930F940D2CEDB7FEB73C960FB6F89481
:10953000FEBF0FBEEDBF46C041145104610471046B
:10954000B9F0AF92BF92DF92CF925F924F928BE9C8
:1095500098E09F938F93DF93CF930F940D2C8DB74B
:109560009EB70A960FB6F8949EBF0FBE8DBF2AC055
:10957000C114D104E104F104A9F0AF92BF92DF92CB
:10958000CF9283E998E09F938F93DF93CF930F94CB
:109590000D2CEDB7FEB738960FB6F894FEBF0FBE90
:1095A000EDBF10C0AF92BF928FE898E09F938F936A
:1095B000DF93CF930F940D2C0F900F900F900F907F
:1095C0000F900F90DF91CF91FF90EF90DF90CF90B1
:1095D000BF90AF907F906F905F904F900895CF9223
:1095E000DF92FF920F931F93CF93DF931F921F92EF
:1095F000CDB7DEB76901DB0112960D911C9113976F
:10960000423309F470C0B8F4453109F477C04731EA
:1096100009F487C0443109F09DC0D80115962C91FA
:1096200015971696ED91FC911797CF01820F911D1A
:10963000820F911D5CC0463409F483C0473409F49D
:1096400084C04B3309F086C0F90181819381913048
:1096500029F0933031F4482F885004C048E0480F77
:1096600001C0482F21E0D80113963C91381708F427
:1096700020E031E0F8015281451708F430E051E074
:10968000481708F050E0822F852B382319F4252342
:1096900009F460C0D6011296FC90913051F030F080
:1096A000923049F0933051F42FEF09C020E031E0BF
:1096B00007C021E004C020E03FEF02C020E030E01E
:1096C000F7FE07C0B601C8012A83398374DD3981EA
:1096D0002A81F6018081830F80838181820F8183BB
:1096E000FF0C71F737C0B901C80165DD33C01192B5
:1096F000E817F907E1F7C80189DD2CC0C80170DD62
:10970000882349F1F80125810680F781E02DCF01FA
:10971000820F911D820F911D1192E817F907E1F751
:1097200019C0D9011C92F801828111968C9311976E
:109730008581815012968C931297838113968C9316
:1097400009C0D80115968C9103C0D80111968C914F
:10975000F601808381E00F900F90DF91CF911F91F0
:109760000F91FF90DF90CF90089588E290E00197ED
:10977000F1F708952EE93FE0009729F0F9013197BC
:10978000F1F70197F9CF08950F93FC010150040FF1
:1097900084A996A9941718F0081728F402C008178E
:1097A00050F0041740F42150260F83A995A996176D
:1097B00020F4281720F480E007C0281720F481E067
:1097C000261710F0F8CF81E00F910895DB01ED919D
:1097D000FC9119942F923F925F926F927F928F9299
:1097E0009F92AF92BF92CF92DF92EF92FF920F9330
:1097F0001F93CF93DF931F92CDB7DEB71C01C62E08
:10980000142FD22EDC011496ED90FC901597C70111
:1098100088DC082FF1018481958186DC982E013047
:1098200019F48FE0A82E02C0AA24AA94D10114969C
:109830008D919C91159771DC082FF10184819581A0
:1098400068DCB82ED10114968D919C91159781DC1E
:10985000B0E6BD1530F4009721F0E80EF91E01E6E0
:1098600010C0F1018481958176DCF0E4FD1530F4BF
:10987000009721F0E80EF91E01E403C021E1E20E99
:10988000F11CBD1480F4D10150961C925097539650
:109890001C92539754961C92549751961C92519730
:1098A00052961C92C3C0B01670F3892D90E0F70158
:1098B00024912F3F21F4FFEFEF1AFF0A59C00D1139
:1098C0004EC0D10114968D919C9115972ADC970179
:1098D0002F5F3F4FF701882311F08230E1F484912C
:1098E000D10153968C935397F901249154962C935C
:1098F0005497F7013396E4915096EC935097F70103
:109900003496E4915196EC935197F7013596E49192
:109910005296EC9320C08491982F9F709250D10161
:1099200052969C93529782958F7051968C93519733
:10993000F9012491822F8F7054968C93549722951D
:109940002F7053962C935397F7013296E491E2953A
:10995000EF705096EC93E114F10479F467C0F701CD
:109960003296E491EA219C012E0F311DE20EF31E86
:109970000B1509F488CF0F5F9ACFF101848195818F
:10998000D3DBB82ED10153969C9053975496DC901C
:10999000549751968C915197C80E52969C919D0D5B
:1099A000512E591A0D2D292D452D6C2DC101ECDE9E
:1099B0008823C9F1C7018B0D911D5C0187E0890DDA
:1099C000F82EF694F694F694D50C41019CE1890E9C
:1099D000911C6F2C712C5D1431F15C2D8501802F51
:1099E0008A198F15E0F4F8018491D10112966D91D6
:1099F0007C9113975C965C935C975D965C925D9707
:109A00005F961C925F975E968C9394014BE3C10125
:109A10005983DCDE0F5F1F4F5981585FE0CFA60CE2
:109A2000B71C5394D8CFF101808901C080E00F901A
:109A3000DF91CF911F910F91FF90EF90DF90CF902A
:109A4000BF90AF909F908F907F906F905F903F906E
:109A50002F900895EF92FF920F931F93CF93DF9370
:109A60001F92CDB7DEB78C01DC011296ED90FC9011
:109A70001397D196ED91FC91D29782E0199520E051
:109A800030E04AE0B701C801A1DEF82ED801D19636
:109A9000ED91FC91D29783E01995D801D196ED9183
:109AA000FC91D29780E01995FF2081F1F801628145
:109AB00073819E012F5F3F4F46E4C80187DE898195
:109AC000D8018C9312966D917C9113979E012F5F14
:109AD0003F4F47E4C8017ADE8981F80181836281C2
:109AE000738120E030E048E4C80170DED8011B96A5
:109AF0008C931B9798012D5C3F4F12966D917C9132
:109B0000139747E1C80162DE81E001C080E00F9059
:109B1000DF91CF911F910F91FF90EF9008951F92C9
:109B20000F920FB60F9211240BB60F922F933F9303
:109B30004F935F936F937F938F939F93AF93BF9355
:109B4000EF93FF93E0911102F09112021995FF91AA
:109B5000EF91BF91AF919F918F917F916F915F91A5
:109B60004F913F912F910F900BBE0F900FBE0F9012
:109B70001F9018951F920F920FB60F9211240BB6DB
:109B80000F922F933F934F935F936F937F938F9396
:109B90009F93AF93BF93EF93FF93E0910F02F091E8
:109BA00010021995FF91EF91BF91AF919F918F9105
:109BB0007F916F915F914F913F912F910F900BBECD
:109BC0000F900FBE0F901F9018951F920F920FB617
:109BD0000F9211240BB60F922F933F934F935F93E5
:109BE0006F937F938F939F93AF93BF93EF93FF9365
:109BF000E0910502F09106021995FF91EF91BF9156
:109C0000AF919F918F917F916F915F914F913F9114
:109C10002F910F900BBE0F900FBE0F901F901895B5
:109C20001F920F920FB60F9211240BB60F922F9323
:109C30003F934F935F936F937F938F939F93AF93D4
:109C4000BF93EF93FF93E0910302F0910402199503
:109C5000FF91EF91BF91AF919F918F917F916F9104
:109C60005F914F913F912F910F900BBE0F900FBEC0
:109C70000F901F9018951F920F920FB60F921124FC
:109C80000BB60F922F933F934F935F936F937F93F6
:109C90008F939F93AF93BF93EF93FF93E0910D0248
:109CA000F0910E021995FF91EF91BF91AF919F91A5
:109CB0008F917F916F915F914F913F912F910F9075
:109CC0000BBE0F900FBE0F901F9018951F920F9212
:109CD0000FB60F9211240BB60F922F933F934F9311
:109CE0005F936F937F938F939F93AF93BF93EF9304
:109CF000FF93E0910B02F0910C021995FF91EF9107
:109D0000BF91AF919F918F917F916F915F914F9193
:109D10003F912F910F900BBE0F900FBE0F901F9091
:109D200018951F920F920FB60F9211240BB60F9237
:109D30002F933F934F935F936F937F938F939F9353
:109D4000AF93BF93EF93FF93E0910902F0910A0262
:109D50001995FF91EF91BF91AF919F918F917F9155
:109D60006F915F914F913F912F910F900BBE0F908C
:109D70000FBE0F901F9018951F920F920FB60F9263
:109D800011240BB60F922F933F934F935F936F93D2
:109D90007F938F939F93AF93BF93EF93FF93E09144
:109DA0000702F09108021995FF91EF91BF91AF91D1
:109DB0009F918F917F916F915F914F913F912F91E3
:109DC0000F900BBE0F900FBE0F901F901895CF9362
:109DD000DF93282F30E0F901E351FE4A8491F90125
:109DE000E35DFE4AD491F901E951FF4AC491CC23C5
:109DF00089F0811115DAEC2FF0E0EE0FFF1FEC581F
:109E0000F74FA591B491EC91ED2381E090E021F41E
:109E100080E002C080E090E0DF91CF9108951F9331
:109E2000CF93DF93282F30E0F901E351FE4A84916C
:109E3000F901E35DFE4AD491F901E951FF4AC49169
:109E4000CC23C1F0162F8111EBD9EC2FF0E0EE0FEF
:109E5000FF1FED54FF4AA591B4918FB7F8941111EB
:109E600005C09C91ED2FE095E92302C0EC91ED2B0C
:109E7000EC938FBFDF91CF911F9108951F920F92A6
:109E80000FB60F9211240BB60F922F933F934F935F
:109E90005F936F937F938F939F93AF93BF93EF9352
:109EA000FF938091600490916104A0916204B0914D
:109EB0006304892B8A2B8B2B59F180915F04E091ED
:109EC0005D04F0915E049081892780838091600415
:109ED00090916104A0916204B09163041816190670
:109EE0001A061B060CF055C0809160049091610425
:109EF000A0916204B09163040197A109B109809314
:109F0000600490936104A0936204B093630441C021
:109F100080911302EEE8F8E0E4919FEF9093130232
:109F2000E230C9F050F4EE2399F0E13081F59091E0
:109F30006F009D7F90936F002AC0E43019F1E0F02C
:109F4000E53029F5909173009D7F909373001FC0B9
:109F500010926E001CC0909170009D7F90937000D5
:109F600091E09093B0009091B100987F94609093AD
:109F7000B1001092B3000BC0909171009D7F90933F
:109F8000710005C0909172009D7F9093720060E017
:109F900046DFFF91EF91BF91AF919F918F917F919C
:109FA0006F915F914F913F912F910F900BBE0F904A
:109FB0000FBE0F901F9018951F93CF93DF93182F0C
:109FC000EB010F94761B209711F460E004C0CF3FA3
:109FD000D10531F461E0812FDF91CF911F911FCF27
:109FE000E12FF0E0E351FE4AE4914E2F50E0FA01F8
:109FF0003197E231F10508F09DC08827EC57FF4FFB
:10A000008F4F0D94D93384B5806884BDC7BD97C088
:10A0100084B5806284BDC8BD92C080918000806894
:10A0200080938000D0938900C093880088C080917D
:10A030008000806280938000D0938B00C0938A0060
:10A040007EC080918000886080938000D0938D00D6
:10A05000C0938C0074C08091B00080688093B00081
:10A06000C093B3006CC08091B00080628093B00058
:10A07000C093B40064C08091900080688093900089
:10A08000D0939900C09398005AC08091900080624C
:10A0900080939000D0939B00C0939A0050C0809111
:10A0A0009000886080939000D0939D00C0939C00A6
:10A0B00046C08091A00080688093A0008091A0009D
:10A0C0008F7B8093A000D093A900C093A80037C0D5
:10A0D0008091A00080628093A000D093AB00C093D9
:10A0E000AA002DC08091A00088608093A000D0932A
:10A0F000AD00C093AC0023C08091200180688093A4
:10A100002001D0932901C093280119C0809120011A
:10A11000806280932001D0932B01C0932A010FC04D
:10A1200080912001886080932001D0932D01C093FD
:10A130002C0105C0C038D1050CF04CCF46CFDF91C3
:10A14000CF911F9108958F929F92AF92BF92CF921D
:10A15000DF92EF92FF926B017C01B8D84B015C015A
:10A16000C114D104E104F104E9F0B0D8DC01CB0161
:10A1700088199909AA09BB09883E9340A105B10530
:10A1800078F321E0C21AD108E108F10888EE880EC0
:10A1900083E0981EA11CB11CC114D104E104F10498
:10A1A00021F7DECFFF90EF90DF90CF90BF90AF9080
:10A1B0009F908F9008952FB7F894609155047091F7
:10A1C000560480915704909158042FBF08950F931F
:10A1D0001F93CF93DF93EC018881813011F4EBDF83
:10A1E00004C069857A858B859C850D811E812F81B0
:10A1F0003885601B710B820B930B28EE33E040E037
:10A2000050E00F94803089819A81AB81BC81BC0180
:10A21000CD01620F731F841F951FDF91CF911F9196
:10A220000F910895CF93DF93FC012081213051F4E9
:10A23000EC0182E08083BFDF69877A878B879C8708
:10A2400081E001C080E0DF91CF9108951F920F92CD
:10A250000FB60F9211242F933F938F939F93AF9339
:10A26000BF938091550490915604A0915704B091EA
:10A2700058043091540423E0230F2D3720F4019625
:10A28000A11DB11D05C026E8230F0296A11DB11D19
:10A29000209354048093550490935604A09357043C
:10A2A000B09358048091590490915A04A0915B0492
:10A2B000B0915C040196A11DB11D80935904909347
:10A2C0005A04A0935B04B0935C04BF91AF919F913B
:10A2D0008F913F912F910F900FBE0F901F90189567
:10A2E0000F931F93462F50E060E070E022E0440F90
:10A2F000551F661F771F2A95D1F74470552766278B
:10A300007727FC0103851485258536850B7F402B37
:10A31000512B622B732B4387548765877687AC015B
:10A32000455F5F4F60E81F910F910D94D91DCF924B
:10A33000DF92EF92FF920F931F93AC014D5A5F4F44
:10A34000062F10E020E030E09801112700270027B9
:10A3500011272F773327FA01C080D180E280F38064
:10A36000F0E8EF220C291D292E293F29FA0100834C
:10A370001183228333836DEE1F910F91FF90EF9035
:10A38000DF90CF900D94D91DCF93DF931F92CDB75F
:10A39000DEB7789484B5826084BD84B5816084BD65
:10A3A00085B5826085BD85B5816085BD80916E0073
:10A3B000816080936E0010928100809181008260A4
:10A3C00080938100809181008160809381008091E1
:10A3D00080008160809380008091B10084608093D0
:10A3E000B1008091B00081608093B00080919100B5
:10A3F00082608093910080919100816080939100B0
:10A40000809190008160809390008091A100826093
:10A410008093A1008091A10081608093A100809130
:10A42000A00081608093A0008091210182608093D0
:10A43000210180912101816080932101809120017F
:10A4400081608093200180917A00846080937A00FB
:10A4500080917A00826080937A0080917A00816096
:10A4600080937A0080917A00806880937A001092BD
:10A47000C10082E08093C0001092C50087E0809305
:10A48000C4008091C10080618093C1008091C100AF
:10A4900088608093C1008091C10080688093C10072
:10A4A0008091C1008F7D8093C10010926404E0E828
:10A4B000FAE084918F010F5F1F4F882321F00E94E3
:10A4C00040A1F801F6CFE9E3FBE284918F010F5F31
:10A4D0001F4F882321F00E9440A1F801F6CF14B746
:10A4E00010FF0DC0E7E7FAE084917F019FEFE91AC2
:10A4F000F90A882321F00E9440A1F701F5CF11FF4E
:10A500000DC0E6E6FAE084917F019FEFE91AF90AAF
:10A51000882321F00E9440A1F701F5CF12FF0DC062
:10A52000E4E5FAE084917F019FEFE91AF90A8823B4
:10A5300021F00E9440A1F701F5CF13FF0DC0E3E425
:10A54000FAE084917F019FEFE91AF90A882321F04C
:10A550000E9440A1F701F5CF15FF0CC0E2E3FAE03D
:10A5600084918F010F5F1F4F882321F00E9440A12B
:10A57000F801F6CF14BEEBE2FAE084918F010F5F91
:10A580001F4F882321F00E9440A1F801F6CF80E2FE
:10A590000E9440A1E4E2FAE084918F010F5F1F4F17
:10A5A000882321F00E9440A1F801F6CF8AE00E94A2
:10A5B00040A1E9E3FBE284918F010F5F1F4F8823E5
:10A5C00021F00E9440A1F801F6CFE4E1FAE0849185
:10A5D0008F010F5F1F4F882321F00E9440A1F801D7
:10A5E000F6CFE0E0FAE084918F010F5F1F4F8823E0
:10A5F00021F00E9440A1F801F6CFE7ECF9E0849148
:10A600008F010F5F1F4F882321F00E9440A1F801A6
:10A61000F6CFE9E3FBE284918F010F5F1F4F8823A0
:10A6200021F00E9440A1F801F6CFE0EBF9E084911F
:10A630008F010F5F1F4F882321F00E9440A1F80176
:10A64000F6CFE9E3FBE284918F010F5F1F4F882370
:10A6500021F00E9440A1F801F6CF80915E18909100
:10A660005F18BE016F5F7F4F009719F0681B790B71
:10A6700002C06456784181EA99E00E94F66360E284
:10A6800075E08AE899E00E94F6638AE00E9440A1A2
:10A6900081E080937F048093800480938104809381
:10A6A0008204809383040F942C118CE0E3E7F4E0A0
:10A6B000A3EFBEE001900D928A95E1F70E94A8B544
:10A6C0006D9A9D9A8091010180628093010188E0DA
:10A6D0000F94B3278091010188608093010186E087
:10A6E0000F94B32787ED80937A0010927E0010922A
:10A6F0007D0080917E00816080937E0080917E004D
:10A70000846080937E0080E888BD80916E008460C4
:10A7100080936E006AEF70E080E090E014DD85E0E9
:10A7200090E090936A048093690460E0809116023F
:10A73000909117020F94490E20E030E040EA50E477
:10A740000F94742C87FF0AC0809116029091170213
:10A7500040979093170280931602E7CF81E391E030
:10A76000909319028093180260E0809167049091A1
:10A7700068040F94490E20E030E848E953E40F9450
:10A780000433181654F4809167049091680440963D
:10A790009093680480936704E7CF809114029091AE
:10A7A00015020E94AA9620E030E040EA50E40F949F
:10A7B000742C87FF0AC08091140290911502409773
:10A7C0009093150280931402E8CF809165049091D4
:10A7D00066040E94AA9620E030E046E153E40F941C
:10A7E0000433181654F480916504909166044096E1
:10A7F0009093660480936504E8CF98E288E10FB6F1
:10A80000F894A895809360000FBE909360008091AB
:10A810000A01886080930A0180910A018061809317
:10A820000A0180910A01806280930A010E94DADAAB
:10A8300080912101887F816080932101E090030F46
:10A84000F090040F0091050F1091060F28E430E0FE
:10A8500040E050E060E170E088E694E10E94D79F1C
:10A86000E090070FF090080F0091090F10910A0F68
:10A8700028E430E040E050E060E170E083EF93E1F5
:10A880000E94D79FE0900B0FF0900C0F00910D0FDE
:10A8900010910E0F23E030E040E050E060E270E005
:10A8A0008EE793E10E94D79FE0900F0FF090100F7A
:10A8B0000091110F1091120F2EE130E040E050E0B6
:10A8C00060E170E089E093E10E94D79F61E088E653
:10A8D00094E10F94ED1E61E083EF93E10F94ED1E80
:10A8E00061E088E694E10F94801F61E083EF93E1DB
:10A8F0000F94801F64E088E694E10F94501F64E099
:10A9000083EF93E10F94501F60E088E694E10F9489
:10A910001D1F60E083EF93E10F941D1F61E08EE740
:10A9200093E10F94801F60E08EE793E10F94501F36
:10A9300060E08EE793E10F941D1F61E08EE793E1E5
:10A940000F94ED1E64E08EE793E1F1DC61E08EE7A9
:10A9500093E1C6DC40E050E0BA018EE793E10F944A
:10A96000BC1F60E08EE793E10F94AB1E60E08EE7C2
:10A9700093E10F947E1E61E08EE793E10F94801FB8
:10A9800060E08EE793E10F94501F60E08EE793E163
:10A990000F941D1F61E08EE793E10F94ED1E60E0C0
:10A9A00089E093E19DDC4FEF5FEF6FE070E089E0BD
:10A9B00093E10F94BC1F61E089E093E10F94AB1E1B
:10A9C00063E089E093E10F947E1E80910A0181602B
:10A9D00080930A0180910A01826080930A0180912C
:10A9E0000A01846080930A0180910A018064809347
:10A9F0000A010F9A179A0E9A169A0D9A159A0C9A9E
:10AA0000149A809107018B7F809307019FB7F89478
:10AA1000809108018460809308019FBF24982C9A3C
:10AA2000809107018F77809307019FB7F8948091F9
:10AA300008018068809308019FBF809101018F7E8B
:10AA4000809301019FB7F894809102018061809307
:10AA500002019FBF389A4098179A10926F04399A52
:10AA60004198169A109270043A9A4298159A109248
:10AA700071043B9A4398149A809180008C7F809354
:10AA8000800080918100877E886080938100809122
:10AA900080008F738093800080918100887F826026
:10AAA0008093810080E090E49093890080938800F7
:10AAB000109285001092840080916F0082608093D4
:10AAC0006F0010926E0410926D0410926C0410923C
:10AAD0006B0481E08093471878940E9444DB1092C5
:10AAE0007204809101018860809301010E9483AE0D
:10AAF0000F94B41820910C1830E0790188E3E81A1B
:10AB0000F108F7FE04C0790197E3E91AF108F5941A
:10AB1000E7942E51310936952795F22E0E94AEFB0F
:10AB200005E019E023E147E06CE08E2D0F94CF1B88
:10AB300084E00F94EF1800910C1810E002571109EF
:10AB40001695079560910D18625143E553E08F2DDE
:10AB50000F944C1C60910D18665049E553E0802F0E
:10AB60000F944C1C0F94951B8111DACF64EC79E0A3
:10AB700080E090E00E94F28A159840E6542E5DE055
:10AB8000452E6EE9C62E6AE0D62E70E0A72E70E044
:10AB9000B72E2AE0722E30E2632E80918206853035
:10ABA00010F40E9426B3809100188823E9F003DB9B
:10ABB0000091FC171091FD172091FE173091FF179F
:10ABC000DC01CB01801B910BA20BB30BB7FD0CC0BA
:10ABD0001092001880915615811112C10E9446ED05
:10ABE0008091561581110CC180918206882309F449
:10ABF00098C080915315882309F480C00091810684
:10AC0000509E800111240F551B4F61EE7AE0C80160
:10AC10000F94F32B892BF9F087E497E10E94D1A3DD
:10AC200087E497E10F944A0A109254151092531535
:10AC3000EEECFAE084918F010F5F1F4F882341F003
:10AC40000E9440A1F801F6CF80915415811156C0A1
:10AC50000F94EA0655C0F80101900020E9F73197FA
:10AC60007F01E01AF10A109247176EE470E0C80104
:10AC70000F9423344C01009729F4F7013197E00F2A
:10AC8000F11F0EC060E270E00F9423348C010F5F5F
:10AC90001F4F6AE270E0C4010F942334FC01319726
:10ACA000418272821382F80101900020E9F7319706
:10ACB000AF01401B510BB80187E497E10E9414A437
:10ACC00080914717882309F4BFCFEEE1FBE284911E
:10ACD0008F010F5F1F4F882321F00E9440A1F801D0
:10ACE000F6CFE7E8FAE084918F010F5F1F4F8823CA
:10ACF00009F4AACF0E9440A1F801F5CF0F94820772
:10AD000080918206882369F0815080938206809129
:10AD100081068F5F853018F48093810602C01092FF
:10AD200081068091DE0E882309F460C0E9E3FBE22E
:10AD300084918F010F5F1F4F882321F00E9440A153
:10AD4000F801F6CFEFEBFAE084918F010F5F1F4F10
:10AD5000882321F00E9440A1F801F6CF8091DE0EF9
:10AD600080FD51C08091DE0E84FD4DC090E2F92E31
:10AD70008091DE0E81FD64C08091DE0E85FD60C095
:10AD800000E28091DE0E82FD77C08091DE0E86FDAE
:10AD900073C010E28AE00E9440A11F926F921F923E
:10ADA0001F931F920F931F92FF92DF92CF921F92D9
:10ADB0000F94A51D1092DE0E0FB6F894DEBF0FBEE5
:10ADC000CDBF80918404882389F01092551587E4C3
:10ADD00097E10E94D1A387E497E10F944A0A109269
:10ADE000541510925315A4D60E948C9680E00F94AF
:10ADF0006104A114B10409F4D0CE0E940000C9CEB0
:10AE00000E9494ECF1CE609195047091960480912B
:10AE10009704909198040F947A2C20918504309196
:10AE2000860440918704509188040F94D92CAB017B
:10AE3000BC018BEB9AE00E94B26388E5F82E98CFB4
:10AE40006091990470919A0480919B0490919C0464
:10AE50000F947A2C2091890430918A0440918B04BC
:10AE600050918C040F94D92CAB01BC0187EB9AE074
:10AE70000E94B26309E585CF60919D0470919E04A4
:10AE800080919F049091A0040F947A2C20918D04BE
:10AE900030918E0440918F04509190040F94D92CDE
:10AEA000AB01BC0183EB9AE00E94B2631AE572CF5A
:10AEB00081E0809327021092AE1283E50E947AB758
:10AEC000882319F00E9405B703C083E50E944BB7A1
:10AED000811102C00D9458070895CF93DF93EEE1DE
:10AEE000FBE28491EF012196882321F00E9440A18A
:10AEF000FE01F7CFE4E6FBE08491EF012196882381
:10AF000021F00E9440A1FE01F7CFDF91CF9108957B
:10AF10000F931F9388E50E944BB78823E9F00E94A6
:10AF2000E4B68B01072E000C220B330B00934C0E62
:10AF300010934D0E20934E0E30934F0EDB012FEFEA
:10AF400030E00F94E13320ED37E040E050E00F9423
:10AF5000A230B9018EE230D88AE50E944BB788232F
:10AF600029F00E94E4B681E00E94908C85E40E9462
:10AF70004BB7882339F00E94E4B682E01F910F910D
:10AF80000C94908C1F910F91089588E50E944BB707
:10AF9000882329F00E94E4B688E694E1C8D96DE6DA
:10AFA00073E088E694E10E94AA8089E50E944BB78D
:10AFB000882329F00E94E4B683EF93E1B8D963E7D0
:10AFC00073E083EF93E10E94AA8085E40E944BB76F
:10AFD000882329F00E94E4B689E093E1A8D96FE7BD
:10AFE00073E089E093E10C94AA80CF92DF92EF9214
:10AFF000FF920F931F93CF93DF93CDB7DEB72897C0
:10B000000FB6F894DEBF0FBECDBF80E4E82E83E01C
:10B01000F82E8E010F5F1F4F6E0189E0C80ED11C04
:10B02000F70181917F010E947AB7882319F00E946D
:10B03000E4B602C060E070E0F801619371938F01A3
:10B04000EC15FD0569F709811A816091030F709174
:10B05000040F8091050F9091060F0115110571F0F5
:10B060000F942732980140E050E07B018C016DE69F
:10B0700073E088E694E10E94338109C00F9427327F
:10B08000AB016DE673E088E694E10E94E5800B81F8
:10B090001C816091070F7091080F8091090F9091AA
:10B0A0000A0F0115110571F00F942732980140E045
:10B0B00050E07B018C0163E773E083EF93E10E9432
:10B0C000338109C00F942732AB0163E773E083EF4C
:10B0D00093E10E94E5800D811E8160910B0F7091BC
:10B0E0000C0F80910D0F90910E0F0115110571F04D
:10B0F0000F942732980140E050E07B018C0169E712
:10B1000073E08EE793E10E94338109C00F942732E8
:10B11000AB0169E773E08EE793E10E94E5800F8160
:10B12000188560910F0F7091100F8091110F909101
:10B13000120F01151105E1F00F942732980140E03C
:10B1400050E07B018C016FE773E089E093E10E949E
:10B15000338128960FB6F894DEBF0FBECDBFDF91C6
:10B16000CF911F910F91FF90EF90DF90CF900895B6
:10B170000F942732AB016FE773E089E093E12896E3
:10B180000FB6F894DEBF0FBECDBFDF91CF911F91F8
:10B190000F91FF90EF90DF90CF900C94E5800F938C
:10B1A0001F93CF93DF9388E50E944BB7C82F89E5A3
:10B1B0000E944BB7082F8AE50E944BB7182F85E4F1
:10B1C0000E944BB7D82FC11108C0011118C011112E
:10B1D00022C0811138C0C1E007C0002311F0111155
:10B1E00002C0C0E001C0C82F6DE673E088E694E1BC
:10B1F0000F94A002011104C0CC2319F101C0C0E0DA
:10B2000063E773E083EF93E10F94A002111104C090
:10B21000CC23C9F001C0C0E069E773E08EE793E199
:10B220000F94A002DD2351F06FE773E089E093E112
:10B23000DF91CF911F910F910D94A002C111F4CF16
:10B2400004C01111E9CFD111EFCFDF91CF911F9140
:10B250000F9108956DE673E088E694E10F94B902CA
:10B2600063E773E083EF93E10F94B90269E773E05A
:10B270008EE793E10F94B9026FE773E089E093E101
:10B280000D94B902CF92DF92EF92FF920F931F932A
:10B29000CF93DF93CDB7DEB728970FB6F894DEBF14
:10B2A0000FBECDBF80E4E82E83E0F82E8E010F5F45
:10B2B0001F4F6E0189E0C80ED11CF70181917F01FB
:10B2C0000E947AB7882319F00E94E4B602C060E0B9
:10B2D00070E0F801619371938F01EC15FD0569F73A
:10B2E00049815A816DE673E088E694E14115510584
:10B2F00019F00F94110302C00F94E9024B815C8195
:10B3000063E773E083EF93E14115510519F00F9462
:10B31000110302C00F94E9024D815E8169E773E079
:10B320008EE793E14115510519F00F94110302C006
:10B330000F94E9024F8158856FE773E089E093E14C
:10B340004115510581F028960FB6F894DEBF0FBE67
:10B35000CDBFDF91CF911F910F91FF90EF90DF90C4
:10B36000CF900D94110328960FB6F894DEBF0FBE50
:10B37000CDBFDF91CF911F910F91FF90EF90DF90A4
:10B38000CF900D94E9024F925F926F927F928F92CD
:10B390009F92AF92BF92CF92DF92EF92FF92CF93A4
:10B3A000DF9300D01F92CDB7DEB70E9435DB8BE470
:10B3B0000E947AB7882399F00E9414B76B017C0130
:10B3C00020E030E0A9010F94043387FD08C0C0924B
:10B3D0005C0ED0925D0EE0925E0EF0925F0E82E502
:10B3E0000E947AB7882361F00E9414B76B017C0138
:10B3F00020E030E0A9010F94742C87FF89C006C0BB
:10B40000C12CD12C20E8E22E2FEBF22E84E40E94F6
:10B410007AB7882329F00E9414B74B015C0106C05B
:10B42000812C912C90E8A92E9FEBB92E87E50E94E4
:10B430007AB7882329F00E9414B72B013C0106C07B
:10B44000412C512C80E8682E8FEB782E88E40E94E6
:10B450007AB7882339F00E9414B769837A838B8383
:10B460009C8308C080E090E0A0E8BFEB89839A83CA
:10B47000AB83BC8320E030E0A901C501B4010F9487
:10B48000043387FD45C020E030E0A901C301B201CB
:10B490000F94043387FD3CC020E030E0A9016981AE
:10B4A0007A818B819C810F94043387FD31C020E029
:10B4B00030E0A901C501B4010F94742C882391F1E7
:10B4C00020E030E040E05FE3C501B4010F94D92CE7
:10B4D0006B017C0129813A814B815C81C301B201FE
:10B4E0000F94D92C4B015C01A7019601C701B6014D
:10B4F0000F94D92C2BED3FE049E450E40F94D92C64
:10B500009B01AC01C501B4010F94BA316B017C0100
:10B5100020E030E0A901C701B6010F94043387FF92
:10B5200004C00BC0C12CD12C7601C092580ED09211
:10B53000590EE0925A0EF0925B0EE9E3FBE2849121
:10B540007F019FEFE91AF90A882321F00E9440A1A8
:10B55000F701F5CF40915C0E50915D0E60915E0E4B
:10B5600070915F0E89E59BE00E94B263E3E5FBE02A
:10B5700084917F01AFEFEA1AFA0A882321F00E9432
:10B5800040A1F701F5CFC090580ED090590EE09031
:10B590005A0EF0905B0E20E030E0A901C701B60121
:10B5A0000F94742C882331F042E0C701B6010E9449
:10B5B00019A20DC0EEE4FBE084917F01BFEFEB1A0E
:10B5C000FB0A882321F00E9440A1F701F5CF8AE011
:10B5D0000F900F900F900F90DF91CF91FF90EF9011
:10B5E000DF90CF90BF90AF909F908F907F906F90A3
:10B5F0005F904F900C9440A1FF920F931F93CF93B5
:10B60000DF93CDB7DEB76C970FB6F894DEBF0FBEF1
:10B61000CDBF80E090E0A0E2B1E489839A83AB8360
:10B62000BC8380E090E0A6E3B3E48D839E83AF8388
:10B63000B88780E090E0A0EAB1E489879A87AB8779
:10B64000BC8741E061E081E00E94FDAF882319F0F2
:10B6500081E00E949C7585E40E944BB7882319F015
:10B660000E9414B704C060E070E080E090EC6D8B45
:10B670007E8B8F8B988F8AE50E947AB7882379F02A
:10B680008AE50E947AB7882319F00E9414B703C094
:10B6900060E070E0CB0169877A878B879C8788E5BB
:10B6A0000E947AB7882379F088E50E947AB78823C8
:10B6B00019F00E9414B703C060E070E0CB01698309
:10B6C0007A838B839C8389E50E947AB7882379F0FB
:10B6D00089E50E947AB7882319F00E9414B703C045
:10B6E00060E070E0CB016D837E838F83988785E572
:10B6F0000E944BB7882319F00E9414B704C060E081
:10B7000070E088EC92EC698B7A8B8B8B9C8B8CE451
:10B710000E944BB7882319F00E9414B703C060E061
:10B7200070E0CB016D877E878F87988B82E40E94C3
:10B730007AB7882321F00E94E4B6162F01C015E0E5
:10B74000F090FB148091CC06811171C001E0212F93
:10B75000AE014F5E5F4FBE016F5F7F4FCE014596DA
:10B760000E94847E882309F462C081E0809381076F
:10B7700080918107882309F446C060E0812F0F94EF
:10B78000C624809150118823D1F10093541184ED87
:10B790009DE80E94E3FB80918107882321F081E0EE
:10B7A0000F946104F8CF1092560710925707109229
:10B7B000580710925907109250110E9441960F9409
:10B7C0006B24009354118DE79DE80E94E3FB0E94D7
:10B7D000DB50DC01CB0180529C46AB4FBF4F8093C6
:10B7E000560790935707A0935807B09359071092A4
:10B7F00050110093810761E0812F0F94C62481E0EE
:10B800000F946104B5CF80E090E0A0EAB1E4898FA5
:10B810009A8FAB8FBC8F8091CC06882341F0412F4B
:10B82000BE01675E7F4FCE010D960E947B7F81E057
:10B83000F81202C00F94D91C6C960FB6F894DEBFB4
:10B840000FBECDBFDF91CF911F910F91FF90089553
:10B85000CF92DF92EF92FF92CF93DF93E9E3FBE287
:10B860008491EF012196882321F00E9440A1FE01DE
:10B87000F7CFEFE3FBE08491EF012196882321F0DD
:10B880000E9440A1FE01F7CF8AE50E944BB78823B2
:10B8900059F10E9414B76B017C0120E030E040E0D8
:10B8A00050EC0F94043387FF03C0E8E2FBE013C0C1
:10B8B00020E030E040EA50E4C701B6010F94742C58
:10B8C00018169CF3C092DF0ED092E00EE092E10ECB
:10B8D000F092E20E09C08491EF0121968823C1F015
:10B8E0000E9440A1FE01F7CF4091DF0E5091E00E83
:10B8F0006091E10E7091E20E85E29BE033D78AE021
:10B90000DF91CF91FF90EF90DF90CF900C9440A10A
:10B91000DF91CF91FF90EF90DF90CF9008952F921D
:10B920003F924F925F926F927F928F929F92AF92CF
:10B93000BF92CF92DF92EF92FF920F931F93CF931C
:10B94000DF93CDB7DEB763970FB6F894DEBF0FBEB7
:10B95000CDBF41E061E081E00E94FDAF8111CFC029
:10B9600092EF892E92E1992E83EF9EE09A8B898B3C
:10B97000FE0131965F010BE413E11F01F3E0F00FCC
:10B98000FB8BF4016591759185919491E989FA8910
:10B99000C190D190E190F190FA8BE98BA7019601CB
:10B9A0000F94DD302B013C0120E030E040EA51EC07
:10B9B0000F94043387FD10C020E030E040EA51E4EA
:10B9C000C301B2010F94742C181634F0F1014082B7
:10B9D0005182628273820DC0F80184911816B4F707
:10B9E000F7FAF094F7F8F094F101C082D182E28284
:10B9F000F382F101C190D190E190F1901F0120E01C
:10BA000030E040EA51ECC701B6010F94043387FFE0
:10BA100003C0EEE1FBE20BC020E030E040EA51E47D
:10BA2000C701B6010F94742C18163CF5F2CF84911F
:10BA30008F010F5F1F4F882321F00E9440A1F80162
:10BA4000F6CFE7E0FBE084918F010F5F1F4F882363
:10BA500021F00E9440A1F801F6CF61E089EF9AE061
:10BA60000E9472AA0E94957788E290E0988B8F8757
:10BA700088EC90E09E878D873BC0F4E08F0E911C90
:10BA80000F5F1F4F8B8980137CCF83E7E82E84E004
:10BA9000F82E10E0F50181919191A191B1915F0192
:10BAA000F70181939193A193B1937F01812F0E941C
:10BAB0006BB21F5F133071F70E9441D560E089EED1
:10BAC0009AE00E9472AA83E992E0988B8F8704E63D
:10BAD00010E01E870D87BE01615F7F4FCE010D967E
:10BAE0000E94CCEE8AEB92E0988B8F871E870D87A1
:10BAF000BE01615F7F4FCE010D960E94CCEE639632
:10BB00000FB6F894DEBF0FBECDBFDF91CF911F916E
:10BB10000F91FF90EF90DF90CF90BF90AF909F90EC
:10BB20008F907F906F905F904F903F902F900895EF
:10BB300088E893E190934B0E80934A0E80916F00BA
:10BB40008D7F80936F000E948CB8882359F00E94EB
:10BB50008CB88823C1F3809108138F5F8F70809316
:10BB60000813F1CF1092490E1092480E80916F0089
:10BB7000826080936F008FB7F8941092F60810924D
:10BB8000F7081092F8081092F9088FBF0E9435DB71
:10BB90000F94CE0682ED9EE00E94ADD20E94287DD9
:10BBA0000C94A8B5CF93DF9300D01F92CDB7DEB72A
:10BBB00083E50E947AB7882319F00E94E4B602C098
:10BBC00064E071E07C836B8380E50E947AB7882310
:10BBD00039F00E94E4B6693883E1780730F402C096
:10BBE00068EE73E07A83698304C088E893E19A83FE
:10BBF0008983BE016D5F7F4FCE0101960E94CCEE1E
:10BC00000F900F900F900F90DF91CF910895FF92BA
:10BC10000F931F93CF93DF930DEB1EE0C0E4D3E0AF
:10BC2000FC2E84E0F80E89910E944BB7882339F0EE
:10BC30000E9414B7F80160837183828393830C5F41
:10BC40001F4FFC12F0CFDF91CF911F910F91FF900A
:10BC50000895FF920F931F93CF93DF930DEA1EE099
:10BC6000C0E4D3E0FC2E84E0F80E89910E944BB72B
:10BC7000882349F00E9414B70F942732F80160839B
:10BC80007183828393830C5F1F4FFC12EECFDF9191
:10BC9000CF911F910F91FF900C94E4E4CF9388EC27
:10BCA00090E00E9446B8811140C084E40E944BB7E6
:10BCB0008823C1F10E9414B7C1E020E030E0A9015F
:10BCC0000F94742C811101C0C0E0C093D10ECC231D
:10BCD00049F10E9414B7E091A31124E0E29FF00122
:10BCE0001124E353F14F608371838283938320E0B7
:10BCF00030E0A9016091CD0E7091CE0E8091CF0EF3
:10BD00009091D00E0F94742C81110CC080E090E0C3
:10BD1000A0E4B0E48093CD0E9093CE0EA093CF0E0E
:10BD2000B093D00ECF910C9451D4CF910895CF936E
:10BD3000DF9385E40E947AB7882319F00E9405B743
:10BD400003C085E40E944BB7882359F0E9E3FBE286
:10BD50008491EF012196882321F00E9440A1FE01E9
:10BD6000F7CF81E40E947AB7882319F00E9405B7C3
:10BD700003C081E40E944BB7882359F0E5EEFAE056
:10BD80008491EF012196882321F00E9440A1FE01B9
:10BD9000F7CFC0911307D09114078991882319F028
:10BDA0000E9440A1FACF8AE0DF91CF910C9440A18C
:10BDB0000F931F93CF938C01C62FF80181918F01B0
:10BDC000882331F0CC2321F00F948E19C150F5CF88
:10BDD000CF911F910F910895CF93DF93EC0189913B
:10BDE000882319F00F948E19FACFDF91CF9108951F
:10BDF0000F931F93CF93DF93EC010E94DB500E81D2
:10BE00001F8128853985011511052105310599F511
:10BE10002C85222309F443C03A8521502C8721E048
:10BE2000230F2A874D85241301C01A86FE0124E0C2
:10BE3000329FE00DF11D1124068517852089318977
:10BE40000A831B832C833D83DC01CB01800F911F70
:10BE5000A11DB11D8E839F83A887B9878C819D8189
:10BE6000892BE9F09FB7F894809102018460809358
:10BE700002019FBF14C0DC01CB01801B910BA20B00
:10BE8000B30BB7FD0CC09FB7F894809102018B7F74
:10BE9000809302019FBF1E821F8218861986DF9140
:10BEA000CF911F910F910895CF93DF93FC0184915F
:10BEB000EF012196882321F00F948E19FE01F7CF10
:10BEC000DF91CF9108958091A011982F93709130B8
:10BED00031F081608D7F8093A0110D9499190895A0
:10BEE000CF93DF931F92CDB7DEB79091A011292F8A
:10BEF0002370233041F0916092609093A011898368
:10BF00000F949D1989810F90DF91CF910D948E1917
:10BF1000CF93DF93C091A011C2FB992790F98917A5
:10BF2000C9F0C3FBCC27C0F9811102C090E201C067
:10BF300094E2C11102C020E001C022E0D82F822F7C
:10BF4000892BCEDF8091A011D0FB82F9C0FB83F951
:10BF50008093A011DF91CF910895CF92DF92EF925D
:10BF6000FF921F93CF93DF931F921F92CDB7DEB73F
:10BF7000182F80E069837A83CBDF812F8F738064F1
:10BF8000AFDFA1DF6981C62E7A81D72E11E1115072
:10BF900069F0F601E590F4908F2D0F948E198E2D97
:10BFA0000F948E1982E0C80ED11CF1CF0F900F9024
:10BFB000DF91CF911F91FF90EF90DF90CF90089588
:10BFC00080E0A6DF81E08CDF6FE070E080E090E051
:10BFD0000C94A3501F93CF93DF931F92CDB7DEB77E
:10BFE000182F81E0698394DF6981862F806878DF6C
:10BFF000812F8F7080680F90DF91CF911F9170CF4C
:10C00000CF92DF92EF92FF920F931F93CF93DF9324
:10C01000C42E633010F06250805F8150982F917071
:10C02000D92EC82FC6956150D62FD295D07F83E7E1
:10C03000E82E8BE0F82E01E0F7011491602F6D0FD0
:10C040008C2FC8DF40DFCC2059F0D11002C0812FE7
:10C0500001C080E00F948E19DD2029F0812F04C0EB
:10C0600080E00F948E1980E00F948E190F5FFFEF20
:10C07000EF1AFF0A053001F7DF91CF911F910F9161
:10C08000FF90EF90DF90CF900895CF92DF92FF92D4
:10C090000F931F93CF93DF93633010F06250885F4C
:10C0A000DFEFD80F6150C62FC295C07F8A01F12CF7
:10C0B0006F2D6C0F8D2F8EDF06DFF801C590D490A9
:10C0C0008D2D0F948E198C2D0F948E19F3940E5F75
:10C0D0001F4F80E1F812ECCFDF91CF911F910F91AC
:10C0E000FF90DF90CF900895CF93C82F80E010DFAE
:10C0F0008C2F8F738068CF91F3CE2F923F924F9207
:10C100005F926F927F928F929F92AF92BF92CF92E7
:10C11000DF92EF92FF920F931F93CF93DF93CDB7F0
:10C12000DEB766970FB6F894DEBF0FBECDBF898726
:10C130000F94A8192985211131C00E944BAE40915E
:10C14000A8115091A9112091AA113091AB11242767
:10C15000352790910102A90149276091D10870917A
:10C16000D2086F5F7F4F94E6969F9001979F300DA6
:10C17000112437FF02C021503F4F232F332724279C
:10C180003527282780918506909186068217930788
:10C1900009F4AAC130938606209385060E944BAE0F
:10C1A0008C878BEF94E10E94E7506D877E878F87A5
:10C1B000988B80910102909102029A8B898B209139
:10C1C000D1083091D2082F5F3F4F44E6429FC00113
:10C1D000439F900D112497FF02C081509F4F9A8773
:10C1E000292F220F220B2B879B8B6091D3087091F4
:10C1F000D4088091D5089091D6080F9422322B0153
:10C200003C012090AA113090AB116091A411709163
:10C21000A5118091A6119091A7110F9422324B0184
:10C220005C017D8B6C8BE090A811F090A91121141A
:10C23000310469F021E02414350424F4C201821988
:10C24000930903C0C1018419950903970CF420E0F8
:10C2500080911A028170821719F091E0988702C0CC
:10C260008985888781E02E8B3FDF2DDE5F924F929C
:10C270002BE8C22E2BE0D22EDF92CF928E010F5FE1
:10C280001F4F1F930F930F940D2CC801A5DD0F9026
:10C290000F900F900F900F900F902E892223A1F0F6
:10C2A00089E89BE001DE3F922F92DF92CF921F93AD
:10C2B0000F930F940D2CC8018FDD0F900F900F90EE
:10C2C0000F900F900F902E899885992331F0622F4F
:10C2D00081E02E8B0E94F8B82E8980911A0220FBF3
:10C2E00080F980931A02E114F10481F08C899D8910
:10C2F00033243394E816F90624F4C4018E199F09F7
:10C3000003C0C7018819990903970CF4312C809157
:10C310001A0282FB882780F9831519F022242394BE
:10C3200001C0298481E1E0DECEDD9F928F929BE8FF
:10C33000C92E9BE0D92EDF92CF921F930F930F94BB
:10C340000D2CC80149DD0F900F900F900F900F90AA
:10C350000F90332099F089E89BE0A6DDFF92EF92E1
:10C36000DF92CF921F930F930F940D2CC80134DDF1
:10C370000F900F900F900F900F900F90222021F0B0
:10C38000632D82E00E94F8B880911A0230FA82F997
:10C3900080931A0286E0A8DE96DD8A859B85992720
:10C3A0009F938F938BE89BE09F938F931F930F93A3
:10C3B0000F940D2CC80110DD85E20F948E1988E0D2
:10C3C00093DE8CE3882E912CA12CB12C6D857E857B
:10C3D0008F859889A50194010F948030CA01B90115
:10C3E000A50194010F9480300F900F900F900F9043
:10C3F0000F900F902436310598F47F936F933F93FD
:10C400002F938FE79BE09F938F931F930F930F942E
:10C410000D2C0FB6F894DEBF0FBECDBF85E012C065
:10C420007F936F933F932F9387E79BE09F938F9327
:10C430001F930F930F940D2C0FB6F894DEBF0FBE11
:10C44000CDBF86E0F801E80FF11D80E280833BDD7F
:10C4500066E0C801ADDC86E147DE35DD89899A8971
:10C4600099279F938F938BE89BE09F938F931F93C4
:10C470000F930F940D2CC801AFDC85E20F948E1939
:10C480000F900F900F900F900F900F909B89992312
:10C4900079F085E029DE17DD2C85211102C016E038
:10C4A00001C014E080E00F948E19812F0F948E1933
:10C4B00080E11E141F046CF417DE05DD8C858111EC
:10C4C00002C012E001C010E080E00F948E19812FAD
:10C4D00006C00ADEF8DC80E20F948E1980E20F9429
:10C4E0008E19998591110EC0ECE5F2E080E09191F2
:10C4F000992311F08927FBCF90918706981781F037
:10C500008093870688E1F0DDDEDC60E18CE592E077
:10C510004FDC0E944BAE909188069813809388065A
:10C5200080915515882351F120914A17222321F13A
:10C530008091F4179091F517A091F617B091F71725
:10C540000097A105B105B9F0BC01CD016D597F4F30
:10C550008F4F9F4F24E630E040E050E00F94803052
:10C560006091F8177091F9178091FA179091FB1765
:10C570000F94803001C020E02093E108D090E108C2
:10C580002985211105C0809189068D1509F482C085
:10C59000D09289068D2D69E10F94A63320E1929FF8
:10C5A000C001112469E170E00F94C63380E090E887
:10C5B0005C0102C0B594A7946A95E2F791E0ED2C76
:10C5C000F12C692F8CE09E8B05DD7DDC20E030E0D6
:10C5D000C12C9E89490189E1880E911CE814F90457
:10C5E00034F42E153F0534F000E010E004C00FEFE6
:10C5F0001FEF01C08501913059F09D3049F023E0D3
:10C60000C21202C0016006C0C11004C0106802C09E
:10C610000FEF1FEF812F9E8B0F948E19802F0F9499
:10C620008E19C39494019E892436310599F69F5F33
:10C630009E3039F68CE058DD46DC80E20F948E198E
:10C640008E010F5F1F4F89E08D1578F4FF92EF92F6
:10C650008FE89BE09F938F931F930F930F940D2C64
:10C66000C801BADB87E99BE00EC0FF92EF928BE82E
:10C670009BE09F938F931F930F930F940D2CC801F2
:10C68000ABDB83E99BE010DC0F900F900F900F90D5
:10C690000F900F900F94A11966960FB6F894DEBF15
:10C6A0000FBECDBFDF91CF911F910F91FF90EF9003
:10C6B000DF90CF90BF90AF909F908F907F906F90C2
:10C6C0005F904F903F902F900895AC01485F5F4F6F
:10C6D000BC016C5F7F4F0C94CBD30E94DB50609306
:10C6E0006A1170936B1180936C1190936D11089582
:10C6F000CF92DF92EF92FF92CF93DF936A017B019B
:10C70000FC018491EF012196882321F00E9440A131
:10C71000FE01F7CF4AE0C701B601DF91CF91FF904C
:10C72000EF90DF90CF900C9499A1CF92DF92EF928F
:10C73000FF92CF93DF936A017B01FC018491EF01AB
:10C740002196882321F00E9440A1FE01F7CF42E00C
:10C75000C701B601DF91CF91FF90EF90DF90CF90AE
:10C760000C9419A2CF92DF92EF92FF92CF93DF93B6
:10C770006A017B01FC018491EF012196882321F05D
:10C780000E9440A1FE01F7CF42E0C701B601DF9150
:10C79000CF91FF90EF90DF90CF900C9419A20F9360
:10C7A0001F93CF93DF9300D01F92CDB7DEB7FC016C
:10C7B00084918F010F5F1F4F882361F049835A8353
:10C7C0006B837C830E9440A1F80149815A816B816F
:10C7D0007C81EECFCB01BA010F900F900F900F909C
:10C7E000DF91CF911F910F910C94FFA10F931F9395
:10C7F000CF93DF938B01FC018491EF012196882375
:10C8000021F00E9440A1FE01F7CFB801110F880B63
:10C81000990BDF91CF911F910F910C94FFA10F9372
:10C820001F93CF93DF931F921F92CDB7DEB7FC010A
:10C8300084918F010F5F1F4F811102C08B0108C0CF
:10C8400069837A830E9440A1F80169817A81F0CFDF
:10C85000F80181918F01882319F00E9440A1F8CF3F
:10C860000F900F90DF91CF911F910F9108950F932B
:10C870001F93CF93DF93E091480EF091490E4281D0
:10C880005381648175811416150616061706FCF48B
:10C8900020911B0920FF1BC03091060120918406C6
:10C8A0003695369541E03427832F81702E7F822B79
:10C8B00080938406909183069170892341F0809142
:10C8C000DE0E81608093DE0E80E00E94EFDAE09160
:10C8D000480EF091490E86819781A085B185181682
:10C8E00019061A061B0634F580911B0981FD22C02A
:10C8F000409106018091840690E0042E000C550BB7
:10C9000040955095550F440B542F48275927407296
:10C9100055274827592740938406809183068072C3
:10C92000482341F08091DE0E80628093DE0E81E02C
:10C930000E94EFDAE091480EF091490E82859385CE
:10C94000A485B585181619061A061B060CF04DC0ED
:10C9500090911B098091840692FF25C090917204EA
:10C96000992309F442C093B1482F50E0892F829552
:10C970008F7091E08927082F017010E08827992790
:10C98000801B910B842795278470992784279527EE
:10C9900080938406209183062470822331F1809154
:10C9A000DE0E84601DC090910001282F30E092952A
:10C9B0009170C92F80E0D82F882799278C1B9D0B59
:10C9C0008227932780749927822793278093840650
:10C9D000909183069074892341F08091DE0E8064EB
:10C9E0008093DE0E82E00E94EFDA809184068093CD
:10C9F0008306DF91CF911F910F910895EF92FF92DF
:10CA00001F93CF93DF931F92CDB7DEB7182FE3EBC1
:10CA1000FBE084917F012FEFE21AF20A882331F0C4
:10CA200099830E9440A1F7019981F3CFE12FF92F5B
:10CA300084917F019FEFE91AF90A882321F00E946F
:10CA400040A1F701F5CFEAE9FBE084917F012FEFE8
:10CA5000E21AF20A882321F00E9440A1F701F5CFE3
:10CA60000F90DF91CF911F91FF90EF9008952F923B
:10CA70003F924F925F926F927F928F929F92AF926E
:10CA8000BF92CF92DF92EF92FF920F931F93CF93BB
:10CA9000DF93CDB7DEB7C251D1400FB6F894DEBFF9
:10CAA0000FBECDBF41E061E081E00E94FDAF81118A
:10CAB0000C948275FE0131968CE3DF011D928A95FC
:10CAC000E9F70091840EC453DF4F0883CC5CD0405B
:10CAD0008AE40E944BB7882321F00E94A7B60C94E9
:10CAE000827586E50E947AB7882349F00E94E4B6F1
:10CAF000C652DF4F79836883CA5DD04006C0C652F4
:10CB0000DF4F19821882CA5DD040C652DF4F0881BC
:10CB10001981CA5DD0400530110570F0EFE9FDE0E4
:10CB200084918F010F5F1F4F882311F40C9482753D
:10CB30000E9440A1F801F4CF84E40E947AB78823D0
:10CB400019F00E9405B703C084E40E944BB7C85196
:10CB5000DF4F8883C85ED040C652DF4F08811981FD
:10CB6000CA5DD040033011058CF484E50E947AB789
:10CB7000882319F00E9405B703C084E50E944BB7D3
:10CB8000CE51DF4F8883C25ED04006C011E0CE5147
:10CB9000DF4F1883C25ED04088E50E947AB78823B1
:10CBA00021F00E94E4B6162F01C012E089E50E9430
:10CBB0007AB7882321F00E94E4B6062F01C002E074
:10CBC00080E50E947AB781110BC0C752DF4F1883EE
:10CBD000C95DD040C553DF4F0883CB5CD0400CC04B
:10CBE0000E94E4B6C752DF4F6883C95DD040C55389
:10CBF000DF4F6883CB5CD040C752DF4F0881C95DEF
:10CC0000D040023018F4EAE6FDE008C0C553DF4F1B
:10CC10001881CB5CD040123068F4F5CF84918F013D
:10CC20000F5F1F4F882311F40C9482750E9440A15E
:10CC3000F801F4CF83E50E947AB7882319F00E94A7
:10CC400014B704C060E070E88BEB95E420E030E0BE
:10CC500040E752E40F94BA3160939F027093A002B0
:10CC60008093A1029093A2028CE40E947AB7882359
:10CC700081F00E9414B720915218309153184091BE
:10CC80005418509155180F94DD300F9422327B01C7
:10CC900004C05DEFE52EFF24FA9482E50E947AB786
:10CCA000882381F00E9414B72091521830915318B4
:10CCB00040915418509155180F94DD300F94223242
:10CCC0005B0103C043EAA42EB12C86E40E947AB72C
:10CCD000882381F00E9414B720915618309157187C
:10CCE00040915818509159180F94DD300F9422320A
:10CCF0008B0102C00CEF1FEF82E40E947AB78823F9
:10CD000081F00E9414B72091561830915718409125
:10CD10005818509159180F94DD300F9422326B013E
:10CD200003C038EAC32ED12C81E02DEFE2162FEF9D
:10CD3000F2063CF0950129503109E216F3060CF495
:10CD400080E021E034EAA316B1043CF4A701475F78
:10CD50005F4F4A155B050CF420E0882483940C3F58
:10CD60004FEF14073CF0A60149505109041715076D
:10CD70000CF4812C9924939459EAC516D1043CF4FF
:10CD8000A801475F5F4F4C155D050CF4912C811194
:10CD90000BC0222321F08BE59DE030DE14C0811012
:10CDA00012C0911015C01DC083E69DE0CE5EDE4F1F
:10CDB0002883C251D14022DECE5EDE4F2881C2518F
:10CDC000D1402111E8CF882019F083E59DE016DEDF
:10CDD000992011F40C9482758CE49DE00FDE0C9484
:10CDE0008275C652DF4F88819981CA5DD040892BF8
:10CDF00021F1E6E3FDE084914F019FEF891A990A42
:10CE0000882321F00E9440A1F401F5CFC851DF4FE3
:10CE1000A881C85ED040AA2369F0ECE2FDE08491CD
:10CE20004F01BFEF8B1A9B0A882321F00E9440A17B
:10CE3000F401F5CF8AE00E9440A10E9435DB80E03A
:10CE40000E9490B681E00E94C8B1882349F0C45383
:10CE5000DF4F8881CC5CD0400E9490B60C948275E4
:10CE60000E94C3B085E40E947AB7882319F00E941B
:10CE700005B703C085E40E944BB7CC51DF4F8883D0
:10CE8000C45ED040C752DF4FF881C95DD040EF2F5C
:10CE9000F0E0C751DF4FF983E883C95ED040C55346
:10CEA000DF4F3881CB5CD040232F30E0C351DF4FC0
:10CEB00039832883CD5ED040C752DF4F5881C95D8A
:10CEC000D040C553DF4F4881CB5CD040549FA00178
:10CED0001124C052DF4F59834883C05ED040C752EF
:10CEE000DF4F5881C95DD0405170CB52DF4F58831E
:10CEF000C55DD040C052DF4F88819981C05ED0406F
:10CF0000880F991FC750DF4F99838883C95FD0402E
:10CF1000CD53DF4F19821882C35CD040C452DF4F1B
:10CF2000188219821A821B82CC5DD040C554DF4F13
:10CF3000188219821A821B82CB5BD040AFEFBFEF01
:10CF4000C954DF4FB983A883C75BD04097010F2C2A
:10CF5000000C440B550BCB5FDE4F288339834A838B
:10CF60005B83C550D140A5014E195F09C75FDE4FF5
:10CF700059834883C950D140C801012E000CAA0B27
:10CF8000BB0BC55FDE4F88839983AA83BB83CB50DD
:10CF9000D140D601A01BB10BC15FDE4FB983A8837E
:10CFA000CF50D140CB52DF4F0881C55DD040002328
:10CFB00091F0C553DF4F0881CB5CD040C353DF4FA6
:10CFC0000883CD5CD04011E0CF52DF4F1883C15DA4
:10CFD000D04010E011C0C553DF4F1881CB5CD0406A
:10CFE00011500FEFCF52DF4F0883C15DD040C353C4
:10CFF000DF4F0883CD5CD04081E0CB52DF4F08810A
:10D00000C55DD0400827CB52DF4F0883C55DD040B7
:10D010002CE0C954DF4F48815981C75BD040249F21
:10D02000C001259F900D1124DC01AD5DBA4EC154A5
:10D03000DF4FB983A883CF5BD040440F551F440F07
:10D04000551FCF50DF4F59834883C15FD040C9542B
:10D05000DF4F88819981C75BD040C052DF4FE881A4
:10D06000F981C05ED0408E0F9F1F9C01220F331F9D
:10D07000220F331FCB50DF4F39832883C55FD04049
:10D08000C954DF4F88819981C75BD040C750DF4FBB
:10D0900048815981C95FD040840F951FDC01AA0FD8
:10D0A000BB1FAA0FBB1FC550DF4FB983A883CB5F3F
:10D0B000D040C953DF4F19821882C75CD040C75196
:10D0C000DF4FE881F981C95ED0403197C350DF4F0F
:10D0D000F983E883CD5FD040CD53DF4F288139817C
:10D0E000C35CD040032E000C440B550BC150DF4FE6
:10D0F000288339834A835B83CF5FD040CD53DF4F92
:10D1000048815981C35CD040440F551FCD5FDE4F2D
:10D1100059834883C350D140C353DF4F0881CD5C4E
:10D12000D040101709F4C9C2CB5FDE4F6881798106
:10D130008A819B81C550D1400F947A2C6B017C0170
:10D14000C75FDE4F88819981C950D140C350DF4FFE
:10D1500068817981CD5FD0400F94C633072E000CD3
:10D16000880B990B0F947A2C4B015C01C150DF4F57
:10D17000688179818A819B81CF5FD0400F947A2C1E
:10D180009B01AC01C501B4010F94D92C9B01AC01EA
:10D19000C701B6010F94DE306B017C01C55FDE4F25
:10D1A000688179818A819B81CB50D1400F947A2C00
:10D1B0004B015C01C15FDE4F88819981CF50D14026
:10D1C000C351DF4F68817981CD5ED04061507109D4
:10D1D0000F94C633072E000C880B990B0F947A2CF2
:10D1E0002B013C01612F012E000C770B880B990B52
:10D1F0000F947A2C9B01AC01C301B2010F94D92C7E
:10D200009B01AC01C501B4010F94DE304B015C0100
:10D2100020E030E0A901C701B6010F94742C87FD0E
:10D2200005C020E030E040E05FE303C020E030E0F4
:10D23000A901C701B6010F94DE300F945332C355D4
:10D24000DF4F688379838A839B83CD5AD04020E067
:10D2500030E0A901C501B4010F94742C87FD05C00D
:10D2600020E030E040E05FE303C020E030E0A901CF
:10D27000C501B4010F94DE300F945332C755DF4F10
:10D28000688379838A839B83C95AD040C954DF4F0E
:10D2900088819981C75BD0400196C954DF4F99833B
:10D2A0008883C75BD040CD5FDE4FE881F981C350F2
:10D2B000D140E10FF11D17FDFA95EE0FFF1FA1EA16
:10D2C000B0E0AC0FBD1FEA0FFB1F91838083C652F5
:10D2D000DF4F2881CA5DD040CC51DF4F4881C45E0A
:10D2E000D040BE0167557F4FCE0183559F4F0F94AD
:10D2F0003C25C554DF4F688379838A839B83CB5B4E
:10D30000D0409B01AC010F948A33882341F0C45371
:10D31000DF4F8881CC5CD0400E9490B6CEC1C5540E
:10D32000DF4F288139814A815B81CB5BD040C45279
:10D33000DF4F688179818A819B81CC5DD0400F94D9
:10D34000DE30C452DF4F688379838A839B83CC5D50
:10D35000D040C953DF4F88819981C75CD040CF50FE
:10D36000DF4FE881F981C15FD0408E0F9F1FEDE64E
:10D37000F0E0EC0FFD1FE80FF91FC554DF4F2881C7
:10D3800039814A815B81CB5BD040248335834683DE
:10D390005783C355DF4F288039804A805B80CD5A40
:10D3A000D040EDE3F0E0EC0FFD1FE80FF91F248201
:10D3B000358246825782C755DF4F88809980AA8080
:10D3C000BB80C95AD040C953DF4FE881F981C75C9F
:10D3D000D040CB50DF4F48815981C55FD040E40F2A
:10D3E000F51F8DE390E08C0F9D1FE80FF91F8482DD
:10D3F0009582A682B782C953DF4FE881F981C75C65
:10D40000D040C550DF4FA881B981CB5FD040EA0F33
:10D41000FB1FE80FF91F20E030E040E85FE32483C2
:10D42000358346835783A201910169817A818B817B
:10D430009C810F94DE3069837A838B839C83A50162
:10D4400094016D817E818F8198850F94DE306D838C
:10D450007E838F839887C554DF4F288139814A8125
:10D460005B81CB5BD04069857A858B859C850F94E9
:10D47000DE3069877A878B879C87A2019101C20180
:10D48000B1010F94D92C9B01AC016D857E858F85F0
:10D4900098890F94DE306D877E878F87988BA501E2
:10D4A0009401C501B4010F94D92C9B01AC01698989
:10D4B0007A898B899C890F94DE30698B7A8B8B8B70
:10D4C0009C8BC554DF4F288139814A815B81CB5BBE
:10D4D000D040CA01B9010F94D92C9B01AC016D89D0
:10D4E0007E898F89988D0F94DE306D8B7E8B8F8B2C
:10D4F000988FA5019401C201B1010F94D92C9B0111
:10D50000AC01698D7A8D8B8D9C8D0F94DE30698F87
:10D510007A8F8B8F9C8FC554DF4F288139814A8148
:10D520005B81CB5BD040C201B1010F94D92C9B0130
:10D53000AC016D8D7E8D8F8D98A10F94DE306D8F37
:10D540007E8F8F8F98A3C554DF4F288139814A8100
:10D550005B81CB5BD040C501B4010F94D92C9B01FA
:10D56000AC0169A17AA18BA19CA10F94DE3069A3C3
:10D570007AA38BA39CA372016101E894F7F86DA0D4
:10D580007EA00FA138A5C453DF4F3883CC5CD040B8
:10D590009301402FC453DF4F5881CC5CD040C7016A
:10D5A000B6010F94043318163CF06301E02EC45307
:10D5B000DF4FF880CC5CD040CDA2DEA2EFA2F8A66F
:10D5C00075016401E894F7F869A47AA40BA54CA549
:10D5D000C453DF4F4883CC5CD0409301402FC453E9
:10D5E000DF4F5881CC5CD040C701B6010F940433A3
:10D5F00018163CF06301E02EC453DF4FF880CC5C7A
:10D60000D040C9A6DAA6EBA6FCA620E030E040E8B0
:10D610005FE369AD7AAD8BAD9CAD0F94DE3069AF41
:10D620007AAF8BAF9CAFC154DF4FA881B981CF5B7C
:10D63000D0401C962D923D924D925C921F97FD0119
:10D64000808A918AA28AB38AC554DF4F28813981A2
:10D650004A815B81CB5BD04054962D933D934D9393
:10D660005C93579780E00F946104CF52DF4F08819D
:10D67000C15DD040100FC154DF4F28813981CF5B8D
:10D68000D040245F3F4FC154DF4F39832883CF5BA5
:10D69000D040C953DF4F48815981C75CD0404C5FAF
:10D6A0005F4FC953DF4F59834883C75CD040C45391
:10D6B000DF4F1882CC5CD0402FCDCD53DF4F888117
:10D6C000C35CD0408F5FC752DF4F1881C95DD04027
:10D6D0008117E8F4CD53DF4F08811981C35CD04036
:10D6E0000F5F1F4FCD53DF4F19830883C35CD040BA
:10D6F000C554DF4F288139814A815B81CB5BD040A3
:10D70000CA01B9010F948A33882309F44BCC80E015
:10D710000E94C8B1882349F0C453DF4F8881CC5C94
:10D72000D0400E9490B60C947975C554DF4F288183
:10D7300039814A815B81CB5BD040CA01B9010F942A
:10D740008A3381110C94797589AC9AACABACBCACC2
:10D7500020E030E0A901C501B4010F94742C8823A6
:10D7600009F408C2A501940169817A818B819C81A9
:10D770000F94BA31C954DF4F688379838A839B83BE
:10D78000C75BD04069837A838B839C83A501940116
:10D790006D817E818F8198850F94BA31C154DF4F9E
:10D7A000688379838A839B83CF5BD0406D837E833C
:10D7B0008F839887A501940169857A858B859C85DF
:10D7C0000F94BA31CD53DF4F688379838A839B836B
:10D7D000C35CD04069877A878B879C87A5019401B9
:10D7E0006D857E858F8598890F94BA316B017C0198
:10D7F000C954DF4F288139814A815B81C75BD040A2
:10D80000CA01B9010F94D92C9B01AC01C701B60123
:10D810000F94DD30CB52DF4F688379838A839B83FB
:10D82000C55DD0406D877E878F87988BA501940159
:10D8300069897A898B899C890F94BA316B017C0143
:10D84000C154DF4F288139814A815B81CF5BD04051
:10D85000CA01B9010F94D92C9B01AC01C701B601D3
:10D860000F94DD30C353DF4F688379838A839B83B2
:10D87000CD5CD040698B7A8B8B8B9C8BA5019401FE
:10D880006D897E898F89988D0F94BA316B017C01E7
:10D89000CD53DF4F288139814A815B81C35CD04001
:10D8A000CA01B9010F94D92C9B01AC01C701B60183
:10D8B0000F94DD306D8B7E8B8F8B988FA50194013B
:10D8C000698D7A8D8B8D9C8D0F94BA316B017C01A3
:10D8D000C154DF4F288139814A815B81CF5BD040C1
:10D8E000C954DF4F688179818A819B81C75BD040B1
:10D8F0000F94D92C9B01AC01C701B6010F94DD3008
:10D90000C953DF4F688379838A839B83C75CD04088
:10D91000698F7A8F8B8F9C8FA501940169A17AA161
:10D920008BA19CA10F94BA316B017C01CD53DF4FC9
:10D93000288139814A815B81C35CD040C154DF4F6B
:10D94000688179818A819B81CF5BD0400F94D92CEB
:10D950009B01AC01C701B6010F94DD306B017C0166
:10D9600069A37AA38BA39CA3A50194016D8D7E8DE1
:10D970008F8D98A10F94BA314B015C01CD53DF4FCD
:10D98000288139814A815B81C35CD040C954DF4F13
:10D99000688179818A819B81C75BD0400F94D92CA3
:10D9A0009B01AC01C501B4010F94DD304B015C015A
:10D9B0006D8F7E8F8F8F98A3C353DF4F288139815E
:10D9C0004A815B81CD5CD040CB52DF4F6881798149
:10D9D0008A819B81C55DD0400F94D92C2B013C01DD
:10D9E000C953DF4F288139814A815B81C75CD040B0
:10D9F000CA01B9010F94D92C9B01AC01C301B2013A
:10DA00000F94DD30CF52DF4F688379838A839B8305
:10DA1000C15DD0402B013C01E89477F829A53AA5D7
:10DA20004BA55CA56DA17EA18FA198A50F94DE30BA
:10DA30002FEF36EE4BED5EE20F94D92C9B01AC013B
:10DA4000C301B2010F94742C18160CF093C0C95383
:10DA5000DF4F288139814A815B81C75CD040C70193
:10DA6000B6010F94D92C2B013C01C353DF4F288101
:10DA700039814A815B81CD5CD040C501B4010F94EE
:10DA8000D92C9B01AC01C301B2010F94DD30CF5200
:10DA9000DF4F288139814A815B81C15DD0400F947D
:10DAA000BA312B013C016DA77EA78FA798ABC95354
:10DAB000DF4F288139814A815B81C75CD040C50135
:10DAC000B4010F94D92C4B015C01CB52DF4F28815C
:10DAD00039814A815B81C55DD040C701B6010F9491
:10DAE000D92C9B01AC01C501B4010F94DD30CF529C
:10DAF000DF4F288139814A815B81C15DD0400F941D
:10DB0000BA316B017C0169AB7AAB8BAB9CABC9546E
:10DB1000DF4F288139814A815B81C75BD040C301D7
:10DB2000B2010F94D92C9B01AC01CD53DF4F68811A
:10DB300079818A819B81C35CD0400F94DE304B0198
:10DB40005C01C154DF4F288139814A815B81CF5B01
:10DB5000D040C701B6010F94D92C9B01AC01C5017F
:10DB6000B4010F94DE30DC01CB01B0588DAB9EAB1D
:10DB7000AFABB8AF2DA53EA54FA558A9C154DF4FF7
:10DB8000288339834A835B83CF5BD0405058CD5381
:10DB9000DF4F288339834A835B83C35CD04089A9E4
:10DBA0009AA9ABA9BCA9C953DF4F88839983AA83DB
:10DBB000BB83C75CD0400DA91EA92FA938ADCB509F
:10DBC000DF4F088319832A833B83C55FD040C0524F
:10DBD000DF4F08811981C05ED040B801110F880B5A
:10DBE000990B0F947A2C9B01AC01C452DF4F6881D2
:10DBF00079818A819B81CC5DD0400F94BA31CB5220
:10DC0000DF4F688379838A839B83C55DD040C6528A
:10DC1000DF4F08811981CA5DD040012B09F46DC224
:10DC200040903715509038156090391570903A151E
:10DC3000209143153091441540914515509146155A
:10DC4000C301B2010F94DD30CC51DF4F688379837B
:10DC50008A839B83C45ED040C0903315D090341526
:10DC6000E0903515F090361520913F153091401514
:10DC70004091411550914215C701B6010F94DD3016
:10DC8000C751DF4F688379838A839B83C95ED04005
:10DC900080902F1590903015A0903115B0903215CE
:10DCA00020913B1530913C1540913D1550913E150A
:10DCB000C501B4010F94DD30C351DF4F6883798310
:10DCC0008A839B83CD5ED04020912B1530912C15FB
:10DCD00040912D1550912E15C452DF4F2883398362
:10DCE0004A835B83CC5DD040A3019201C452DF4FD5
:10DCF000688179818A819B81CC5DD0400F94DD3031
:10DD0000CF50DF4F688379838A839B83C15FD04084
:10DD10008091271590912815A0912915B0912A1569
:10DD2000C353DF4F88839983AA83BB83CD5CD040E4
:10DD3000A7019601BC01CD010F94DD306B017C0180
:10DD40000091231510912415209125153091261549
:10DD5000CF52DF4F088319832A833B83C15DD040B4
:10DD6000A5019401CF52DF4F688179818A819B811F
:10DD7000C15DD0400F94DD304B015C01C751DF4FD6
:10DD8000288139814A815B81C95ED0400F94D92CAA
:10DD90002B013C01C351DF4F288139814A815B81CE
:10DDA000CD5ED040C701B6010F94D92C9B01AC01C8
:10DDB000C301B2010F94DD30C954DF4F688379830A
:10DDC0008A839B83C75BD040C351DF4F2881398151
:10DDD0004A815B81CD5ED040CF50DF4F6881798131
:10DDE0008A819B81C15FD0400F94D92C2B013C01CB
:10DDF000CC51DF4F288139814A815B81C45ED0409C
:10DE0000C501B4010F94D92C9B01AC01C301B2012F
:10DE10000F94DD302B013C01CC51DF4F288139813B
:10DE20004A815B81C45ED040C701B6010F94D92CF2
:10DE30006B017C01C751DF4F288139814A815B81A9
:10DE4000C95ED040CF50DF4F688179818A819B8144
:10DE5000C15FD0400F94D92C9B01AC01C701B60122
:10DE60000F94DD306B017C012091471530914815EE
:10DE70004091491550914A150F94D92C4B015C01E2
:10DE800020914B1530914C1540914D1550914E15E8
:10DE9000C301B2010F94D92C9B01AC01C501B4019F
:10DEA0000F94DE304B015C0120914F1530915015DD
:10DEB0004091511550915215C954DF4F68817981B5
:10DEC0008A819B81C75BD0400F94D92C9B01AC0108
:10DED000C501B4010F94DE304B015C01CF52DF4F1E
:10DEE000688179818A819B81C15DD0409058A7016A
:10DEF00096010F94D92CCF52DF4F688379838A83A0
:10DF00009B83C15DD040A3019201C353DF4F688161
:10DF100079818A819B81CD5CD0400F94D92C9B0163
:10DF2000AC01CF52DF4F688179818A819B81C15DCD
:10DF3000D0400F94DD30C353DF4F688379838A83E9
:10DF40009B83CD5CD040C954DF4F288139814A8101
:10DF50005B81C75BD040C452DF4F688179818A8181
:10DF60009B81CC5DD0400F94D92C9B01AC01C35355
:10DF7000DF4F688179818A819B81CD5CD0400F948D
:10DF8000DD309B01AC01C501B4010F94DE304B01C3
:10DF90005C0120E030E0A9010F940433181624F04E
:10DFA000B7FAB094B7F8B094A7019601C701B601CB
:10DFB0000F94D92C6B017C01A3019201C301B20122
:10DFC0000F94D92C9B01AC01C701B6010F94DE3030
:10DFD0006B017C01C954DF4F288139814A815B8103
:10DFE000C75BD040CA01B9010F94D92C9B01AC0189
:10DFF000C701B6010F94DE300F9449339B01AC0189
:10E00000C501B4010F94BA31AB01BC0185E09DE0BC
:10E010000E94B2638AE00E9440A18AE00E9440A16F
:10E02000EFEEFCE084918F010F5F1F4F882321F0FA
:10E030000E9440A1F801F6CF48E0CD53DF4F688140
:10E0400079818A819B81C35CD0400E9419A2EAEE4B
:10E05000FCE084918F010F5F1F4F882321F00E9405
:10E0600040A1F801F6CF48E0C953DF4F68817981BC
:10E070008A819B81C75CD04090580E9419A2E5EE2E
:10E08000FCE084918F010F5F1F4F882321F00E94D5
:10E0900040A1F801F6CFCB50DF4F688179818A81AA
:10E0A0009B81C55FD040905848E00E9419A28AE049
:10E0B0000E9440A1C652DF4F08811981CA5DD0403D
:10E0C00003301105D4F0ECECFCE084918F010F5F7C
:10E0D0001F4F882321F00E9440A1F801F6CF48E0AD
:10E0E000CB52DF4F688179818A819B81C55DD040A9
:10E0F0000E9419A28AE00E9440A1C851DF4F1881F6
:10E10000C85ED0401111E9C1C154DF4F2881398167
:10E110004A815B81CF5BD040CB56DF4F2883398368
:10E120004A835B83C559D040C953DF4F88819981A9
:10E13000AA81BB81C75CD040C756DF4F88839983D3
:10E14000AA83BB83C959D040C12CD12C60E8E62EEC
:10E150006FE3F62EC356DF4FC882D982EA82FB8274
:10E16000CD59D040CE018B569F4F0E94FB8BC75795
:10E17000DF4FC882D982EA82FB82C958D040C35798
:10E18000DF4F188219821A821B82CD58D040CD539E
:10E19000DF4F088119812A813B81C35CD040CF5673
:10E1A000DF4F088319832A833B83C159D040CE01B6
:10E1B00087579F4F0E94FB8BCB56DF4F28813981B9
:10E1C0004A815B81C559D040CD53DF4F28833983C5
:10E1D0004A835B83C35CD040C756DF4F4880598079
:10E1E0006A807B80C959D040C356DF4F88809980B0
:10E1F000AA80BB80CD59D040C757DF4F8881998115
:10E20000AA81BB81C958D040C154DF4F888399830C
:10E21000AA83BB83CF5BD040C357DF4F08811981EE
:10E220002A813B81CD58D040C954DF4F08831983E0
:10E230002A833B83C75BD040CF56DF4FC880D9804D
:10E24000EA80FB80C159D040A7019601C301B20109
:10E250000F94D92CC953DF4F688379838A839B83BA
:10E26000C75CD040C954DF4F288139814A815B8126
:10E27000C75BD040C501B4010F94D92C9B01AC0100
:10E28000C953DF4F688179818A819B81C75CD04007
:10E290000F94DD30C358DF4F688379838A839B8373
:10E2A000CD57D040C154DF4F288139814A815B81ED
:10E2B000CF5BD040C501B4010F94D92C4B015C0158
:10E2C000A7019601CD53DF4F688179818A819B81B7
:10E2D000C35CD0400F94D92C9B01AC01C501B401A3
:10E2E0000F94DD30CF57DF4F688379838A839B8318
:10E2F000C158D040C954DF4F288139814A815B81A0
:10E30000C75BD040CD53DF4F688179818A819B8183
:10E31000C35CD0400F94D92C6B017C01C154DF4FFA
:10E32000288139814A815B81CF5BD040C301B20132
:10E330000F94D92C9B01AC01C701B6010F94DD30BD
:10E34000CB57DF4F688379838A839B83C558D0403E
:10E35000CE0183589F4F0E94FB8BC757DF4F088128
:10E3600019812A813B81C958D040C357DF4F48806B
:10E3700059806A807B80CD58D040CF56DF4F88804F
:10E380009980AA80BB80C159D040C358DF4F888193
:10E390009981AA81BB81CD57D040C954DF4F888372
:10E3A0009983AA83BB83C75BD040CF57DF4F888157
:10E3B0009981AA81BB81C158D040C154DF4F888365
:10E3C0009983AA83BB83CF5BD040CB57DF4F888133
:10E3D0009981AA81BB81C558D040CD53DF4F888336
:10E3E0009983AA83BB83C35CD040CB56DF4FC880E0
:10E3F000D980EA80FB80C559D040C756DF4F48819D
:10E4000059816A817B81C959D040C356DF4F8881C9
:10E410009981AA81BB81CD59D0400093AF1210934E
:10E42000B0122093B1123093B2124092B3125092B4
:10E43000B4126092B5127092B6128092B712909296
:10E44000B812A092B912B092BA12C954DF4F088123
:10E4500019812A813B81C75BD0400093BB12109386
:10E46000BC122093BD123093BE12C154DF4F0881FD
:10E4700019812A813B81CF5BD0400093BF1210935A
:10E48000C0122093C1123093C212CD53DF4F0881C6
:10E4900019812A813B81C35CD0400093C312109341
:10E4A000C4122093C5123093C612C092C712D092E4
:10E4B000C812E092C912F092CA124093CB12509344
:10E4C000CC126093CD127093CE128093CF129093A2
:10E4D000D012A093D112B093D212CE51DF4F188137
:10E4E000C25ED040112309F465C2E9E0FCE08491EA
:10E4F0008F010F5F1F4F882321F00E9440A1F80178
:10E50000F6CFC553DF4FC880CB5CD040CA94DC2C1B
:10E51000C553DF4F1882CB5CD04000ECC154DF4FB5
:10E520000883CF5BD04019E7CD53DF4F1883C35C1E
:10E53000D04004E4C953DF4F0883C75CD0408E014C
:10E540000B561F4FCF54DF4F19830883C15BD04058
:10E550000C501109CD54DF4F19830883C35BD040A1
:10E560000C501109CB54DF4F19830883C55BD04091
:10E57000D7FC27C10D2D000F110BCE51DF4F198392
:10E580000883C25ED040212C312CC954DF4F188241
:10E59000C75BD040CE51DF4FE881F981C25ED040E9
:10E5A000E20DF31D21EA30E02C0F3D1FE20FF31FB7
:10E5B000008111817801EE0CFF1CEE0CFF1CEDE6D2
:10E5C000F0E0EC0FFD1FEE0DFF1D408051806280DA
:10E5D0007380CB52DF4F288139814A815B81C55DD1
:10E5E000D040C301B2010F94DD304B015C01E1E08A
:10E5F000F0E0EC0FFD1FEE0DFF1D84AD95ADA6AD57
:10E60000B7ADCB56DF4F88839983AA83BB83C559A7
:10E61000D040C052DF4FE881F981C05ED040E00FAA
:10E62000F11FEE0FFF1FEE0FFF1F41E050E04C0FF8
:10E630005D1FE40FF51F84AD95ADA6ADB7ADC7570F
:10E64000DF4F88839983AA83BB83C958D040C358BE
:10E65000DF4F188219821A821B82CD57D040CA54CC
:10E66000DF4F5881C65BD0405F93CB54DF4F88812A
:10E67000C55BD0408F93CC54DF4F9881C45BD040B2
:10E680009F93CD54DF4FA881C35BD040AF93CE544E
:10E69000DF4FB881C25BD040BF93CF54DF4FE881DA
:10E6A000C15BD040EF930DB71EB7045211090FB6EE
:10E6B000F8941EBF0FBE0DBFADB7BEB71196EFEAFF
:10E6C000F2E184E201900D928A95E1F70E94168BA7
:10E6D000C358DF4F288139814A815B81CD57D040B3
:10E6E000C301B2010F94DD307B018C010FB6F894A9
:10E6F000DEBF0FBECDBF9B01AC01C553DF4F6881AC
:10E70000CB5CD040C154DF4F7881CF5BD040CD533C
:10E71000DF4F8881C35CD040C953DF4F9881C75C0D
:10E72000D0400F9404331816A4F4C553DF4FE88289
:10E73000CB5CD040C154DF4FF882CF5BD040CD538B
:10E74000DF4F0883C35CD040C953DF4F1883C75CD9
:10E75000D04020E030E0A901C501B4010F9404339A
:10E7600087FD0CC0E6E0FCE084918F010F5F1F4F36
:10E77000882339F00E9440A1F801F6CF80E20E9480
:10E7800040A145E0C501B4010E9419A2C954DF4F60
:10E790000881C75BD0400F5FC954DF4F0883C75B58
:10E7A000D04014E0210E311CC752DF4F1881C95DE3
:10E7B000D040011708F4EECE8AE00E9440A1DA941E
:10E7C000D7CE8AE00E9440A1C652DF4F088119814E
:10E7D000CA5DD0400430110509F0ECC0EDEDFBE05E
:10E7E00084918F010F5F1F4F81110CC01E0115E92D
:10E7F000210E311C2E0129E8420E511C8E010358B6
:10E800001F4F1BC00E9440A1F801EACF80E20E9486
:10E8100040A145E0C501B4010E9419A2D394F4E0DF
:10E82000EF0EF11CC752DF4F2881C95DD040D216D0
:10E8300060F08AE00E9440A1CA94C7FCB7C06C2C6B
:10E84000660C7708E12CF12CD12CF701E60DF71DB1
:10E8500041EA50E04C0F5D1FE40FF51F808191816C
:10E860005C01AA0CBB1CAA0CBB1CE1E0F0E0EC0FA5
:10E87000FD1FEA0DFB1D44AD55AD66AD77ADD10171
:10E880004D935D936D937C931397C052DF4FE88156
:10E89000F981C05ED040E80FF91FEE0FFF1FEE0FA9
:10E8A000FF1F21E030E02C0F3D1FE20FF31F84AD6E
:10E8B00095ADA6ADB7ADF20180839183A283B383FA
:10E8C000D8011D921D921D921C9213971F930F93B6
:10E8D0005F924F923F922F92EDB7FEB7B4970FB66B
:10E8E000F894FEBF0FBEEDBFADB7BEB71196EFEA0D
:10E8F000F2E184E201900D928A95E1F70E94168B75
:10E90000EDE6F0E0EC0FFD1FEA0DFB1DD8012D91A7
:10E910003D914D915C9160817181828193810F94D1
:10E92000DD30C553DF4F2881CB5CD040C154DF4F71
:10E930003881CF5BD040CD53DF4F4881C35CD0409E
:10E94000C953DF4F5881C75CD0400F94DD304B0175
:10E950005C010FB6F894DEBF0FBECDBF20E030E003
:10E96000A9010F94043387FD51CFEAEDFBE08491B8
:10E970009F012F5F3F4F882309F44BCFCE5EDE4FC0
:10E980002883C251D140CF5EDE4F3883C151D14080
:10E990000E9440A1CE5EDE4F2881C251D140CF5EA1
:10E9A000DE4F3881C151D140F901E1CF8AE00E94A8
:10E9B00040A108C0C652DF4F08811981CA5DD0400E
:10E9C000012B21F08BEB9BE00F947327C851DF4F95
:10E9D0001881C85ED040111185C08CE0E3EFFEE0E5
:10E9E000DE01A358BF4F01900D928A95E1F781E0B7
:10E9F0008093840ECE0183589F4F0E94ADD2C355A1
:10EA0000DF4F288139814A815B81CD5AD0406091A6
:10EA1000F30E7091F40E8091F50E9091F60E0F9416
:10EA2000DD306B017C012DEB37E346E855EB0F94AD
:10EA3000043387FD4BC02DEB37E346E855E3C701B0
:10EA4000B6010F94742C18160CF440C0C755DF4F54
:10EA5000288139814A815B81C95AD0406091F70E83
:10EA60007091F80E8091F90E9091FA0E0F94DD30AE
:10EA70006B017C012DEB37E346E855EB0F94043333
:10EA800087FD24C02DEB37E346E855E3C701B60107
:10EA90000F94742C1816D4F0C554DF4F2881398197
:10EAA0004A815B81CB5BD0406091FB0E7091FC0E84
:10EAB0008091FD0E9091FE0E0F94DD30CB57DF4F0D
:10EAC000688379838A839B83C558D0408CE0FE019C
:10EAD000E358FF4FA3EFBEE001900D928A95E1F756
:10EAE00081E005C0C453DF4F8881CC5CD040809367
:10EAF000840E0E94A9B00E9441D58091840E81119C
:10EB00000E94A8B5CE5EDE4F0FB6F894DEBF0FBEF2
:10EB1000CDBFDF91CF911F910F91FF90EF90DF90CC
:10EB2000CF90BF90AF909F908F907F906F905F90AD
:10EB30004F903F902F900895DF92EF92FF920F93A6
:10EB40001F93CF93DF93CDB7DEB72C970FB6F89412
:10EB5000DEBF0FBECDBF182F0E9435DBD090840ED4
:10EB600080E00E9490B60E94C3B081E08093471875
:10EB7000111119C088E50E944BB7F82E89E50E9453
:10EB80004BB7082F8AE50E944BB7E82EF11006C05C
:10EB9000011113C0882369F0F02E10C0002369F022
:10EBA000F02E182F0BC0FF24F39401E0EE24E39421
:10EBB00002C0F82E082F11E001C010E00E9495B8A5
:10EBC000111105C0E11003C0F11006C02BC082E096
:10EBD0000E94849C1123C1F380E090E0A0E8B0E49F
:10EBE0008093ED069093EE06A093EF06B093F006A7
:10EBF0009C01AD016091FB0E7091FC0E8091FD0EA9
:10EC00009091FE0E0F94742C87FF0FC019821A8208
:10EC10001B821C82BE016F5F7F4F8DEE96E00E94CB
:10EC200012B203C00111D8CF0CC0111102C0FF20D5
:10EC3000A9F080E00E94849C112381F081E00E9471
:10EC4000849C0E94A8B51D821E821F8218861123F3
:10EC500069F080E090E0A5E3B3E412C00111EECFCB
:10EC60000E94A8B51D821E821F821886E110F1CF76
:10EC70008091FB0E9091FC0EA091FD0EB091FE0EC6
:10EC800089839A83AB83BC83BE016B5F7F4FCE01C8
:10EC900001960E9412B280E090E0A0EAB0E4898779
:10ECA0009A87AB87BC8711110BC0011109C0409135
:10ECB000F70E5091F80E6091F90E7091FA0E04C0A3
:10ECC00040E050E06BE373E44D835E836F837887AD
:10ECD00011110BC0F11009C04091F30E5091F40EC8
:10ECE0006091F50E7091F60E04C040E050E060EACD
:10ECF00070E449835A836B837C83AE01475F5F4F27
:10ED0000BE016B5F7F4FCE0101960E940EB28091D3
:10ED10004618809347188D2D0E9490B60E94A9B086
:10ED200083E080935B020E9441D52C960FB6F89445
:10ED3000DEBF0FBECDBFDF91CF911F910F91FF902E
:10ED4000EF90DF90089510923E0880914408882348
:10ED500031F00F94931881E699E70C94E3FB20912E
:10ED6000010230910202409155115091561160916B
:10ED7000571170915811C901840F951F2436310520
:10ED800024F4853691053CF416C02436310531F063
:10ED90008436910584F484E690E00DC04730510537
:10EDA0006105710514F0069706C04A3F5F4F6F4F2B
:10EDB0007F4F6CF4069690930202809301021092AA
:10EDC00055111092561110925711109258118091AE
:10EDD0000102909102028A3091053CF0883E23E0C6
:10EDE00092072CF087EE93E002C08AE090E09093C7
:10EDF00002028093010280E00C947D60CF93DF9348
:10EE000000D01F92CDB7DEB75C834B837A836983D2
:10EE1000BE016D5F7F4FCE0101960E94CCEE0F9038
:10EE20000F900F900F90DF91CF910895282F809130
:10EE3000551190915611A0915711B09158118130F0
:10EE40009048A105B10540F010925511109256114D
:10EE5000109257111092581180913308882331F085
:10EE6000809155118093D5061092521180912708F8
:10EE70001816FCF4082E000C990B821B91092091A6
:10EE8000D506022E000C330B2817390794F097FF94
:10EE900002C080E090E08093D506092E000CAA0BFA
:10EEA000BB0B8093551190935611A0935711B093BB
:10EEB00058118091D5066623A9F0909128088917EA
:10EEC00014F48093280820912808022E000C330B9C
:10EED0002C5F3F4F482F082E000C550B2417350789
:10EEE0001CF4845080932808089580915311863033
:10EEF000D8F496E0899FF0011124E657F94F20914C
:10EF00004502309146023183208340915511509142
:10EF10005611609157117091581142835383648345
:10EF200075838F5F80935311089583EA96E70C945D
:10EF3000E3FBE0915311EE2369F0E150E0935311AC
:10EF400086E0E89FF0011124E657F94F8081918116
:10EF50000C94E3FBEACF10925411EBCF0F931F9365
:10EF6000CF93DF9361E081E061DFD0912808C0E0BA
:10EF700001E61FE0D1111DC080914408811106C037
:10EF800080915B02882309F4B7C00AC08091D5063E
:10EF90008111F6CFE0DF80915211882389F3B3C04D
:10EFA00081E09091D506911180E024E04BEA5FE08A
:10EFB000A0C0D13009F580914408811106C080912C
:10EFC0005B02882309F498C00DC08091D50681307A
:10EFD000B1F785E392E90E94BCAE8091521188237B
:10EFE00071F391C081E09091D506913009F080E0F5
:10EFF00023E049E95FE07DC0D23059F580914408B3
:10F00000811106C080915B02882309F475C017C086
:10F010008091D5068230B1F70E942C82882319F0A6
:10F020000E94A9B807C048EB51E064E170E080E0BD
:10F0300090E0E4DE80915211882321F364C081E0E6
:10F040009091D506923009F080E020E24AE85FE036
:10F0500050C0D33059F580914408811106C0809189
:10F060005B02882309F448C017C08091D50683301D
:10F07000B1F70F942C11882319F00E94A9B807C08A
:10F0800048EB51E064E170E080E090E0B7DE809111
:10F090005211882321F337C081E09091D506933037
:10F0A00009F080E020E24BE65FE023C0D43021F598
:10F0B00080914408811105C080915B028823E1F0B2
:10F0C0000FC08091D5068430B9F710934411009396
:10F0D00043110E94C7B280915211882369F313C073
:10F0E00081E09091D506943009F080E020E249E774
:10F0F0005FE06C2F0E94B9B8CF5FDF5FC53009F0C9
:10F1000039CFC0932708DF91CF911F910F910895B8
:10F11000CF92DF92EF92FF920F931F93CF93DF93E3
:10F1200061E081E083DED0912808C0E00FE91EE0B5
:10F1300080EBE82E8EE0F82E98E5C92E9FE0D92EC0
:10F14000D1111DC080914408811106C080915B02DD
:10F15000882309F4A6C00AC08091D5068111F6CF94
:10F16000FADE80915211882389F3A2C081E0909148
:10F17000D506911180E024E04CE55FE08FC0D130EE
:10F1800019F580914408811106C080915B028823A3
:10F1900009F487C00FC08091D5068130B1F7D092B5
:10F1A0004411C09243110E94C7B28091521188232A
:10F1B00061F37EC081E09091D506913009F080E046
:10F1C00020E24EE45FE06AC0D23019F58091440835
:10F1D000811106C080915B02882309F462C00FC0D0
:10F1E0008091D5068230B1F7F0924411E09243113C
:10F1F0000E94C7B280915211882361F359C081E007
:10F200009091D506923009F080E020E243EA5EE07A
:10F2100045C0D33011F580914408811105C080911B
:10F220005B028823F1F10FC08091D5068330B9F7D6
:10F2300010934411009343110E94C7B28091521160
:10F24000882369F335C081E09091D506933009F0A9
:10F2500080E020E24EE85EE021C0D43011F58091DC
:10F260004408811105C080915B028823D1F00DC054
:10F270008091D5068430B9F788EA93EF0E94BCAE3E
:10F2800080915211882379F313C081E09091D506C3
:10F29000943009F080E023E044E85EE06C2F0E94A7
:10F2A000B9B8CF5FDF5FC53009F04ACFC0932708F8
:10F2B000DF91CF911F910F91FF90EF90DF90CF9052
:10F2C00008958F929F92AF92BF92CF92DF92EF926A
:10F2D000FF920F931F93CF93DF9361E081E0A6DD50
:10F2E000C091280800E09924939487ECE82E8DE0E3
:10F2F000F82E92EEC92E9DE0D92E2CEDA22E2DE0F7
:10F30000B22EC1111EC080914408811105C08091A8
:10F310005B028823B1F00AC08091D5068111F7CF36
:10F320001ADE80915211882391F32DC281E09091D1
:10F33000D506911180E024E048E75EE0602F0E944E
:10F34000B9B88091071390910813891B8F7009F049
:10F35000E6C1809155158111E2C18091561588232F
:10F3600021F080914A178111DAC1C13009F58091ED
:10F370004408811106C080915B02882309F45EC0B5
:10F380000DC08091D5068130B1F788E898E70E94DA
:10F39000BCAE80915211882371F3F5C181E0909148
:10F3A000D506913009F080E023E04AE65EE043C0F4
:10F3B000C23001F580914408811105C080915B0243
:10F3C0008823E1F10DC08091D5068230B9F78EE235
:10F3D00090EC0E94BCAE80915211882379F3D3C186
:10F3E00081E09091D506923009F080E023E04EE56F
:10F3F0005EE021C0C33011F580914408811105C041
:10F4000080915B028823D1F00DC08091D5068330B6
:10F41000B9F78EEA97E70E94BCAE8091521188231B
:10F4200079F3B1C181E09091D506933009F080E085
:10F4300023E040E55EE0602F0E94B9B810E0D4E020
:10F440008090D708811018C0609135027091360203
:10F45000072E000C880B990B0F947A2C9B01AC01A2
:10F460006091D3087091D4088091D5089091D60806
:10F470000F94742C87FD37C0CD1334C0809144089D
:10F48000811105C080915B02882361F120C08091C9
:10F49000D5068C13F7CF8091E00883FD67C18110FA
:10F4A00065C12091AA113091AB11809135029091E4
:10F4B0003602281739070CF059C117DD8AEB9FE88F
:10F4C0000E94E3FB809152118823E1F25CC181E04C
:10F4D0009091D5069C1380E020E240E45EE0602F2E
:10F4E0000E94B9B8DF5F80915615882309F4C5C022
:10F4F00080914A17882309F49CC080915515882370
:10F5000079F1CD1357C080914408811106C08091D4
:10F510005B02882309F44EC01AC08091D5068C1373
:10F52000F6CF109255158BEF94E10E941251B092D4
:10F530004411A09243110E94C7B26FEF8FEC9DE07F
:10F540000E9472AA80915211882309F31CC181E0A4
:10F550009091D5069C1380E020E244E35EE027C052
:10F56000CD1328C080914408811105C080915B02B1
:10F57000882301F114C08091D5068C13F7CFD09267
:10F580004411C09243110E94C7B26FEF81EE9DE01B
:10F590000E9472AA80915211882341F3F4C081E045
:10F5A0009091D5069C1380E020E248E15EE0602F58
:10F5B0000E94B9B8DF5FCD1337C080914408811134
:10F5C00005C080915B02882379F123C08091D50624
:10F5D0008C13F7CF0E94D5FF8091B20880938106EB
:10F5E000109282060E94985D0F942C1D0E948C96AA
:10F5F0001092D2081092D10810922D026FEF86EE71
:10F600009DE00E9472AA91DC809152118823C9F278
:10F61000BAC081E09091D5069C1380E020E24DE0D5
:10F620005EE0602F0E94B9B8DF5F112309F44BC080
:10F630006EC011116CC0CD1345C08091440881117A
:10F6400006C080915B02882309F43CC00DC0809104
:10F65000D5068C13F6CF87E690E90E94BCAE809168
:10F660005211882371F38FC081E09091D5069C13CD
:10F6700080E023E04FEF5DE022C0111148C0CD13C0
:10F6800021C080914408811105C080915B028823CC
:10F69000C9F00DC08091D5068C13F7CF87E690E9AD
:10F6A0000E94BCAE80915211882379F36CC081E036
:10F6B0009091D5069C1380E023E044EF5DE0602F3D
:10F6C0000E94B9B8DF5FCD1321C080914408811139
:10F6D00005C080915B028823C9F00DC08091D506DA
:10F6E0008C13F7CF84EA9BEF0E94BCAE809152113D
:10F6F000882379F348C081E09091D5069C1380E07F
:10F7000023E045E25EE0602F0E94B9B8DF5F0F5F43
:10F71000CF5F053009F0F5CDD093270834C0C13054
:10F7200011F580914408811105C080915B02882306
:10F73000D1F00DC08091D5068130B9F787E598EFFB
:10F740000E94BCAE80915211882379F31CC081E0E5
:10F750009091D506913009F080E023E043E75EE028
:10F76000602F0E94B9B811E0D2E06ACE9092541195
:10F7700089ED9EE80E94E3FBF0924411E092431170
:10F780000E94C7B29FCEDF91CF911F910F91FF9042
:10F79000EF90DF90CF90BF90AF909F908F900895A3
:10F7A000AF92BF92CF92DF92EF92FF920F931F938F
:10F7B000CF93DF935C017B0120E030E0F501E20FA5
:10F7C000F31FE491EE2319F02F5F3F4FF7CFF701BE
:10F7D000CF018E199F0941914111FACF04E110E048
:10F7E000081B11093327021713071CF0DD24D394DB
:10F7F00002C082E0D82E80910D1890E06D2D70E04F
:10F800006F5F7F4F0F94C633C62EC6E0C60F809140
:10F810004018C81750F08091421890E02C2F30E02B
:10F820002B503109821793079CF5D0E0E114F104C5
:10F83000C1F18AE30F94CE1C82E0D8120FC0CC0D28
:10F8400080914018C81768F12091421830E08C2F41
:10F8500090E00B97281739071CF423C0DD2309F12A
:10F86000802F880F080F000F00934318C09344188F
:10F8700080E20F94CE1CC701DF91CF911F910F91B1
:10F88000FF90EF90DF90CF90BF90AF900D943A191A
:10F8900010924318C0934418C5010F942D19D1E05C
:10F8A000C5CFDF91CF911F910F91FF90EF90DF9027
:10F8B000CF90BF90AF9008950F93CF939CE0899F16
:10F8C000802D112491E0980F9093250F2CE0280FA4
:10F8D0002093260F4091401850E030E02E5F3F4FBC
:10F8E0002417350744F1292F30E04091421850E0A9
:10F8F0002417350704F56623A9F091E090932C189E
:10F90000C3E0C80F0BE020E84C2F60E08CE098E1EA
:10F910000E94C44B882319F08C2F0F94251C109241
:10F920002C1803C081E080932C188091260F109230
:10F93000431880934418CF910F910895CF92DF928E
:10F94000EF92FF920F93CF93DF93982F862F6A0148
:10F950007901692FB1DF909140188091260F8917A6
:10F9600008F453C0909142188091250F981708F41D
:10F970004CC0002359F060E070E0F701E60FF71F7C
:10F98000E491EE2351F06F5F7F4FF7CFD701BD01B8
:10F990006E197F098D918111FACFC62FD4E1D61B44
:10F9A000F6018491882339F00F940819D81BFFEFD2
:10F9B000CF1ADF0AF5CF8AE30F94CE1CDD2329F09E
:10F9C00080E20F94CE1CD150F9CF8091260F6AEFC0
:10F9D000C69F602D1124605860934318809344188B
:10F9E000C701002349F0DF91CF910F91FF90EF9075
:10F9F000DF90CF900D942D19DF91CF910F91FF9053
:10FA0000EF90DF90CF900D943A19DF91CF910F9145
:10FA1000FF90EF90DF90CF9008950F93CF93DF93F7
:10FA2000CDB7DEB7ED85FE856081718182819381DE
:10FA30000F942232CB010E94BC8A00E09C014985D0
:10FA40005A8568858F817ADFDF91CF910F91089574
:10FA50008CE0E2EDFEE0A3EFBEE001900D928A950E
:10FA6000E1F70895CF92DF92EF92FF92CF93DF9369
:10FA7000EC01C090AE06D090AF06E090B006F090DA
:10FA8000B106A7019601688179818A819B810F94D3
:10FA9000742C87FF04C0C882D982EA82FB82C0909E
:10FAA000B206D090B306E090B406F090B506A70178
:10FAB00096016C817D818E819F810F94742C87FFCC
:10FAC00004C0CC82DD82EE82FF82C0901B02D09007
:10FAD0001C02E0901D02F0901E02A70196016881B1
:10FAE00079818A819B810F940433181624F4C8828B
:10FAF000D982EA82FB82C0901F02D0902002E0905F
:10FB00002102F0902202A70196016C817D818E81F5
:10FB10009F810F940433181624F4CC82DD82EE8288
:10FB2000FF82C090B606D090B706E090B806F0907D
:10FB3000B906A7019601688579858A859B850F940A
:10FB4000742C87FF04C0C886D986EA86FB86C090DD
:10FB50002302D0902402E0902502F0902602A70113
:10FB60009601688579858A859B850F9404331816DC
:10FB700024F4C886D986EA86FB86DF91CF91FF9070
:10FB8000EF90DF90CF900895CF93DF9380E50E94B0
:10FB90004BB7882351F00E9414B76093740E709392
:10FBA000750E8093760E9093770E89E40E944BB782
:10FBB000882381F00E9414B72CEA35EC47E25EE31B
:10FBC0000F94D92C6093700E7093710E8093720E07
:10FBD0009093730E84E40E944BB7882381F00E94B7
:10FBE00014B72CEA35EC47E25EE30F94BA31609328
:10FBF0006C0E70936D0E80936E0E90936F0EE9E312
:10FC0000FBE28491EF012196882321F00E9440A11C
:10FC1000FE01F7CF4091740E5091750E6091760EF3
:10FC20007091770E87E090E10E94B2632CEA35EC88
:10FC300047E25EE36091700E7091710E8091720EDA
:10FC40009091730E0F94BA31AB01BC0183E090E147
:10FC50000E9495632CEA35EC47E25EE360916C0EFE
:10FC600070916D0E80916E0E90916F0E0F94D92C45
:10FC7000AB01BC018FEF9FE00E9495638AE0DF91AA
:10FC8000CF910C9440A10F931F93CF93DF938C01DE
:10FC9000E9E3FBE28491EF012196882321F00E94A1
:10FCA00040A1FE01F7CFB80182EF9FE00E940F64F0
:10FCB00082E20E9440A18AE00E9440A181E0DF919F
:10FCC000CF911F910F9108958091D70881111AC08B
:10FCD0006091350270913602072E000C880B990B4B
:10FCE0000F947A2C9B01AC016091D3087091D408D9
:10FCF0008091D5089091D6080F94742C881F88277E
:10FD0000881F089580E008958F929F92AF92BF92CE
:10FD1000CF92DF92EF92FF920F931F93CF93DF93D7
:10FD20001F92CDB7DEB75C014B016A01122FE5E4EB
:10FD3000F0E184917F019FEFE91AF90A882321F00D
:10FD40000E9440A1F701F5CF8091E00883FD36C005
:10FD500020E030E0A901F601608171818281938108
:10FD60000F94742C882351F1F090D708F11024C01F
:10FD70002091AA113091AB118091350290913602F9
:10FD800028173907CCF4EEE1FBE284918F010F5F75
:10FD90001F4F882321F00E9440A1F801F6CFECE12B
:10FDA000F0E184918F010F5F1F4F882309F494C005
:10FDB0000E9440A1F801F5CF0F946B2491E090933D
:10FDC000CC0680915515882321F0109255159093FB
:10FDD000CB068BEF94E10E941251002339F081E0B1
:10FDE0008093541189ED9EE80E94E3FB0E9435DB6D
:10FDF00090E1E3EFFEE0ABEBB6E001900D929A9557
:10FE0000E1F720E030E0A901F50160817181828194
:10FE100093810F94742C882321F056DF882309F4F2
:10FE200053C082E08983B401CE0101960F94A122D0
:10FE300020E030E0A901F601608171818281938127
:10FE40000F94742C882399F0002351F081E0809363
:10FE5000541182E89EE80E94E3FB80E00F94610465
:10FE600040E050E060E271E4C6010F9434240023C6
:10FE700039F081E0809354118DE79DE80E94E3FB07
:10FE800061E0812F0F94C62480E00F9461040F94E9
:10FE9000D40364E670E080E090E00E94F28A0E9461
:10FEA000DB50DC01CB0180529C46AB4FBF4F8093AF
:10FEB000560790935707A0935807B093590710928D
:10FEC0005011FF24F39408C040E050E060E772E472
:10FED000C5010F943424A5CF8F2D0F90DF91CF91C2
:10FEE0001F910F91FF90EF90DF90CF90BF90AF9058
:10FEF0009F908F900895CF92DF92EF92FF920F9391
:10FF00001F93CF93DF9300D01F92CDB7DEB77C0154
:10FF10006B01042F10915011109256071092570741
:10FF200010925807109259071092501180E00E94C9
:10FF3000419611110F946B2461E0802F0F94C62419
:10FF40000E9495B820E030E0A901F701608171813D
:10FF5000828193810F94742C882341F1112339F00D
:10FF600081E0809354118DE79DE80E94E3FB81E0DE
:10FF70008093810780918107882351F0112341F0FC
:10FF800060E0802F0F94C62481E00F946104F2CFCB
:10FF900081E08093541186E29DE80E94E3FB40E0FB
:10FFA00050E060EC70E4C7010F9434248DDE8111C1
:10FFB00041C0F60180819181A281B38189839A83B6
:10FFC000AB83BC8311E0C12CD12C80EAE82E81E404
:10FFD000F82E20E030E0A90169817A818B819C8133
:10FFE0000F940433181674F4109354118FEC9CE89A
:10FFF0000E94E3FB40E050E060E87FE3CE01019621
:020000021000EC
:100000000F94342410928107109354111092BA0661
:1000100080E39FE80E94E3FB8091BA06811104C04F
:1000200081E00F946104F8CFC982DA82EB82FC820E
:10003000813079F281E08093541185EC99EA0E9435
:10004000E3FB8091C7069091C806A091C906B091C4
:10005000CA068093FF0E9093000FA093010FB093F8
:10006000020F8093F1069093F206A093F306B093EB
:10007000F4060E9493F280E090E0A8ECB2E4898359
:100080009A83AB83BC83AE014F5F5F4F6FEB76E02B
:100090008BEB96E00E940EB280E090E0A0EAB0E424
:1000A00089839A83AB83BC83BE016F5F7F4F83ECF0
:1000B00096E00E9412B20E949577EBE0F0E1849105
:1000C0008F010F5F1F4F882321F00E9440A1F8018C
:1000D000F6CF8091CB06882349F08091561588236E
:1000E00019F081E0809355151092CB061092CC0642
:1000F0000F900F900F900F90DF91CF911F910F9164
:10010000FF90EF90DF90CF900895CF93DF9383E43B
:1001100097E118D089EE95E1892B41F48AEC95E1BD
:1001200011D089EA95E1DF91CF910CC0C0E0D0E019
:10013000CE018050994E06D06F97CA3C8EEFD807FB
:10014000B9F7ECCF21E334E0FC013183208304963E
:100150000C9486B80F931F93CF93DF938C01EB0120
:100160008991882319F00E9440A1FACFEFECFFE0BB
:100170008491EF012196882321F00E9440A1FE0185
:10018000F7CFF801ED5AFF4F80819181A281B381B1
:1001900088279927AF77BB27CD01AA27BB27BC01AA
:1001A000660F771F6078682B062E000C770B880B84
:1001B000990B0E94FFA18DE00E9440A18AE0DF918F
:1001C000CF911F910F910C9440A18F929F92AF926B
:1001D000BF92EF92FF920F931F93CF93DF937C0117
:1001E0008A01EB018991882319F00E9440A1FACF7E
:1001F000E0EBFFE08491EF012196882321F00E943B
:1002000040A1FE01F7CFC7010F94951FDC0120E14B
:1002100036E041EC50E00F94BE304B015C01F70139
:100220008789908DA18DB28D2227382F492F5A2F83
:10023000D8010F94BE309B01AC01C501B4010F94ED
:100240008030CA01B9014AE00E9499A18AE0DF9199
:10025000CF911F910F91FF90EF90BF90AF909F9023
:100260008F900C9440A12F923F924F925F926F9289
:100270007F928F929F92AF92BF92CF92DF92EF9236
:10028000FF920F931F93CF93DF93EC011B01290182
:100290003A01670178010F94951FDC0120E136E0F7
:1002A00041EC50E00F94BE304B015C015E2D4D2DB2
:1002B0003C2D2227C301B2010F9471309B01AC0188
:1002C000C501B4010F9480302F8B388F498F5A8F1E
:1002D000AE01495E5F4F63E9CE010F94D91DA601BF
:1002E000B101CE01DF91CF911F910F91FF90EF905F
:1002F000DF90CF90BF90AF909F908F907F906F9046
:100300005F904F903F902F9060CFAF92BF92CF926F
:10031000DF92EF92FF920F931F93CF93DF931F9281
:10032000CDB7DEB77C016B018A0159018091AC1118
:10033000811119C0F701808191810F943A3089832E
:10034000F60181936F01BE016F5F7F4FC5010E946F
:1003500088F1F701408151814F5F5F4F51834083A6
:100360000150110939F70F90DF91CF911F910F9133
:10037000FF90EF90DF90CF90BF90AF9008958F9255
:100380009F92AF92BF92CF92DF92EF92FF920F9324
:100390001F93CF93DF931F921F92CDB7DEB7E091EB
:1003A000AC11E1114AC059016C018B017B01E40ED3
:1003B000F51E0E151F0509F440C0F60180809180DE
:1003C000F80161918F016983C4016A830F943A3007
:1003D0006A81681729F1C4010F946330C4010F9436
:1003E0003A3099818917E1F0E9E3FBE284918F01CA
:1003F0000F5F1F4F882321F00E9440A1F801F6CF24
:10040000E5E5F0E184918F010F5F1F4F882321F014
:100410000E9440A1F801F6CF81E08093AC110DC09D
:10042000BE016F5F7F4FC5010E9488F1F601808198
:100430009181019691838083BCCF0F900F90DF91C3
:10044000CF911F910F91FF90EF90DF90CF90BF90D1
:10045000AF909F908F9008958F929F92AF92BF928E
:10046000CF92DF92EF92FF920F931F93CF93DF9380
:10047000CDB7DEB7CB54D1090FB6F894DEBF0FBEAF
:10048000CDBF19AA1AAA1BAA1CAA80E390E3A0E375
:10049000B0E08DA79EA7AFA7B8AB23961FAE1EAE48
:1004A000239784E690E021969FAF8EAF219710921C
:1004B000AC119E012F5B3F4F44E050E0BE01635DF5
:1004C0007F4FCE01CF965BDF21968EAD9FAD2197FA
:1004D000029621969FAF8EAF219723961FAE1EAE38
:1004E000239781E02C968FAF2C979E012F5B3F4F77
:1004F00041E050E0BE01655B7F4FCE01CF963FDF0C
:100500009E012F5B3F4F40E150E063E07FE0CE0172
:10051000CF9635DF9E012F5B3F4F40E150E06DEB02
:100520007EE0CE01CF962BDF9E012F5B3F4F40E157
:1005300050E06DEA7EE0CE01CF9621DF9E012F5B79
:100540003F4F44E050E069EA7EE0CE01CF9617DFEE
:100550009E012F5B3F4F44E050E065EA7EE0CE0114
:10056000CF960DDF9E012F5B3F4F44E050E061EAE4
:100570007EE0CE01CF9603DF9E012F5B3F4F44E02C
:1005800050E06DE97EE0CE01CF96F9DE9E012F5B53
:100590003F4F44E050E069E97EE0CE01CF96EFDEC8
:1005A0009E012F5B3F4F44E050E065E97EE0CE01C5
:1005B000CF96E5DE9E012F5B3F4F40E150E065E8BE
:1005C0007EE0CE01CF96DBDE9E012F5B3F4F4CE0FD
:1005D00050E063E774E0CE01CF96D1DE80E090E09A
:1005E000A0E2B1E489A79AA7ABA7BCA79E012F5BA5
:1005F0003F4F44E050E0BE01675D7F4FCE01CF9694
:10060000BEDE2B961FAE2B9719AA1AAA1BAA1CAAEC
:1006100083E02A968FAF2A9729968FAF29979E015C
:100620002F5B3F4F41E050E0BE01665B7F4FCE0144
:10063000CF96A5DE9E012F5B3F4F44E050E0BE0108
:100640006F5C7F4FCE01CF969ADE9E012F5B3F4FAE
:1006500041E050E0BE01675B7F4FCE01CF968FDE59
:100660009E012F5B3F4F41E050E0BE01685B7F4F32
:10067000CE01CF9684DE1AE0115061F09E012F5B0F
:100680003F4F44E050E0BE016F5C7F4FCE01CF96FC
:1006900076DEF2CF23960EAD1FAD239721968EAD59
:1006A0009FAD219790934C0280934B029E012F5B4C
:1006B0003F4F44E050E06FED7EE0CE01CF965FDE2D
:1006C00023961FAF0EAF23979E012F5B3F4F44E24F
:1006D00050E06FEA72E1CE01CF9651DE83E02896BA
:1006E0008FAF289727968FAF27971DA21EA21FA214
:1006F00018A619A21AA21BA21CA219AA1AAA1BAAFE
:100700001CAA9E012F5B3F4F41E050E0BE01695B98
:100710007F4FCE01CF9633DE9E012F5B3F4F41E0EE
:1007200050E0BE016A5B7F4FCE01CF9628DE9E016E
:100730002F5B3F4F44E050E0BE016F5D7F4FCE0125
:10074000CF961DDE9E012F5B3F4F44E050E0BE017F
:100750006B5D7F4FCE01CF9612DE0AE010E00150B4
:10076000110961F09E012F5B3F4F44E050E0BE0154
:100770006F5C7F4FCE01CF9602DEF1CF26961FAE83
:1007800026978FEF25968FAF25979E012F5B3F4FC2
:1007900041E050E0BE016B5B7F4FCE01CF96EFDDB5
:1007A0009E012F5B3F4F41E050E0BE016C5B7F4FED
:1007B000CE01CF96E4DD19AA1AAA1BAA1CAA1CE036
:1007C00011509E012F5B3F4F44E050E0112339F060
:1007D000BE016F5C7F4FCE01CF96D1DDF1CF60E8D7
:1007E0007EE0CE01CF96CBDD9E012F5B3F4F44E0F4
:1007F00050E06CE77EE0CE01CF96C1DD9E012F5B1D
:100800003F4F44E050E068E77EE0CE01CF96B7DD91
:10081000C12C80E8D82E8BE3E82E85E4F82E812CBD
:10082000912C90E8A92E9FE3B92E11112EC09E01A4
:100830002F5B3F4F44E050E064E77EE0CE01CF966F
:100840009EDD9E012F5B3F4F44E050E060E77EE07D
:10085000CE01CF9694DD9E012F5B3F4F44E050E0E8
:100860006CE67EE0CE01CF968ADD89AA9AAAABAA71
:10087000BCAA9E012F5B3F4F44E050E0BE016F5C7D
:100880007F4FCE01CF967BDD22C0C9AADAAAEBAAA0
:10089000FCAA9E012F5B3F4F44E050E0BE016F5C1D
:1008A0007F4FCE01CF966BDD19AA1AAA1BAA1CAAEC
:1008B00004E0015061F09E012F5B3F4F44E050E0A7
:1008C000BE016F5C7F4FCE01CF9659DDF2CF1F5F27
:1008D000153009F0AACF84E190E09EAF8DAF9E0164
:1008E0002F5B3F4F42E050E0BE01635C7F4FCE0183
:1008F000CF9645DD9E012F5B3F4F44E050E068E618
:100900007EE0CE01CF963BDD9E012F5B3F4F44E062
:1009100050E064E67EE0CE01CF9631DD9E012F5B94
:100920003F4F44E050E060E67EE0CE01CF9627DD09
:1009300080E290E09CAF8BAF9E012F5B3F4F42E087
:1009400050E0BE01655C7F4FCE01CF9618DD249646
:100950001FAE249780E090E0A0E4B0E48D8F9E8FDE
:10096000AF8FB8A380E090E0A4E3B2E4898F9A8FC0
:10097000AB8FBC8F1D8A1E8A1F8A188E198A1A8A0D
:100980001B8A1C8A1D861E861F86188A80E090E0BE
:10099000A0E5B1E489879A87AB87BC871D821E8258
:1009A0001F82188680E090E0A0E0B1E489839A83FA
:1009B000AB83BC839E012F5B3F4F41E050E0BE0103
:1009C0006D5B7F4FCE01CF96DADC9E012F5B3F4FF0
:1009D00044E050E0BE01635E7F4FCE01CF96CFDC96
:1009E0009E012F5B3F4F44E050E0BE01675E7F4FAA
:1009F000CE01CF96C4DC9E012F5B3F4F44E050E018
:100A0000BE016B5E7F4FCE01CF96B9DC9E012F5B9E
:100A10003F4F44E050E0BE016F5E7F4FCE01CF9666
:100A2000AEDC9E012F5B3F4F44E050E0BE01635FB0
:100A30007F4FCE01CF96A3DC9E012F5B3F4F44E05A
:100A400050E0BE01675F7F4FCE01CF9698DC9E01DC
:100A50002F5B3F4F44E050E0BE016B5F7F4FCE0104
:100A6000CF968DDC9E012F5B3F4F44E050E0BE01EE
:100A70006F5F7F4FCE01CF9682DC9E012F5B3F4F91
:100A800041E050E061ED7EE0CE01CF9678DC10E0F1
:100A900011110CC08091CD0E9091CE0EA091CF0E71
:100AA000B091D00E89AB9AABABABBCAB9E012F5BC8
:100AB0003F4F44E050E0BE016F5C7F4FCE01CF96C8
:100AC0005EDC1F5F153021F78091DB149091DC1400
:100AD0009AAF89AF9E012F5B3F4F42E050E0BE01CD
:100AE000675C7F4FCE01CF964ADC8091661490916F
:100AF00067149AAF89AF9E012F5B3F4F42E050E0F1
:100B0000BE01675C7F4FCE01CF9639DC8091F11337
:100B10009091F2139AAF89AF9E012F5B3F4F42E055
:100B200050E0BE01675C7F4FCE01CF9628DC1AAE45
:100B300019AE9E012F5B3F4F42E050E0BE01675C63
:100B40007F4FCE01CF961BDC1AAE19AE9E012F5BF4
:100B50003F4F42E050E0BE01675C7F4FCE01CF9631
:100B60000EDC1AAE19AE9E012F5B3F4F42E050E003
:100B7000BE01675C7F4FCE01CF9601DC80917C1374
:100B800090917D139AAF89AF9E012F5B3F4F42E05A
:100B900050E0BE01675C7F4FCE01CF96F0DB1AAE0E
:100BA00019AE9E012F5B3F4F42E050E0BE01675CF3
:100BB0007F4FCE01CF96E3DB1AAE19AE9E012F5BBD
:100BC0003F4F42E050E0BE01675C7F4FCE01CF96C1
:100BD000D6DB1AAE19AE9E012F5B3F4F42E050E0CC
:100BE000BE01675C7F4FCE01CF96C9DB1AAE19AE4E
:100BF0009E012F5B3F4F42E050E0BE01675C7F4F9C
:100C0000CE01CF96BCDB8091BB149091BC14A09117
:100C1000BD14B091BE1488279927AF77BB27B8AF12
:100C2000AFAB9E012F5B3F4F42E050E0BE01695CDD
:100C30007F4FCE01CF96A3DB80914614909147144D
:100C4000A0914814B091491488279927AF77BB2702
:100C5000B8AFAFAB9E012F5B3F4F42E050E0BE010B
:100C6000695C7F4FCE01CF968ADB9E012F5B3F4FA1
:100C700044E050E06CE57EE0CE01CF9680DB9E0143
:100C80002F5B3F4F44E050E068E57EE0CE01CF9619
:100C900076DB13E0115078F084E0189FB001112446
:100CA000645B714F9E012F5B3F4F44E050E0CE01EB
:100CB000CF9665DBEFCF19AA1AAA1BAA1CAA1CE1C2
:100CC000115061F09E012F5B3F4F44E050E0BE01A8
:100CD0006F5C7F4FCE01CF9652DBF2CF19AA1AAAD2
:100CE0001BAA1CAA14E0115061F09E012F5B3F4F1C
:100CF00044E050E0BE016F5C7F4FCE01CF963FDBFA
:100D0000F2CF8091AC1181114CC02196EEACFFACBA
:100D1000219723968EAD9FAD23979EAB8DAB84E636
:100D200090E021969FAF8EAF21979E012F5B3F4FA2
:100D300044E050E06EED73E0CE01CF9620DB9E01E3
:100D40002F5B3F4F42E050E0BE016B5C7F4FCE0116
:100D5000CF9615DBE9E3FBE284918F010F5F1F4F14
:100D6000882321F00E9440A1F801F6CFB701645614
:100D700071098FE790E10E94F6634DA95EA960E0DA
:100D800070E082E790E10E947863EFE6F0E1849101
:100D90008F010F5F1F4F882321F00E9440A1F801AF
:100DA000F6CF9091AC1181E08927C55BDF4F0FB67C
:100DB000F894DEBF0FBECDBFDF91CF911F910F9191
:100DC000FF90EF90DF90CF90BF90AF909F908F906B
:100DD0000895CF93DF93CDB7DEB72C970FB6F89475
:100DE000DEBF0FBECDBF8091F30E9091F40EA091A7
:100DF000F50EB091F60E89839A83AB83BC83809104
:100E0000F70E9091F80EA091F90EB091FA0E8D8325
:100E10009E83AF83B8878091FB0E9091FC0EA091CA
:100E2000FD0EB091FE0E89879A87AB87BC870E9422
:100E3000E4E40E9451D480E00E946BB281E00E9401
:100E40006BB282E00E946BB20E94DADA0E944EE539
:100E50004CE050E063EF7EE0CE0101960F94EF335B
:100E6000892B51F02C960FB6F894DEBF0FBECDBF84
:100E7000DF91CF910C9441D52C960FB6F894DEBF3C
:100E80000FBECDBFDF91CF91089561E0FC0180815D
:100E90000C940F4F8EBD0DB407FEFDCF08958FEF5C
:100EA0008EBD0DB407FEFDCF8EB508950F931F9331
:100EB000CF93DF938B010E94DB50EB01F0DF8F3F7C
:100EC00049F00E94DB506C1B7D0B60177107B0F37B
:100ED00080E001C081E0DF91CF911F910F910895D3
:100EE000CF92DF92EF92FF921F93CF93DF9300D0C8
:100EF0001F92CDB7DEB76C01162FFC019281892FAE
:100F0000806A86958CBD90FD03C081E0963009F41F
:100F100080E08DBD60E0F601808129833A834B83B8
:100F20005C830E940F4F6CE271E0C601BFDF812F2E
:100F30008064B0DF88E1E82EF12C5C814B813A813E
:100F40002981DA01C9010E2C04C0B695A7959795A1
:100F500087950A94D2F729833A834B835C839ADF7F
:100F6000F8E0EF1AF10829813A814B815C8188EF22
:100F7000E8168FEFF80629F7112321F0183021F039
:100F80008FEF03C085E901C087E884DF1C3009F4D6
:100F900086DF10E084DFF601838387FF04C01F3FF4
:100FA00011F01F5FF7CF0F900F900F900F90DF9110
:100FB000CF911F91FF90EF90DF90CF9008950F9306
:100FC0001F93CF93DF93EC0189018C81833039F03B
:100FD00089E0440F551F661F771F8A95D1F79A0144
:100FE000AB0168E1CE017CDF882311F086E02FC0E1
:100FF0008EEF8EBD80E090E00DB407FEFDCFF801CE
:10100000E80FF91F20812EBD0DB407FEFDCF218111
:101010002EBD0296811522E0920771F70DB407FEEE
:10102000FDCF8FEF37DF8FEF35DF39DF8B838F71A8
:10103000853029F083E18983CE0127DF09C068E587
:1010400072E0CE0133DF182F811106C087E189835A
:10105000CE011BDF10E00FC020E030E0A9016DE001
:10106000CE013EDF811103C01ADF882311F086E133
:10107000EECFCE010ADF812FDF91CF911F910F912B
:101080000895EF92FF920F931F93CF93DF93EC019C
:1010900079018C81833039F089E0440F551F661F38
:1010A000771F8A95D1F79A01AB0161E1CE0118DF74
:1010B000882329F084E08983CE01E7DE35C00E94D1
:1010C000DB508B01ECDE8B838F3F49F40E94DB50B9
:1010D000601B710B6D327140A8F381E103C08E3F3C
:1010E00039F08FE08983CE01D0DE8FEFD3DE1CC0D4
:1010F0008FEF8EBDF701D701A150BE4F0DB407FE93
:10110000FDCF9EB591938EBDEA17FB07B9F70DB4DD
:1011100007FEFDCF8EB58C93C2DEC1DECE01B5DEFB
:101120008FEFB8DE81E001C080E0DF91CF911F91A9
:101130000F91FF90EF9008958F929F92AF92BF9280
:10114000CF92DF92EF92FF92CF93FC01C080D180CB
:10115000E280F38020E030E0A901C701B6010F94DE
:10116000742C87FF08C0C701B601905820E030E01A
:1011700048EC52E406C020E030E048EC52E4C701FD
:10118000B6010F94D92C0F9422326B017C01603A86
:10119000F6E87F07F1E08F07910584F020EA36E852
:1011A00041E050E00F94A230CA01B9012AE030E0DA
:1011B00040E050E00F94A230605D01C060E26093B7
:1011C000CD0680E1C81687E2D806E104F10494F068
:1011D000C701B60120E137E240E050E00F94A230B1
:1011E000CA01B9012AE030E040E050E00F94A2309B
:1011F000605D01C060E26093CE06E8EECE16E3E0EB
:10120000DE06E104F10494F0C701B60128EE33E0F4
:1012100040E050E00F94A230CA01B9012AE030E06A
:1012200040E050E00F94A230605D01C060E2609346
:10123000CF06C701B60124E630E040E050E00F944D
:10124000A2308AE0882E912CA12CB12CCA01B901C0
:10125000A50194010F94A230605D6093D0068EE2E8
:101260008093D106C701B601A50194010F94A23065
:10127000C62FCA01B901A50194010F94A230605D87
:101280006093D206C05DC093D3068DEC96E0CF91FB
:10129000FF90EF90DF90CF90BF90AF909F908F9096
:1012A00008958F929F92AF92BF92CF92DF92EF926A
:1012B000FF92CF9320E030E048EC52E4FC016081E3
:1012C0007181828193810F94D92C0F9422326B010A
:1012D0007C0197FF0AC0F094E094D094C094C11CA4
:1012E000D11CE11CF11C8DE201C08BE28093CD0684
:1012F000C701B60120E137E240E050E00F94A23090
:101300008AE0882E912CA12CB12CCA01B901A5012B
:1013100094010F94A230605D6093CE06C701B601C0
:1013200028EE33E040E050E00F94A230CA01B9014A
:10133000A50194010F94A230605D6093CF06C701B0
:10134000B60124E630E040E050E00F94A230CA013C
:10135000B901A50194010F94A230605D6093D0069D
:101360008EE28093D106C701B601A50194010F94C6
:10137000A230C62FCA01B901A50194010F94A23071
:10138000605D6093D206C05DC093D3068DEC96E09D
:10139000CF91FF90EF90DF90CF90BF90AF909F9054
:1013A0008F9008958F929F92AF92BF92CF92DF92CB
:1013B000EF92FF92FC01C080D180E280F38020E0B8
:1013C00030E0A901C701B6010F94742C87FF04C057
:1013D000C701B601905802C0C701B6010F9422326E
:1013E0006B017C016031F7E27F078105910584F094
:1013F00020E137E240E050E00F94A230CA01B90189
:101400002AE030E040E050E00F94A230605D01C07F
:1014100060E26093CF0688EEC81683E0D806E10448
:10142000F10494F0C701B60128EE33E040E050E04B
:101430000F94A230CA01B9012AE030E040E050E048
:101440000F94A230605D01C060E26093D006E4E6D4
:10145000CE16D104E104F10494F0C701B60124E6EC
:1014600030E040E050E00F94A230CA01B9012AE018
:1014700030E040E050E00F94A230605D01C060E2D7
:101480006093D106FAE0CF16D104E104F1049CF098
:101490008AE0882E912CA12CB12CC701B601A501A0
:1014A00094010F94A230CA01B901A50194010F94CF
:1014B000A230605D01C060E26093D206C701B60150
:1014C0002AE030E040E050E00F94A230605D60938D
:1014D000D3068FEC96E0FF90EF90DF90CF90BF9017
:1014E000AF909F908F90089520E030E040E251E46B
:1014F000FC0160817181828193810F94D92C0F94BA
:1015000022329B0177FF06C022273327261B370B89
:101510008DE201C08BE28093CE06C90168EE73E0D4
:101520000F94C633CB01EAE0F0E0BF010F94C6335D
:10153000805D8093CF06C90164E670E00F94C633E6
:10154000CB01BF010F94C633805D8093D006C901E3
:10155000BF010F94C633282FCB01BF010F94C633B0
:10156000805D8093D1068EE28093D206205D209329
:10157000D3068EEC96E008959C0197FD0EC084364C
:10158000910584F064E670E00F94C633CB016AE005
:1015900070E00F94C633805D06C031952195310906
:1015A0008DE201C080E28093D1062A30310564F0DB
:1015B000EAE0F0E0C901BF010F94C633CB01BF01DF
:1015C0000F94C633805D01C080E28093D206C901CA
:1015D0006AE070E00F94C633805D8093D30681ED9E
:1015E00096E00895CF92DF92EF92FF926B017C011B
:1015F00083E3C816D104E104F10470F082E3C81A51
:10160000D108E108F10862E370E080E090E00E9418
:10161000A3500E94A799ECCFC701B6010E94A35026
:10162000FF90EF90DF90CF900C94A7994F925F922C
:101630006F927F928F929F92AF92BF92CF92DF92E2
:10164000EF92FF92CF93DF93CDB7DEB728970FB617
:10165000F894DEBF0FBECDBF2496AEADBFAD2497CC
:101660008D919D910D90BC91A02D89839A83AB8320
:10167000BC832296EEADFFAD2297C080D180E28080
:10168000F380AEADBFAD8D909D90AD90BC902E8D92
:101690003F8D48A159A1C501B4010F94D92C2B014C
:1016A0003C012AA53BA54CA55DA5C701B6010F9439
:1016B000D92C9B01AC01C301B2010F94DE302B0188
:1016C0003C012EA93FA948AD59AD69817A818B8132
:1016D0009C810F94D92C9B01AC01C301B2010F94E2
:1016E000DE306D837E838F8398872AA13BA14CA136
:1016F0005DA1C501B4010F94D92C2B013C012EA58D
:101700003FA548A959A9C701B6010F94D92C9B013F
:10171000AC01C301B2010F94DE302B013C012AADB4
:101720003BAD4CAD5DAD69817A818B819C810F941D
:10173000D92C9B01AC01C301B2010F94DE302B0107
:101740003C012A8D3B8D4C8D5D8DC501B4010F94FC
:10175000D92C4B015C012EA13FA148A559A5C70179
:10176000B6010F94D92C9B01AC01C501B4010F94B3
:10177000DE306B017C012AA93BA94CA95DA96981D6
:101780007A818B819C810F94D92C9B01AC01C7017C
:10179000B6010F94DE30EEADFFAD608371838283BE
:1017A00093838D819E81AF81B8852296EEADFFAD8A
:1017B000229780839183A283B3832496AEADBFAD7D
:1017C00024974D925D926D927C92139728960FB656
:1017D000F894DEBF0FBECDBFDF91CF91FF90EF90A9
:1017E000DF90CF90BF90AF909F908F907F906F9041
:1017F0005F904F9008954F925F926F927F928F9279
:101800009F92AF92BF92CF92DF92EF92FF920F938F
:101810001F93CF93DF9300D01F92CDB7DEB78C011B
:10182000DC014D905D906D907C90139714968D9097
:101830009D90AD90BC90179718968D919D910D90AD
:10184000BC91A02D89839A83AB83BC83A3019201B1
:10185000C301B2010F94D92C6B017C01A501940145
:10186000C501B4010F94D92C9B01AC01C701B6018D
:101870000F94DE306B017C0129813A814B815C81C0
:10188000CA01B9010F94D92C9B01AC01C701B60163
:101890000F94DE300F9449339B01AC0160E070E09F
:1018A00080E89FE30F94BA316B017C019B01AC018E
:1018B000C301B2010F94D92CF80160837183828334
:1018C0009383A7019601C501B4010F94D92CD801C7
:1018D00014966D937D938D939C931797A701960112
:1018E00069817A818B819C810F94D92CF801608762
:1018F0007187828793870F900F900F900F90DF91E1
:10190000CF911F910F91FF90EF90DF90CF90BF90FC
:10191000AF909F908F907F906F905F904F900895C1
:10192000DB01833070F494E0899FF0011124E45BC3
:10193000F14FAB01770F660B770B408351836283C6
:101940007383813089F018F08230D9F008952FEF39
:1019500030E00F94E13320ED37E040E050E00F94A9
:10196000A230B9018EE219C02FEF30E00F94E133BD
:1019700020ED37E040E050E00F94A230B9018DE255
:101980000CC02FEF30E00F94E13320ED37E040E062
:1019900050E00F94A230B9018CE20C94DC4F1F93FD
:1019A000CF93DF9360E085E00E941677D0912808FE
:1019B000C0E012E0D11109C080915B028823D9F107
:1019C00021E041E065EE72E115C0D13049F480912B
:1019D0005B02882381F120E041E06CED72E10AC0F6
:1019E000D23061F480915B02882329F120E041E04C
:1019F0006BEC72E18C2F0E9400EF1DC0D33049F4D4
:101A000080915B028823B9F020E041E069EC72E14B
:101A1000F1CFD43081F480915B02882351F021E032
:101A200040E06EEB72E18C2F0E9400EF8C2F0F9440
:101A3000451910935B02CF5FDF5FC53009F0BACF65
:101A4000C0932708DF91CF911F9108951F93CF93E3
:101A5000DF9360E085E00E941677D0912808C0E00F
:101A600012E0D11109C080915B028823D9F121E0F5
:101A700041E061EB72E115C0D13049F480915B0225
:101A8000882381F120E041E068EA72E10AC0D230A7
:101A900061F480915B02882329F120E041E06AE94A
:101AA00072E18C2F0E9400EF1DC0D33049F4809169
:101AB0005B028823B9F020E041E068E972E1F1CFF0
:101AC000D43081F480915B02882351F021E040E022
:101AD0006DE872E18C2F0E9400EF8C2F0F94451956
:101AE00010935B02CF5FDF5FC53009F0BACFC093C0
:101AF0002708DF91CF911F9108951F93CF93DF9314
:101B000060E085E00E941677D0912808C0E012E0DE
:101B1000D11109C080915B028823D9F121E041E015
:101B200060E872E115C0D13049F480915B028823EE
:101B300081F120E041E060E772E10AC0D23061F457
:101B400080915B02882329F120E041E06FE572E19A
:101B50008C2F0E9400EF1DC0D33049F480915B02AE
:101B60008823B9F020E041E060E572E1F1CFD430A4
:101B700081F480915B02882351F021E040E065E42C
:101B800072E18C2F0E9400EF8C2F0F944519109357
:101B90005B02CF5FDF5FC53009F0BACFC093270883
:101BA000DF91CF911F9108951F93CF93DF9360E052
:101BB00085E00E941677D0912808C0E012E0D1118C
:101BC00009C080915B028823D9F121E041E068E3FC
:101BD00072E115C0D13049F480915B02882381F114
:101BE00020E041E068E272E10AC0D23061F4809105
:101BF0005B02882329F120E041E06BE172E18C2F48
:101C00000E9400EF1DC0D33049F480915B0288230D
